:020000040001F9
:10020000F80B0020690801003D090100515B010065
:10021000715B0100915B0100D15B0100B15B0100EA
:10022000000000000000000000000000952901000F
:100230003D090100000000003D0901003D090100E9
:100240000000000000000000000000007D340100FC
:10025000000000003D090100000000000000000057
:100260003D0901003D0901003D0901003D09010072
:10027000000000003D0901003D0901003D090100A9
:100280003D0901003D0901000000000000000000E0
:100290003D0901003D0901000000000000000000D0
:1002A0003D09010000000000000000003D090100C0
:1002B0003D0901003D0901003D0901003D09010022
:1002C0003D0901003D0901003D0901003D09010012
:1002D0003D090100000000003D0901000000000090
:1002E0003D090100000000003D0901000000000080
:1002F0003D090100000000000000000000000000B7
:10030000000000003D0901000000000000000000A6
:1003100000000000000000000000000000000000DD
:10032000000000003D090100000000000000000086
:1003300000000000000000000000000000000000BD
:100340003D09010000015F5F00000000FE0B00009E
:10035000252A0100800600000000000000000000C7
:10036000000000000000000000000000401200201B
:100370000000000001015F5F030100001F01000099
:1003800085060100000000000000000001000000E0
:10039000010000000000000000000000000000005C
:1003A0000000000070000000D45F01008000000029
:1003B000000F000001000000D104010001015F5F97
:1003C000040100001F010000F3070100000000000D
:1003D000000000000000000001000000000000001C
:1003E000000000000000000000000000DF5F0100CE
:1003F000400000000507000001000000DF060100CA
:1004000038B50025054C29462046D4F80024C4F808
:10041000045405F046FCC4F8005438BD200C0020FC
:1004200013B511460022CDE9002242680346382A5E
:10043000046844D194F82820022A19D01AB900F08F
:1004400047F902B010BD21482468D0F80404013AED
:10045000CDE90040082A35D8DFE802F0050A0E137E
:10046000181D22272C006A46184600F02EF9E8E7EE
:10047000184600F018F9E4E76A46184600F016F945
:10048000DFE76A46184600F00BF9DAE76A461846D5
:1004900000F00FF9D5E76A46184600F00DF9D0E7ED
:1004A0006A46184600F00BF9CBE76A46184600F09A
:1004B00009F9C6E76A46184600F00EF9C1E76FF081
:1004C0008000BEE76FF08500BBE700BF200C002076
:1004D0002DE9F04F05680446A1B0002D40F0AA8038
:1004E0002022294602A805F0DCFB12AF2022294673
:1004F0000AA805F0D6FB38222946384605F0D1FB7C
:10050000E26904F11C039846B2B10426E26A04F1E0
:100510002C03EAB10425EEB96FF08306304621B012
:10052000BDE8F08F002EF1D053F8041D3246013E95
:100530000029F7D01646E9E70326F5E7002DEAD0B3
:1005400053F8041D2A46013D0029F7D01546E2E77D
:100550000325F5E738233A460021606805F0DEFB05
:100560003828D9D14FF00109CDE90270334F0DF190
:10057000080A04F1100B4E45D7F800141CD10DF1F8
:1005800028094B46002008EB850EC64533D108B13B
:10059000C7F80014A3683146C7F804340AAA2B46EA
:1005A00002A8FFF73DFF00270646BD4209F10809F2
:1005B00038D1FFF725FFB1E75BF8043FC1F5806252
:1005C000D81C20F00300904204D9FFF719FF6FF008
:1005D0008C06A3E70844CA19C7F8000449466068B6
:1005E000019205F09BFB019ACAF80C0009F1010980
:1005F0004AF8082FBFE758F804CFC1F5806A0CF11C
:10060000030222F00302524503F1080305D87818CB
:1006100043E9020C11440120B7E70028D5D0C7F800
:100620000014D2E7394659E90223606805F08BFBD4
:100630000137BAE76FF0850670E700BF200C002095
:1006400008B528220021024805F02BFB002008BD38
:100650002810002010B5044C0F222046034905F055
:10066000FBFA204610BD00BF51100020F607010024
:1006700008B50121024803F0D1FA002008BD00BFEF
:100680005010002008B5FFF7DBFF40B9FFF7E2FF8D
:10069000FFF7EEFF18B9BDE8084003F02DBB08BD19
:1006A0006FF0850070476FF0850070476FF0850030
:1006B00070476FF0850070476FF0850070476FF0EE
:1006C000850070476FF0850070476FF085007047B8
:1006D000D1E9000103F0F0BA6FF085007047F0B582
:1006E00003680546B3F57D7FA7B007D040F2F53229
:1006F000934207D06FF0850027B0F0BD01F0E8FC11
:100700000020F9E700243C22214607A8CDE9024455
:10071000CDE90444069405F0C4FA3C22214617A80A
:10072000169405F0BEFAEA69019405F11C0302B3C0
:100730000426EA6A05F12C033AB30424731E012B44
:1007400052D8012C50D80423002168680DEB030215
:1007500005F0E4FA04281AD06FF08000CCE7002EF0
:10076000E7D053F8041D3246013E0029F7D0164663
:10077000DFE70326F5E7002CE0D053F8041D2246FE
:10078000013C0029F7D01446D8E70324F5E7022EF0
:1007900016D16E69402E29D806AF33463A4601215C
:1007A000686805F0BBFA8642D6D1CDE9027602A987
:1007B00044B92246019801F062FE044620469BE7B8
:1007C0000021F5E72B6A402BC6D816AACDE90423F1
:1007D000019804AA01F053FEDDE904230446002138
:1007E000686805F0B0FAE9E7012085E76FF0890055
:1007F00082E7002070474D62656420544C532033DB
:100800002E352E3000000000000000000000000027
:1008100000000000000000000000000000000000D8
:10082000D430000001000000407C01008010002056
:100830004A000000407C0100200C00200000000065
:10084000407C0100000C002000000000A8110020E6
:10085000C4050000200C002018010000000C00203E
:100860000800000002F084BC08B572B6002383F3D0
:100870001488BFF36F8F83F30A8883F30B88BFF369
:100880005F8F254B5A6A22F480325A62D3F8942043
:1008900022F00102C3F89420BFF34F8FBFF36F8F94
:1008A0001E4A9A6000F058F81D4B83F309881D4BCF
:1008B00083F30A8883F30B881B4B15A1D1E9000150
:1008C000C3E9000100F0EEF8184B19498B4212D32E
:1008D0000020184B18498B4218D303F00FF8186802
:1008E00050F82240586840F822400132986882420D
:1008F000F5D30C33EAE70022F8E71C6844F822003D
:1009000001325C68A242F8D30833E4E70022F8E73A
:10091000A5EDF5FEA5EDF5FE00ED00E000020100FD
:10092000F80B002000040020F80B0020280801002C
:100930004C0801004C08010064080100EFF3088036
:10094000EFF309812DE9F00F6B46724600F094F940
:1009500008B0FFF787FFFEE738B572B6002383F3D0
:10096000138883F311884FF0FF30274A03F12001E9
:100970000133102B42F82100F8D100234FF0FF344F
:10098000214A03F160010133102B42F82140F8D1D4
:10099000012200251D4B29465A60C3F84843C3F87D
:1009A000084303F580535A60C3F84843C3F808432B
:1009B000A3F55043C3F800558022C3F808431448F8
:1009C00005F06FF929468022124805F06AF9124BAA
:1009D0002946C3F800558022C3F808430F4805F0A4
:1009E00060F9802229460E4805F05BF90D4BC3F8EB
:1009F00008454FF05023C3F8084362B6BFF34F8F4A
:100A0000BFF36F8F38BD00BF00E100E00040015030
:100A100080800050808100500090005080900050F5
:100A2000809100500070015008B5EFF31083012B46
:100A30000C4A07D1126ABFF34F8F511C4A424A41F8
:100A4000104608BD01F086FB00B172B6126ABFF312
:100A50004F8F531C5A425A4101F07CFB0028EFD0C3
:100A600062B6EDE70080FF0008B5EFF31083012BBD
:100A70000B4A06D1D269BFF34F8F02F00102104634
:100A800008BD01F067FB00B172B6D269BFF34F8FAA
:100A900002F0010201F05EFB0028F0D062B6EEE742
:100AA0000080FF00694A10B5D2F8D03043F002034D
:100AB000C2F8D03001F04EFB30B14FF0502300228D
:100AC000C3F81421C3F8182101F053FB28B1012207
:100AD0005F4BC3F8382AC3F878254FF47F02D2F869
:100AE0003031D2F83421BFF34F8FC3F30B03092BFE
:100AF00005D1012A1EBF0122554BC3F8782501F00C
:100B000038FB18B10E22534BC3F8E42E01F022FB40
:100B100030B100224E4BC3F80C270122C3F8102736
:100B20000022D30003F57F03D3F80013BFF34F8FE8
:100B3000013108D0D3F800130132D3F80433B2F5F1
:100B4000807F0B60EDD1EFF31084FFF78DFF00285D
:100B50004DD0BFF34F8F404BD3F80024012AFBD177
:100B6000C3F80425D3F80024012AFBD1012C03D0BB
:100B700001F0F0FA00B172B6FFF776FF58B1374ACC
:100B8000D36923F00103D361BFF34F8F324AD2F808
:100B90000034012BFBD1FFF747FF68B12F4A136ADE
:100BA00023F0FF0343F020031362BFF34F8F2A4A61
:100BB000D2F80034012BFBD1012C03D001F0CAFA8A
:100BC00000B162B60022244BC3F80425D3F80024F8
:100BD000012AFBD1BFF34F8F1C49214BCA6802F495
:100BE000E0621343CB60BFF34F8F00BFFDE7FFF719
:100BF0001BFF0028ADD1154AD2F88C3043F4406376
:100C0000C2F88C304FF47F03D3F83021D3F834315D
:100C1000BFF34F8FC2F30B02092A16D1013B022BFF
:100C200002D8104AD35C83B10C480F4903680A4AC2
:100C30008B420CBF5A230023C2F8103EC36A8B427A
:100C40000CBF5A230023C2F8003E10BD00ED00E0A7
:100C50000040005000A00350009003500080FF00AF
:100C60000400FA054C350100FA50FA507C22014983
:100C700004F0F2BFDC18002038B51D46374B384C65
:100C80005B68C3F308032360EFF30383C4E9012027
:100C90006365C2F3801302F00C020C2AE16038D1C4
:100CA0000BB9EFF3898120222E48216104F0D4FF93
:100CB00025B1202229462C4804F0CEFF274B9A6A02
:100CC000A265D96AE165986B206602F4004060660F
:100CD000586BA06602F08000E0669A62D962D3F891
:100CE000E4202267D3F8E810616702F04001A167B1
:100CF000C3F8E42000F06AF80E211C4801F04BFA1A
:100D00002268D31E042B1CD8DFE803F0090F12154C
:100D1000180013B9EFF38881C5E70146C3E70C213A
:100D20001348BDE8384001F036BA12211148F8E7FF
:100D30000B211148F5E70D211048F2E70E2110486C
:100D4000EFE70F2A98BF1421BDE8384089BF25215D
:100D50000C480D48103A01F0C9BB00BF00ED00E09F
:100D6000DC180020F0180020101900204F35010079
:100D70005D350100693501007B35010086350100D4
:100D800093350100A1350100B53501002DE9F3418E
:100D900006460F460C4DD5F82C80C04710F00104D4
:100DA000FBD1394630466B69984740B9C047C30705
:100DB000FCD42B6A019302B0BDE8F04118472046ED
:100DC00002B0BDE8F08100BFDC35010010B5094C70
:100DD0000020A3689847236902209847A46A4FF42B
:100DE000E1310120A0472346BDE810400121152034
:100DF000184700BFDC35010010B5044C0020236902
:100E00009847E368BDE81040184700BFDC35010093
:100E1000064B82B01868002382B262F30F03000C05
:100E200060F31F43184602B0704700BF1C36010034
:100E3000014B1869704700BF84100020014B5869AE
:100E4000704700BF8410002038B50C4D0C4695F853
:100E5000203013B94FF0FF3038BD0A46014628460E
:100E600000F06CFF064B984205D00B3B9842F1D145
:100E700000206C61F0E76FF00100EDE784100020C6
:100E80000B00AD0BF0B51B4E054696F820300C4616
:100E900091B01BB94FF0FF3011B0F0BD00F06043CE
:100EA000B3F1005F21D100230A460146304600F02D
:100EB00031FC114B98421AD00B3B9842EAD1346175
:100EC00011E0A71B402F28BF4027A9193A466846C2
:100ED00004F0C2FE39466846FFF7D4FF0028DBD194
:100EE0004036B442EDD80020D6E70026F9E76FF08F
:100EF0000100D1E7841000200B00AD0BC3B2012B21
:100F000010B540F096804DF6C023994270D028D895
:100F1000B1F5615F6FD011D8B1F5965F6DD008D88B
:100F2000B1F5966F6BD0B1F5166F6BD06FF007000F
:100F30005DE0B1F5165FF9D1454B33E047F612237A
:100F4000994262D007D8B1F5964F61D0B1F5E14F23
:100F5000ECD1404B26E0B1F5164FE7D14FF41D031D
:100F600020E03D4B994255D011D8B1F5E13F54D026
:100F700007D8B1F5614F53D0B1F5963FD6D1374B75
:100F800010E0B1F5613FD1D14FF06C730AE0B1F5DB
:100F9000612F48D0324B994248D0B1F5E12FC5D1ED
:100FA0004FF0E86310F4E06F46D110F4404103D0F5
:100FB000B1F5804F43D1102110F4405203D0B2F567
:100FC000805F3FD10E2210F4403003D0B0F5403F97
:100FD0003BD10120234C20766276E361A1760A435F
:100FE00024681043C4F82435C4F86C05002010BDF3
:100FF0004FF46503D6E71C4BD4E71C4BD2E74FF404
:101000009E23CFE74FF41D23CCE74FF40003C9E73D
:10101000174BC7E74FF08063C4E74FF0EB73C1E7AE
:101020004FF46B03BEE74FF07063BBE74FF08053A4
:10103000B8E76FF00300DAE76FF00800D7E76FF06A
:101040000A00D4E76FF00900D1E76FF00B00CEE79C
:101050000050270000C0750090D0030000903A01B6
:1010600040420F008410002000F03A0000B013004E
:1010700000A04E0010B5114C204600F0D5FD002117
:10108000206884F8201000F04DFF226842F30732F8
:10109000002A11DB012153099B0003F1604303F592
:1010A0006143D3F8800202F01F0201FA02F2024308
:1010B000C3F88022D3F88032002010BD84100020B5
:1010C00010B5264C002120688EB000F01DFF22686C
:1010D00042F30732002A12DB012053099B0003F17F
:1010E000604303F56143D3F8801202F01F0200FA57
:1010F00002F221EA0202C3F88022D3F880322422CD
:10110000002105A804F0CDFDD4E902124FF0FF3311
:10111000CDE90133CDE903334FF0EB730B93072394
:1011200001A88DF8363001F054F8014600220B4832
:1011300000F03AFA0A4B98420DD10C9B0020238311
:101140001B0CA3760B9BC4E90400E361012384F824
:1011500020300EB010BD6FF00100FAE784100020BF
:101160000000AD0B7FB500250C46C0F808511646AF
:10117000D0F80821D0F8002222F02002C0F8002286
:10118000104AC0F8082301F074F8A560256104F145
:101190004C03D3E8EF1F21F47F0121F47041C3E831
:1011A000E21F002AF5D110222946684604F079FD95
:1011B000042368468DF800300196D4E9001398475F
:1011C00004B070BD10020A0000F01F03400909D1ED
:1011D000074A02EB8303D3F80012064A0A40C3F819
:1011E000002270470022803352F82330FFDE00BF18
:1011F00000258450F0F8FCFF2DE9F04F804690F870
:1012000004A05020664F0E4600FB0A70416885B06E
:1012100049B113F0020304D0836B002B00F0B280BD
:101220000123009300E000914FF0500909FB0A737D
:10123000DB6CD90600F1A6804FF0010BB3180293C6
:10124000029BB34200F0A78006F06043039398F836
:101250000450D8F8004009FB05739A6B9AB9039BB8
:10126000B3F1005F40F09980019200F0A1FD09FB0D
:101270000572D16C204601F0010100F0C8FF28B9C9
:1012800000F09EFDE3E701230193EEE7516C334646
:101290000029BCBFD4F84C155164019A42B109FB36
:1012A00005713078D1E90E23D054D1E90E321344C0
:1012B0001BB1C4F84435C4F848B50022C4F8202155
:1012C000D4F82011C4F85821D4F85811C4F850218A
:1012D000D4F850210822C4F80025009AE2B14FF456
:1012E0008003C4F80433C4F808B000F069FD50234B
:1012F00003FB0A72516800294BD1D26C120748D502
:1013000003FB0A734C33D3E8EF1F21F00801C3E855
:10131000E21F002A36D0F6E7C4F808B0019300F0C7
:101320004FFD09FB0572D16C019B01F001012046C4
:10133000019300F06CFF8446019BD4F84C05D4F86F
:101340004425BCF1000F0DD19342F0D005EB85058B
:1013500007EB0515D1B100F02BFD2946204600F022
:10136000CDFFC2E705EB8505934207EB0515F1D1EB
:101370000028EFD100F01CFD2946204600F0BEFFFA
:1013800000F01EFD074805B0BDE8F08FC4F80CB0B2
:10139000E1E7013654E70448F5E70448F3E700BF06
:1013A000581900200800AD0B0000AD0B0400AD0B78
:1013B000430904D10123034A83409360704700230B
:1013C0009B60FFDE0025845000F01F0340090BD115
:1013D000084A02EB8302D2F80012074B0B4043F09D
:1013E0000303C2F8003270470022803352F82330E2
:1013F000FFDE00BF00258450F0F8FCFF2DE9F84324
:1014000091F8303005460C4690F804800F6853BBC5
:101410005023DFF85091781C03FB0893DE6C46F0F4
:101420000072DA6404D03846FFF7C2FFFFF7CCFF42
:101430006068411C01D0FFF7C7FE94F82C30012BE7
:1014400011D1502303FB0893E06846F02066421C4C
:10145000DE6401D0FFF7B8FEA068431C03D0FFF79D
:10146000A7FFFFF7B1FF94F82F0038B950223D4B8A
:1014700002FB0833DA6C42F08072DA6494F82CC014
:1014800094F82D1094F82E202B68D4F828E041EA27
:101490000C010A43E668D4E90198C3F824E5C3F8CF
:1014A0006C2550B9BCF1010FC3F80C75C3F8149545
:1014B00004BFC3F80885C3F81065D3F8682503F2A4
:1014C0006458012A08BFDA60D3F86425012A13D1D1
:1014D000082149F64046244FC3F8001547F001079C
:1014E0005A60D8F800309BBB2B68D3F88024C3F82F
:1014F00080240022C3F8002500212B6894F83220B4
:10150000C3F81011D3F81001C3F82011D3F820014B
:10151000C3F82411D3F82401C3F84411D3F84401CB
:10152000C3F85811D3F8581143F307335201002B75
:10153000D2B212DB0D49C81880F8002301225809E5
:1015400003F01F0302FA03F341F82030BDE8F883EB
:101550004020B847013EC4D1C6E7054903F00F0358
:10156000CA54F3E7581900202036010000E100E0DA
:1015700014ED00E000F01F0340090BD1084A02EB14
:101580008302D2F80012074B0B4043F00203C2F86B
:10159000003270470022803352F82330FFDE00BF54
:1015A00000258450F0F8FCFF2DE9F34790465022C7
:1015B00090F80490514C02FB09FA04EB0A070D461F
:1015C00097F848100646002940F0858009EB89000D
:1015D00004EB001004F065FB2B69AA6944F80A309B
:1015E0006B69BB6302B1013A502303FB0943DA6321
:1015F0002A6A042A81BFEA699A610022DA6195F8B1
:101600003130B8F1000F37D083F001073F0233B11A
:10161000502303FB0943DA6C42F00102DA645023E1
:1016200003FB09440123C4F8048084F8483034687B
:10163000D4F84C2112BB29463046FFF7DFFE0822C2
:10164000002334688DF80730C4F800250DF1070237
:10165000C4F84425C4F8483501230A25A360E36093
:10166000D4F85831002B38D1254B402043F00103EA
:101670009847013DF4D128E04746C8E708224FF0DB
:101680006409C4F8002563601D4B43F0010AD4F8D7
:101690004431F3B9D4F82431DBB94FF42070D0478A
:1016A000B9F10109F3D14B460022C4F84C21D4F81A
:1016B0004C11C4F81021D4F81011C4F84421D4F806
:1016C0004411C4F80025002BB5D10E4802B0BDE886
:1016D000F0870123E8E70C48F8E70023C4F820313D
:1016E0009845D4F82021C4F80035084B08BF0023E2
:1016F0001F4333680648C3F80473E7E7581900200E
:10170000203601000100AD0B0C00AD0B10020A00E9
:101710000000AD0B2DE9F04784460F469E46164665
:101720000579002A51D04FF0500ADFF8AC80D0F88C
:1017300000900AFB058ADAF8044074B96BB9DAF84C
:101740002C50002D43D1CAF82C20FFF755FD04463C
:10175000CAF82C502046BDE8F0871EF0030F07D0D2
:10176000734632463946BDE8F0476046FFF744BD50
:1017700007F06043B3F1005F4FF0500414D104FB55
:10178000058400F015FBE26A1AB1144C00F018FB56
:10179000E0E7C4E90A7605EB8505484608EB051144
:1017A00000F0B7FD0E4CF1E704FB0584A36B83B199
:1017B00000F0FEFAE36A002BE7D1E36C012243F06C
:1017C0000203C4E90A76E364E5E7064CC2E7034C8A
:1017D000C0E7054CBEE700BF581900200B00AD0B59
:1017E0000000AD0B0600AD0B0A00AD0B2DE9F84370
:1017F00050230679284D046803FB0653D4F804737C
:10180000DA6AC4F8087322B92448C4F80473BDE83E
:10181000F88306EB860005F14C024FEA001802EB54
:101820000012D2E8EFCF4CF0080CC2E8E0CF00285D
:10183000F7D10122E26031B3D96C01EA02094946CD
:10184000204600F0E4FC0028FAD000F0B1FAB9F12B
:10185000000F1CD1D4F8203153B10123E360D4F838
:101860005831002BFBD0204605EB080100F046FD67
:1018700000F0A6FA0023C4F82031D4F82021502229
:1018800002FB0655EB620648C4F80473BFE7D4F8C0
:101890005831002BE7D1EBE7581900200500AD0BBC
:1018A0000000AD0B2DE9F84390F80480484F08EB99
:1018B0008806360106F14C0504683D44D5E8EF3F43
:1018C00043F48052C5E8E02F0028F7D1DB047BD435
:1018D000480705D5502303FB08739B69002B75D07F
:1018E0003C4B3E44C4F808330823C4F800350023B9
:1018F000C4F81031D4F81021C4F84C31D4F84C217C
:10190000C4F844310A03D4F844318B0303F4804310
:1019100002F400524903134301F400410B43D5E89C
:10192000EF2F1A43C5E8E12F0029F8D14FF05009F5
:1019300009FB0879D9F80830BBB9D9F8043063B984
:10194000D5E8EF3F23F47F0323F47043C5E8E23F7B
:10195000002AF5D12048BDE8F8830321304600F085
:1019600063FCD9F80830002BEAD0D4F804335907C7
:1019700013D5502303FB08735A6872B1DB6C1A034A
:101980000BD5D5E8EF3F23F40023C5E8E23F002A5A
:10199000F7D10621304600F047FC502303FB0873C3
:1019A000DB6CDB0401D40D48D5E7D4F84C310BB91E
:1019B00001232360502303FB08735B68002BF2D0E4
:1019C000044BC4F80433EEE70548C4E70548C2E712
:1019D0005819002010020A000200AD0B0000AD0BE8
:1019E0000B00AD0B0800AD0B2DE9F84F056801F0B9
:1019F0006043D5F804A3B3F1005F90F804B08946C2
:101A00001746C5F808A37CD15023404E03FB0B6357
:101A10009A6852B15B68002B5ED1D5F81021002A7C
:101A20005AD0C5F81031D5F81031502404FB0B649E
:101A3000E269C4E90297002A3CD00BEB8B0897427D
:101A40004FEA081824D24FF0000B3A46A1694846E5
:101A5000C4E902BB04F000F9E269A069D21BC11914
:101A6000E26104F0C3F863686BB1B04449463A469A
:101A7000404600F0EAFBE36C990404D55A4641461F
:101A80002846FFF76FFB2248C5F804A3BDE8F88F8E
:101A90004846A16904F0E0F8E36963620023E3616A
:101AA0001C4B9844D8E8EF3F43F40023C8E8E23FDA
:101AB000002AF7D1502303FB0B63586ADA68996850
:101AC000DB6C121A0144C5F83415C5F83825DA0460
:101AD000D9D501232B60D6E7502303FB0B6633696E
:101AE0008BB9F36CC5F834955B04C6E90497C5F867
:101AF0003875C8D5D5F8003243F02003C5F8003258
:101B0000C1E70548C0E70548BEE700BF58190020F7
:101B10000000AD0BA41900200A00AD0B0B00AD0BAB
:101B200050232DE9F0413C4D90F80480046803FBFC
:101B30000853DB6CD4F8000203F48223B3F5805F12
:101B400068D1D4F80463C4F8086309B9830656D48D
:101B5000D4F8003223F02003C4F800324FF4842379
:101B600008EB8801090101F14C072F44D7E8EF0F7A
:101B70001843C7E8EC0FBCF1000FF7D12AB9502386
:101B800003FB08535B68002B41D1244BC4F8083396
:101B900001236360D4F84431002BFBD00023C4F848
:101BA0004C31D4F84C21C4F81031D4F81021C4F8C9
:101BB0004431D4F84431502303FB0853DA6C12F457
:101BC00000421FD1DA61204600F053FB502303FB93
:101BD00008550023AB602B61D7E8EF3F23F47F0368
:101BE00023F47043C7E8E23F002AF5D126F420260B
:101BF00026F404760A48C4F80463BDE8F0814FF483
:101C00008033ADE72046294400F045FBDBE70123A4
:101C10006360EFE70348F0E75819002010020A005C
:101C20000000AD0B0500AD0B2DE9F8432F4A03680A
:101C30000679C3F8082343F30733002B04460DDB72
:101C400001215A0903F01F03994002F12003284A99
:101C500042F82310BFF34F8FBFF36F8F012220464E
:101C60001146FFF75DFF01212046FFF7BFFD502120
:101C70002279204D236801FB0252D46CD3F80C0565
:101C8000E201D3F81495D3F80875D3F8108509D577
:101C90004FF0FF32C3F80C25C3F81425C3F808250C
:101CA000C3F81025A30116D5411C01D0FFF762FC33
:101CB000B9F1FF3F02D04846FFF75CFC22010AD58C
:101CC000B8F1FF3F02D04046FFF754FC7B1C02D026
:101CD0003846FFF74FFC5023002203FB0653DA641B
:101CE00083F848205A60BDE8F88300BF10034A001B
:101CF00000E100E05819002010B5502402790B4B88
:101D000004FB02335B686BB90368D3F810211AB97E
:101D1000D3F80025082A07D011B1D3F83C350B6061
:101D2000034810BD0348FCE70348FAE758190020B0
:101D30000000AD0B0800AD0B0B00AD0BF7B5054671
:101D40001646FFF751FE164B0446984222D1032156
:101D500028462F79FFF7A6FD124B984201D0A042EA
:101D60001BD15022104B02FB07335B6893B90C4C1C
:101D7000284601A9FFF7C0FFA042F9D1019BB34259
:101D800007D301222846114603B0BDE8F040FFF713
:101D9000C7BE064C204603B0F0BD0446FAE700BFBC
:101DA0000000AD0B0B00AD0B581900200800AD0B67
:101DB00072B6024A1368013313607047A8190020F5
:101DC000034A1368013B136003B962B6704700BF52
:101DD000A81900200722024BC3F80423704700BF54
:101DE00000300050084BD3F80801D3F80021003828
:101DF00018BF012080000AB140F00100D3F804317F
:101E00000BB140F002007047003000500022074B39
:101E1000C3F80021D3F80011C3F80421D3F804114A
:101E2000C3F80821D3F80831704700BF00300050D4
:101E3000002317200C49012B03F1010201D813469E
:101E4000F9E703F5C073202A41F823001346F2D1C5
:101E500000231720044A03F5E0710133202B42F8D8
:101E60002100F8D1704700BF0030005010B59DF838
:101E70000840C00B43EA0423064CC90B43EA021393
:101E8000884200D910BDC2B202F5C07244F82230B7
:101E90000130F5E70030005010B59DF8084000F122
:101EA000604043EA042301F16041074C400B490BB9
:101EB00043EA0213884200D910BDC2B202F5E072B3
:101EC00044F822300130F5E700300050C0F30E0333
:101ED000C3F50043B3FA83F3C3F11B03064AC0F30F
:101EE000C730DBB240F4807043F48073C2F8000561
:101EF000C2F80435704700BF00300050430301486A
:101F000018447047FF1FF81F054BC0F30730090244
:101F100041F0300100F5007043F82010704700BF19
:101F200000300050044BC0F30730090200F5007088
:101F300043F82010704700BF00300050003A18BF2F
:101F40000122003918BF012103688900074841EACE
:101F50004201186359605A6842F001025A60BFF3A7
:101F60004F8FBFF36F8F0020704700BF04AAFF00A0
:101F700008B5FFF737FF044B162118600348BDE88A
:101F8000084000F008B900BFEC1F00202636010011
:101F90000C22014903F060BEEC1F002010B501F0D7
:101FA00052FA044690B901F0DDFE044680B90A4AAF
:101FB0002E21D368094823F008031B041B0C43F0AF
:101FC000BF6343F40033D36000F0E5F8204610BD52
:101FD00045F22354FAE700BF00ED00E03C36010073
:101FE000024B1860024B002019607047FC1F002054
:101FF000F81F00201FB5274C426923685A62826986
:102000009A62C269DA62026A1A63426A5A63826A2F
:102010009A63C26ADA63026B1A64426B5A60826B1B
:102020009A60C26BDA60026C1A61426C5A61826C0F
:102030009A61C26CDA61026D1A62826D5A65C26D74
:102040009A65026FDA65026E1A66826E5A66426F90
:102050009A66EFF388825A64EFF389829A64426841
:10206000DA64EFF394821A65026801A81A67FFF731
:102070008FFF2368019ADA6601221A70064B1C68EA
:1020800064086400204621462246234603F0BDFE34
:1020900004B010BDFC1F0020F81F002000B5A1B047
:1020A00001A8FEF7E3FD029B63B15B060AD4019B26
:1020B00023F00203052B05D1044B1B6813B101A8C3
:1020C000FFF798FF21B05DF804FB00BFF81F002068
:1020D000BFF34F8F0549064BCA6802F4E062134311
:1020E000CB60BFF34F8F00BFFDE700BF00ED00E006
:1020F0000400FA05F8B543680C2B26D14B68042B75
:1021000023D14FF0FF3304680E6821683360E1B1DA
:10211000A268D2B10623012001F0EDF8A8B96168E8
:102120000B4BD3E9005CA9420AD3A26865448F181F
:10213000AF4205D8206803F08FFD00203060F8BD65
:102140000130042803F10803EBD10220F7E700BFB8
:102150006C3601004FF47F03D3F83001D3F83431EB
:10216000BFF34F8FC0F30B00A0F109035842584151
:1021700070474FF47F02D2F83031D2F83401BFF308
:102180004F8FC3F30B03092B03D1431E5842584111
:10219000704700207047FEF7F9BD012070476FF0CF
:1021A00003007047002382B00193019802B070478A
:1021B0006FF003007047002382B00193019802B0D2
:1021C0007047022814BF6FF0030000207047FEF72D
:1021D00059BE30B501EB8202914200D130BD51F8B9
:1021E000044B04F07F037F2B4FEA144408BF4FF0E9
:1021F000FF33032CF0D8DFE804F002040608036084
:10220000EAE74360E8E78360E6E7C360E4E70346A4
:10221000D0F8580130B931B9D3F82001003818BFCF
:10222000012070470120704730B504460D4685B047
:1022300010220021684603F034FDD4E900136846FB
:102240008DF80050984705B030BD7FB504460E4666
:10225000154600211022684603F023FD012368463D
:102260008DF80030CDE90165D4E90013984704B03A
:1022700070BD10B50446FFF79BFDD4F8583133B15B
:10228000D4F8043313F4800308BFC4F80035BDE864
:102290001040FFF795BD70B50D4604460522AA21F2
:1022A000D0F83C65A86903F0FCFC0522AB69C4F8D2
:1022B0003435C4F838250022C4F81021D4F81011A0
:1022C0000121E162D4F810110029FBD0C4F84C219F
:1022D000D4F84C11C4F81021D4F81021D4F83C25BE
:1022E0009642EA6109D15A1E043312F8011FAA2945
:1022F00003D19A42F9D10023EB6170BDD0F8583177
:1023000033B1CB6CC3F30032DB0458BFC0F80025F7
:10231000704770B5CE6C0D4606F001010446FFF71C
:1023200076FF38B94FF4800346F00406EE64C4F833
:10233000043370BDD5E90A365AB1296CEA6B761AB6
:10234000964228BF164619443246A86B03F084FC17
:10235000AB6B4FF0FF326A641BB1C4F84435C4F86C
:1023600048650023C4F82031D4F82021C4F858313E
:10237000D4F85821C4F85031D4F850310823C4F8A7
:1023800000354FF48003C4F804330123A360D0E781
:10239000C0037047C00300F5FF407F307047002046
:1023A00070471F2070474FF40040704700F57F4092
:1023B000C03040037047402070475F2070474FF4A3
:1023C000005070474B6830B513F01F052DD10268DF
:1023D0000C681068C0F30720844226D2506855600C
:1023E00094600C7C23F01F0304F001041C438B7CDD
:1023F000DB0003F018031C434B7C5B0003F0060377
:102400002343D3608B68013B23F01F04CB685B0040
:1024100003F00E03234343F0010313615060BFF345
:102420004F8FBFF36F8F284630BD0120FCE7036854
:1024300000205A68C9B258609960D86018615A6023
:10244000704770B50546002403681E68C6F307266A
:10245000B44201D1002070BD21462846FFF7E7FFB6
:102460000134F5E70020704708B5FFF717FE72B694
:1024700020BFFDE7002070470020704770470B46E3
:1024800070B5114618B1032806D0032070BD184658
:10249000BDE87040FFF72EBE5A68082A01D002201E
:1024A000F4E74C68042CFAD11D684FF0FF330E6836
:1024B000296833600029F2D06B68002BEFD0262307
:1024C0007422012000F017FF0028E8D122462323C0
:1024D0000120696800F00FFF04460028DFD1D5E92C
:1024E0000001FFF77DFD30602046CFE730B50C4698
:1024F000154685B038B139B1FFF74DFE041E03DA39
:10250000204605B030BD044640F60D23ADF80E3030
:1025100009230B4901A805F00F028A5C2D091A5402
:10252000013B012BF7D147F630030C21ADF8043005
:10253000FFF731FE0028B4BF04462418E0E700BFCF
:102540008C36010008B5154B83F30A88144800F057
:1025500065FF00BBFFF722FDE8B9FFF783FFD0B9A5
:10256000FFF788FF98B9FFF789FF00F0C3FE352118
:102570000C48FFF710FE00F009FC26210A48FFF77F
:102580000AFE00F03BFA00F097FE002008BDFFF7BE
:1025900073FF0028E7D000F0EBFDEEE70004002019
:1025A000AC1900209C360100D13601002DE9F04F16
:1025B00093B00093574B8146D3F800B00BB2002B79
:1025C0000D461646C1F30268C1F3024A04DA6FF001
:1025D000800013B0BDE8F08F8B42C36001D10020B2
:1025E000F7E708EB0A03042BF1D8CC0F64014FEA9C
:1025F000C80731463A46DBF8080044F0020300F011
:102600007AFE01460028E2D1202202A803F049FB0D
:102610003A46314602A84FEACA0603F01DFB32468D
:102620000099DBF8080044F0060300F064FE07465A
:102630000028CCD1014620220AA803F032FB324602
:1026400000990AA802AE03F007FB33460137B845EC
:1026500014D91A46BC460DE0D2F808E0D1681868D3
:102660007144884203D2596808448645AFD30CF1BF
:10267000010C0832C445EFD10833E7E715F0006FCD
:1026800018BF202409F1180707EB880844F002035B
:10269000474513D1202C26D1002D02DBC5F3C045C0
:1026A0006C0109F128050AAE05EB8A0A44F006041C
:1026B00055451AD1009BC9F87C3090E77268DBF869
:1026C000080056F8081B019300F015FE00287FF45F
:1026D0007EAF56F8042C019B47F8042F56F8082CBF
:1026E00038633A62D4E70024DBE77268234656F881
:1026F000081BDBF8080000F0FEFD00287FF467AF40
:1027000056F8043C45F8043F56F8083C28642B630F
:10271000CEE700BFB01900202DE9F0411F461A4B4B
:102720000D461646D3F8008000F0D9FE044608B9DD
:1027300000F01EFDE368002B01DA00F019FD032D07
:1027400001D900F015FD04EB8504E569E36CED1A91
:1027500016D006233A463146D8F8080000F0CBFDE3
:1027600008B100F005FDBD4228BF3D46E36CE16BBA
:102770002A461944304603F06FFAE36C2B44E364B5
:102780002846BDE8F08100BFB01900202DE9F041D6
:102790001D461A4B0F461646D3F8008000F09FFEE8
:1027A000044608B900F0E4FCE368002B01DA00F00D
:1027B000DFFC032F01D900F0DBFC04EB8704E36AA4
:1027C000E26E9B1AAB4201D200F0D2FC02232A46F1
:1027D0003146D8F8080000F08EFD08B100F0C8FCC2
:1027E000E36EE06D2A463146184403F035FAE36E95
:1027F00000202B44E366BDE8F08100BFB019002043
:102800002DE9F04105464FF001080E4E0E4B37689A
:102810005C681CB928463760BDE8F081226893687F
:1028200013F400700CD1A369012B09D0D368346074
:1028300023B19847002801DA00F09AFCC4F8188008
:10284000246AE6E7B0190020B419002038B5044620
:1028500010B96FF0800038BD8368002BF9D01A687A
:10286000002AF6D05D68002DF3D00B4BE861A86913
:102870001D6020B92B68DB6853B90123AB61A368E5
:1028800004F10C001B681B69984701232360E2E7F1
:1028900098470028F1DADCE7B01900204268024BC3
:1028A00008461A60704700BFB0190020002330B5F9
:1028B00005680446AA68C0E9063312F4406F85B083
:1028C0001CD012F4006202D000F084F90246A96A1A
:1028D0002B6968460B44073123F0070321F00701F9
:1028E000CDE902130093002305490193EB6800F042
:1028F0006DFA684600F0D6FD024B1C6005B030BD95
:1029000001280100B019002001F00C0370B50C2B58
:102910000CBF154605464A060C461ED58B0658BF09
:102920002835AB6913F8026C84F00803C3F3C003C5
:10293000C6F38012934201D000F01AFC16F0A00FEB
:102940001ED176B1032E17D032461C210E48FFF758
:10295000CDFD6FF083032B600CE000F009FC202616
:10296000E2E700F009FB0446FEF746FA2146074875
:1029700000F094FD204670BD284600F00DFAF9E7FE
:1029800032461F210248E2E7F7360100F80B00202B
:1029900013370100EFF308807146EFF30982EFF37C
:1029A0000B830CB406B4FFF7AFFF8646009900F026
:1029B000080001F00801401A02DC12DB04B0704785
:1029C0001EF020031CBF2DE9F00FBDF1080D0A4CCD
:1029D000254626462746A046A146A246A34630B431
:1029E000704704B030BC1EF020031CBF1DF1080D61
:1029F000BDE8F00F04B07047A5EDF5FE084BDA68AE
:102A000082F07F4282F47F0242F48042DA60002248
:102A10001A765A76DA76DA77602283F822207047BF
:102A200000ED00E0009A0A4B9A420FD10122904338
:102A300001460246034604460546064607468046CA
:102A4000814682468346844686460447FEE7000068
:102A5000A5EDF5FE2DE9F041044618B943F6DA304C
:102A6000BDE8F0810029F9D08368002513F4406F98
:102A700014BF01230023134F43F00203DFF8488003
:102A80000B6000F13006236AAB4201D80020E7E773
:102A90001421A369E26906EB830301FB02330C22D4
:102AA0006A4399188968090709D59B58BB4201D028
:102AB0004345D3D1186810B10121FFF725FA01353C
:102AC000E1E700BFB4100020AC10002070B5324C1C
:102AD00086B03248FFF7B5FC236801255A1C0193E4
:102AE0002F4B2260DA681B694FF440760393002372
:102AF0002A4801A902920495ADF814608DF81630A9
:102B0000FFF760FC18B143F6DA3006B070BD2368F9
:102B10008DF816005A1C0193224B20480293224B39
:102B200001A9CDE903352260ADF81460FFF74AFC36
:102B30000028E8D123688DF816005A1C01931B4B1E
:102B4000164802931A4B01A9CDE903352260ADF86E
:102B50001460FFF737FC0028D5D123688DF81600E4
:102B60005A1C0193134B0D480293134B01A9039375
:102B70000223049340F201132260ADF81430FFF7F2
:102B800021FC04460028BED12A4629460348FFF707
:102B9000D5F92046B9E700BFBC190020A8100020D5
:102BA000A4370100E03701000060010020080100A7
:102BB00020080100000C0020200C0020014B1868A8
:102BC000704700BFA4370100014B1B6818687047AD
:102BD000A4370100014B1B6858687047A4370100F7
:102BE00008B5FFF7C5F9FFF711F90A4B5A68103A13
:102BF000D3B2120609D401215A0903F01F039940E8
:102C000002F16003044A42F82310BDE8084000F0D6
:102C1000AFBA00BF00ED00E000E100E00020034B90
:102C2000D8765A6A42F470225A62704700ED00E08A
:102C30000349044BCA68002092B21343CB6070472B
:102C400000ED00E00800FA0500224FF0FF300D4BC8
:102C500002F1A0010132102A43F82100F8D1D3F883
:102C60008022002022F00802C3F88022D3F88022BC
:102C7000D3F8802222F48072C3F88022D3F8803205
:102C8000704700BF00E100E008B5FFF7A3F8082295
:102C9000024BC3F880211A60002008BD00E100E06B
:102CA000064BD3F8D02022F00102C3F8D020D3F88D
:102CB000D02042F00202C3F8D020704700ED00E0BF
:102CC00037B50124FFF7B4F8174D224605234FF41A
:102CD000813016490094FFF7C9F8224607234FF0C8
:102CE000005013490094FFF7D7F8D5E901010723F5
:102CF00000220094FFF7BAF8072300220D490E487E
:102D00000094FFF7C9F82969E8680139FFF7DEF890
:102D1000062300224FF4082008490094FFF7A6F884
:102D2000002003B030BD00BFA4370100FF7F0100C9
:102D3000FF7F0020FFFF032000800020FFFF0F0027
:102D400038B500240E4D002155F8040B0134FFF76F
:102D5000E9F81C2CF7D10020012240F20111094BA7
:102D6000C3F88004C3F88424C3F8C004C3F8C4249F
:102D7000054AC2F840154FF48072C3F8402438BDAC
:102D80003437010000300050009003500122014B05
:102D90001A607047C019002010B50446094B2289FB
:102DA000186861680623806800F0A5FA28B9064B08
:102DB0001B68012B01D100F087F86FF086032360B8
:102DC00010BD00BFB0190020C01900202DE9F84344
:102DD00005461E460068134B9046AA68A0F10804F9
:102DE00040E90233503890420F4601D200F0C0F95A
:102DF000A4F1480948220021484602F052FF00236E
:102E000044E9073344F8143C4FF0807344F8043C21
:102E10006FF0020344E9036744F8208CC5E900938E
:102E2000BDE8F883A5EDF5FE30B5094C02466168B2
:102E30000023084640B105686D68954205D11BB175
:102E4000826860609A60816030BD03468068F1E707
:102E5000441A002038B504462AB10B689B68DB058C
:102E600012D5002038BD0B4B1D680DB900F080F95C
:102E700000222B6899692C338A4203D053F8040F3F
:102E8000A04204D19142ECD16FF0FC00EAE701329C
:102E9000F2E700BFB019002070B504460E46154693
:102EA000002130220C3002F0FCFE064B20461B684D
:102EB000A6606360656100F001FA00232061236071
:102EC00070BD00BFB0190020044B1B681BB11B680C
:102ED0000BB1586870474FF0FF307047B0190020B1
:102EE000064B10B51C680CB900F042F923689B68CA
:102EF00013F4406F14BF0120002010BDB019002052
:102F00002DE9F843904607460C46FFF7E9FF0246D5
:102F100024B96FF080042046BDE8F8836300F8D53B
:102F2000144B04F01F0153F82150002DF1D02B68F1
:102F300029465868FFF78EFFB0B9C4F30721284629
:102F400000F0BBFA04460028E3D1EFF3108972B613
:102F500000F0C1F9064689F3108840B1424629467F
:102F6000FFF79AFF3E60D6E76FF08104D3E76FF07A
:102F70008204D0E7C41900202DE9F04100F0AAF93D
:102F80000023134E134F73607B6000F0E5F8DFF809
:102F90004880304600F022F80446A8B13946802324
:102FA000424600F07FF80546204600F0CBFA206844
:102FB00004F10801FFF74EFD08B100F0D9F82946E9
:102FC0002046FFF773FCE4E7BDE8F04100F071B97B
:102FD000B4190020441A0020C4190020F8B5054691
:102FE00008B900F0C5F82A4E346814F1290F4CD8FE
:102FF000284B196804F128038B4246D2236AA26940
:1030000003EB43030C321344606AE269024402EBAF
:10301000820213449B00E31801D2994201D200F0CE
:10302000A7F823681C4A1B0C1B04934201D000F034
:103030009FF82388B3F5817F01D300F099F8636886
:10304000002B01DA00F094F8144A176807F1240302
:103050001360134A1268934201D900F089F8236A79
:10306000A26903EB43030C32616A1344E2693C60DA
:103070000A4402EB82021344326802EB83026B685B
:1030800032603B626F603846F8BD0027FBE700BF47
:10309000C4100020C837010000005F5FC01000208E
:1030A000C43701002DE9F74F0F46904606460093BE
:1030B00000B109B900F05CF8D6F800A0DAF81820E1
:1030C0000AF1300303EB820BDAF81C40204B1D6839
:1030D00054B10C2202FB04541C601E4B1B689C4222
:1030E00001D900F045F82C4625464FF00009DAF8E2
:1030F0001C204A4500D91CB9002003B0BDE8F08F60
:10310000142303FB09B20023C5E900269268AB60D3
:10311000930516D5B8F1000F02D0009B802B03D089
:10312000019200F025F8019A12F0E00FD0B202D11E
:1031300058F820201AB1019000F01AF8019848F8C8
:1031400020507A6809F10109AA607D600C35CEE74C
:10315000BC100020C037010008B5FFF72FFD034B5E
:103160009860FFF731FD80F3888808BD00ED02E02C
:10317000FFF77AB98230012808B506D8FFF7B0FE0C
:1031800018B9BDE80840FFF7F3BF08BDF8B506461B
:103190000D4600F0A4F9044608B9FFF7E9FFA76857
:1031A0000FB9FFF7E5FFE368991C20D05A1C21D125
:1031B000A5B315F1820F13D102232360EFF310861C
:1031C00072B629462046FFF769FB054686F310884C
:1031D0002368022B24D1204600F086F82846F8BD4B
:1031E00015F1830FEAD0FFF7C3FF0025E6E70223BE
:1031F0002360FAE7002BF6DB204600F094F93B68E9
:103200009B689B0501D50223236015F1810FD5D161
:103210006369002BD2DBFFF7ABFFCFE73546F4E75E
:1032200000232360DAE708B5FFF71EF96FF083008B
:1032300008BD2DE9F3410E46174698460546FFF7AF
:103240004FFE00F060F92946024601A8FFF758FE3C
:10325000044660B943463A4631460198FFF7A6F95D
:10326000044640B16B0002D5019800F03DF82046BD
:1032700002B0BDE8F0810198FFF7E8FA0446F6E7EE
:1032800040F20110704770B50546FFF729FE06466B
:103290002846FFF7C9FD044608B9002070BD014665
:1032A00032462846FFF7D6FD0028F6D12368D868B5
:1032B000F4E76FF00200704700DF70474FF4805072
:1032C0007047B0F5805F03D1EFF30B808038704713
:1032D000002070477047EFF30B8000F1800383F309
:1032E0000B88704700207047EFF30B83803B83F31C
:1032F0000B88704770472DE9F0410E461546002AAD
:103300004AD0C4074BD480F00204C4F34004A400A4
:1033100003F00602062A4AD144F001042246294657
:10332000304602F0A9FBB8BB46E800F205EB060800
:10333000100E120208F1FF3747E800F34FEA13615D
:1033400066D51B0264D5884262D046E800F547E89E
:1033500000F7FFF724F82D0E85424FEA176734D3A4
:10336000FFF71FF8874230D82846FFF713F82246A8
:10337000C6F101010144304602F07EFB002847D02F
:103380000135AF4218D83846FFF702F82246A8EBBD
:10339000000102F071FBD8B30020BDE8F081EFF32B
:1033A0009484A40004F0040444F01204B0E79907E4
:1033B00031D544F00804B1E72846FEF7E9FF064698
:1033C000FEF7F1FF22460146D5E7FEF7F4FF8542FE
:1033D0001ED3FEF7F2FF87421AD82846FEF78EFD6D
:1033E0002246C6F101010144304602F045FB78B1A6
:1033F0000135AF4203D83846FEF7D8FFC6E7284666
:10340000FEF7D4FF0646FEF7DAFF22460146EBE759
:103410006FF07F00C1E74CF2DA20BEE710B504463A
:10342000FFF73EFCFFF74CFC10B143F6DA3010BD5D
:10343000FFF786FC0028F8D1FFF748FB0028F4D1FD
:1034400002232360F3E708B5FFF7E8FB10B143F66A
:10345000DA3008BDFFF7ECFB0028F8D100F01CF8CB
:103460000028F4D162B6FDF7B1FCFFF7EDFB0028B0
:10347000EDD1FFF709FC0028EBD0E8E7EFF3088077
:10348000EFF309812DE9F00F6B467246FDF7F4FB6F
:1034900008B0FFF7A5FBFEE70020704704460D4685
:1034A000A54628470368283383F30988836883F394
:1034B0000B88BFF36F8F4068704703689A68DB68BA
:1034C00012F4806F05D18B422CBF00206FF0FA0000
:1034D00070478B420CBF00206FF0FA00704710B5A8
:1034E000FFF7EFFE0446FFF7FDFE50B9FFF7ECFCD7
:1034F000A3685B681B685B68834218BF0024204692
:1035000010BD0024FBE738B5054648B100F01BF8B4
:10351000B5EBD07F044601D0FFF72AFE204638BD28
:10352000FFF7D2FCF4E7002310B500F1280252F8AF
:10353000041F19B1C16F146C19444C600833202B5F
:10354000F5D110BD70474FF0FF30704700000146C5
:103550004154414C204552524F523A20004861722A
:10356000644661756C740D0A004D656D4D616E6148
:103570006765206661756C740D0A0042757346615B
:10358000756C740D0A0055736167654661756C74DE
:103590000D0A005365637572654661756C740D0A9A
:1035A0000052657365727665642045786365707452
:1035B000696F6E2000506C6174666F726D20657863
:1035C0007465726E616C20696E7465727275707468
:1035D00020284952516E293A20000000110E0100A6
:1035E0009B210100C110010075100100C3210100E1
:1035F000CF210100490E01009F210100310E010081
:103600003D0E0100FD0E0100A5210100B1210100C8
:10361000B72101001C0000001B000200030202028F
:103620000338FDD87047506C6174666F726D204529
:103630007863657074696F6E3A0D0A00416C6C2096
:1036400070696E732068617665206265656E2063BF
:103650006F6E66696775726564206173206E6F6E48
:103660002D7365637572650D0A000000000001008E
:10367000000200000002FF002C0000003001FF00EB
:10368000080000004001FF000C0000003031323320
:103690003435363738394142434445461B5B313B6C
:1036A00033346D5B536563205468726561645D20DB
:1036B00053656375726520696D61676520696E6920
:1036C0007469616C697A696E67211B5B306D0D0AE4
:1036D000001B5B313B33346D426F6F74696E672042
:1036E00054462D4D2076322E302E302D6E6373329F
:1036F0001B5B306D0D0A00556E6B6E6F776E20533D
:10370000504D20535643207265717565737465641E
:103710003A2000556E6B6E6F776E20535643206EC5
:10372000756D626572207265717565737465643A52
:103730002000000000400050005000500090005059
:1037400000A0005000B0005000E0005000F0005019
:103750000000015000100150004001500050015085
:10376000007001500080015000B0015000C00150B5
:1037700000D0015000E0015000F001500000025064
:103780000010025000200250003002500040025051
:10379000006002500080025000A0025000900350D0
:1037A000002584500080010000800100FF7F080098
:1037B000007C01000080010000800800FFFF0F0076
:0C37C0002C120020141200200004010054
:1037E000009A204B9A4208D110B502F07DFA02F0FF
:1037F000A9F906BC96460C46744702F0B9FA009A3D
:10380000184B9A4208D110B502F07AFA02F09AF9F0
:1038100006BC96460C46744702F0AAFA0CB4029A0B
:10382000104B9A420CD14FF0004319430CBC10B519
:1038300000F09EF802F086F906BC96460C467447E6
:1038400002F096FA009A074B9A4202D1064908689C
:10385000744702F08DFA009A024B9A4200D17447E5
:1038600002F086FAA5EDF5FE801000200348044B17
:10387000834202D0034B03B118477047A8110020C0
:10388000A8110020000000000548064B1B1AD90FA4
:1038900001EBA301491002D0034B03B11847704755
:1038A000A8110020A81100200000000010B5064C4F
:1038B000237843B9FFF7DAFF044B13B10448AFF3A1
:1038C00000800123237010BDC018002000000000FC
:1038D000F45F010008B5044B1BB104490448AFF381
:1038E0000080BDE80840CFE700000000C4180020B9
:1038F000F45F0100A3F5803A704700BF174B002B1F
:1039000008BF134B9D46FFF7F5FF00218B460F467E
:103910001348144A121A02F0C4F90E4B002B00D0BF
:1039200098470D4B002B00D0984700200021040041
:103930000D000D48002802D00C48AFF3008002F0C3
:1039400077F820002900FEF7FDFD02F05DF800BFCA
:10395000000008000000000000000000F80B00203C
:10396000A8110020B828002000000000000000007E
:103970002DE9F84304460D4616461F46EFF305832E
:10398000C3F308030BB1FFF7F3FBDFF834903B46BA
:10399000204632462946D9F80080FFF74AFCD9F87C
:1039A00000300446984506D0DB6901461869BDE839
:1039B000F843FFF7EBBBFFF7DDFB2046BDE8F883DC
:1039C000B019002001680E4A0346914215D1C16921
:1039D000A2F11022A2F1EF1291420ED18268012AC7
:1039E0000BD8C26812B101698A4206D0586928B161
:1039F0009B691B1A5842584170470120704700BF0D
:103A000055AA00FF0D4B70B59E68A6B13046FFF772
:103A1000D9FF044678B9F3686BB935690DB920460A
:103A200070BD2846FFF7CEFF28B9EB68B34202D13C
:103A30002E462D69F2E70124F1E700BF4C1A002061
:103A40002DE9F041394E3468F368D4B1B468C4B19B
:103A5000002861D000295FD001FB00F5B5FBF0F034
:103A6000884259D1291D57D8AA070DD025F0030245
:103A700004321C4603E0616891424FD2A469002CD5
:103A8000F9D12046BDE8F0812A46F2E7891A2329B8
:103A900004F12007D4E9050C1AD80123A360A0B1D2
:103AA000C0F818C0A36903B158610023C4E9053305
:103AB0003369DB0702D5FFF7A5FFA0BB2A4600212B
:103AC00038463C4602F0EDF8DBE7C6F80CC0E9E703
:103AD00002F1200804EB08032039C3E9011E216923
:103AE000DFF84CE0DC60196144F808E0AEF1102E1C
:103AF000AEF1EF1EC3F81CE001B1CB60C3E9050CC9
:103B000040B18361996901B14B6101212361C4E92D
:103B10000121CAE7F360F5E70024B2E7D4F808E032
:103B2000BEF1000FB2D0012001F06EFF4C1A002050
:103B300055AA00FFF8B5054600283AD0364E33683E
:103B4000002B36D0B268002A33D0834203D8726883
:103B50001344984202D3012001F056FFA0F1200443
:103B60002046FFF72FFF0028F5D155F8183C012B10
:103B7000F1D145F8180C55E90570DFB1BB68CBB938
:103B800055F81C2C7B68203213447B60386100B1EF
:103B9000C76020220021204602F083F8386908B16E
:103BA00083682BB333699B0703D5FFF72BFF0028EE
:103BB000D1D1F8BD40B3836833BB42686368134416
:103BC000203363600369D4E90521236192B9B9B94F
:103BD000426981696261A161A2B19461A26902B185
:103BE000546103B1DC602022002102F05AF8D9E7C9
:103BF0003C46E2E79161A1690029E9D04A61E7E723
:103C0000F160F8E7F460E9E7F36845F8083C03B1D0
:103C10005C61F460C6E700BF4C1A002038B50D4661
:103C2000142200210446124802F03BF811491248C0
:103C300000F02CF8232D1AD914F003031FBF043D04
:103C4000ED18C3F10403E4182A460021204602F0CF
:103C500028F8074B094AC3E900459C602260A2F19D
:103C60001022203DA2F1EF126560E261DC6038BDF8
:103C70004C1A0020353B0100413A010055AA00FFD3
:103C8000014B1B68184700BFC8100020024B18608A
:103C9000024B002019607047CC100020C810002093
:103CA00010B50A46044619B1024B00211B6898471B
:103CB00010BD00BFD0100020054B0A46197819B17D
:103CC0000146181D02F08EB86FF08800704700BFE3
:103CD000601A002010B5074C00F032F8204602F0C0
:103CE00092F8201F0821FFF7DBFFBDE8104002F02B
:103CF00076B800BF641A002070B50C4D2B787BB9E4
:103D000002F06BF8044670B90126281D6E7002F0AF
:103D100067F8044638B900F00BF8044618B92E705D
:103D20000024204670BDFFF7D5FFFAE7601A002097
:103D30000122024B002083F880257047681A00207A
:103D4000F8B5074C2025264601272046276202F0B9
:103D500033F8013D04F12C04F7D186F88055F8BD05
:103D6000681A002010B50C4C236813B10B4B1B686C
:103D70002BB900F089FC30B90122084B1A600123ED
:103D80002360002010BD0138062801D9044810BD69
:103D9000044B53F8200010BD042000200020002018
:103DA000FE8FFFFF5C5E0100144B2DE9F0430028FD
:103DB00014BF04461C46124F236883B0BB4219D07F
:103DC00016460D4620464FF4147104F1040900F024
:103DD00047F804F58E78484600F0CEF8404600F0EB
:103DE00019FA2B464A4640460649009600F034FB35
:103DF00008B92760002003B0BDE8F0830820002048
:103E0000A5BCC95AFD3F010070B50D4C1D460028E8
:103E100014BF064626460B4B306882B098420DD13F
:103E200006F58E70002633460096144600F03EFBE1
:103E3000002818BF34462C6002B070BD0248FBE772
:103E400008200020A5BCC95AE88FFFFF38B131B166
:103E5000002201440346013081421A70FAD17047B2
:103E600038B131B1002201440346013088421A7052
:103E7000FAD170472DE9F043202B1D4606468846AF
:103E800091468BB026D8DBB202AF8DF80480B046E5
:103E900058F8041B8DF8053021B9404601F038F977
:103EA000044640B9012302224046336001A901F0D3
:103EB00043F9044638B138462021FFF7D1FF2046A8
:103EC0000BB0BDE8F0832A464946404601F034F97C
:103ED0000446F0E702AF1946104600233A4601F0C7
:103EE000B1FA04460028E6D12023B9461D46CCE7A6
:103EF0002DE9F041D0F8F830A6B0002BD8BF02AEC3
:103F000031DD05460027D0F80C4102AEA4F10108CE
:103F10009022D5F8FC403146D0F8000101AB019762
:103F2000B8FA88F8A0474FEA5818044620B9019B10
:103F300053B9B8F1000F16D030469021FFF790FF2B
:103F4000204626B0BDE8F081014632462846FFF7FC
:103F500091FF58B9D5F80431019A1344C5F80431DA
:103F6000B8F1000FE8D16FF03C04E5E704462046C5
:103F700026B0BDE8F08100BF70B5002504461422CC
:103F800004F588762946C0F8F850FC3001F089FE27
:103F900008222946304601F084FE144B30461B6847
:103FA0009847204640F8045B01F098F8104B3046E3
:103FB0001B689847C8B9D4F8F830AB420FDC03EB64
:103FC000830204EB82022021C2F800010120C2E931
:103FD000421008490133C2F8FC10C4F8F830064B0F
:103FE0003046BDE870401B68184770BDF0100020D7
:103FF000EC100020E14F0100E81000202DE9F0470F
:10400000202A88B07AD83F4B00F5887904461B688F
:1040100048461746884698470546F8B940F20116C3
:10402000D4F8F830002B65D02046FFF761FF054635
:1040300038B9D4F8F830002B14DC013EF2D16FF01F
:104040003B056E4620213046FFF70AFF2E4B4846BF
:104050001B689847002818BF6FF01D05284608B058
:10406000BDE8F087D4E94132934203D3D4F80C2160
:10407000012A02D0013ED7D1E1E71F2BFAD96E46C3
:1040800001462022304604F1040A01F00AFE3146BE
:10409000504601F07BF805460028D3D1504601F088
:1040A00031F8504601F01AF82946504601F030F830
:1040B00005460028C6D150462022314601F03CF882
:1040C00005460028BED1034632462021304601F085
:1040D000B9F905460028B5D1D4F8F8303A46002B96
:1040E000C8BF002340463146C8BFC4F8043101F0C0
:1040F000B3FDA7E76FF03F056E46A3E76FF03B0502
:10410000ACE700BFEC100020E810002070B590B0C4
:1041100000287AD03E4C0D464022362106462046E5
:1041200001F0BFFD40225C21A01801F0BAFD2B1D5B
:10413000A34203D904F144039D4252D32B68226861
:10414000534023602B68226C534023646B68626881
:10415000534063606B68626C53406364AB68A268F1
:104160005340A360AB68A26C5340A364EB68E26861
:104170005340E360EB68E26C5340E3642B692269CF
:1041800053402361226D2B695340236562696B693B
:10419000534063616B69626D53406365AB69A269AB
:1041A0005340A361AB69A26D5340A365EB69E2691B
:1041B0005340E361EB69E26D5340E3650021304613
:1041C00000F0A6FF044628B940223046104900F00E
:1041D000B3FF044640216846FFF742FE204610B078
:1041E00070BD631E04F13F01013D1F3415F8010F3E
:1041F00013F8012F42401A7011F8012F2878A342BA
:1042000082EA00020A70F1D1D8E76FF07304E5E7A3
:104210005822002010B54FF49A720021044601F094
:1042200040FD42F21072044BC4F8202104F5967050
:104230001B68BDE810401847F01000202DE9F04F32
:1042400004468846914695B0002900F0A780002AD0
:104250000CBF0126022600238DF80C30002C00F044
:104260009F80DFF844A104AF0AF1400B00212046F3
:1042700000F04EFF034648B1384620210193FFF776
:10428000EFFD019B184615B0BDE8F08F4022514666
:10429000204600F051FF03460028EDD104F1F4055B
:1042A00020222946204600F047FF03460028E3D19C
:1042B0000122204603A900F03FFF03460028DBD17E
:1042C000022E62D020460CA900F060FF03460028B1
:1042D000D2D10146204600F01BFF03460028CBD177
:1042E00040225946204600F027FF03460028C3D14C
:1042F000202220460CA900F01FFF03460028BBD156
:104300003946204600F042FF03460028B4D1394622
:104310002046FFF7FBFE03460028ADD120222946A8
:10432000204600F009FF03460028A5D120460CA92D
:1043300000F02CFF034600289ED10146204600F0E5
:10434000E7FE0346002897D140225946204600F058
:10435000F3FE034600288FD1202220460CA900F04E
:10436000EBFE0346002887D12946204600F00EFFC9
:104370000346002880D19DF80C200132D2B2B2420F
:104380008DF80C20FFF472AF76E74A46414620468E
:1043900000F0D2FE0346002894D06DE701265AE7CC
:1043A0006FF0730304AF67E7582200202DE9F04156
:1043B0000446884615461F46D0F81801E0B013B1F0
:1043C00000EB40004008B5F5807F3ED82844B0F5AA
:1043D000C07F3AD84FF4C0720021684601F061FCFA
:1043E0006946D4F82431D4F81821D4F82801984724
:1043F00070BBD4F8186157B1D4E9493072080DEB9D
:104400000601984720BBD4F8183106EB5306B8F1E3
:10441000000F00D08DB9324669462046FFF70EFFE7
:10442000054610B90123C4F8143131466846FFF738
:1044300017FD284660B0BDE8F0810DEB060041464F
:104440002A462E4401F008FCE5E76FF00405F0E78A
:104450006FF00805EDE700BF2DE9F047044604F1D1
:10446000F4050F4691461E46DDF8208000F036FE2A
:1044700029462046FFF74AFE08B1BDE8F0872846E6
:104480002022012101F00DFCD4F81831C4F8247168
:10449000C4F8289113B92023C4F818314246314694
:1044A0002046BDE8F0470123FFF780BFB2F5806FDB
:1044B00000F295802DE9F04F89B09A46129BB3F532
:1044C000807F00F29080D0F82431164604460F46D3
:1044D0004BB3D0F81C31012B05D0D0F81421D0F803
:1044E00020319A421FDD514600232046129AFFF7E1
:1044F0005DFF014698B900231293002E5ED0DFF8CD
:10450000EC9009F1400B0021204600F001FE202E26
:104510003546014628BF202504F1F40890B108462D
:1045200009B0BDE8F08FBAF1000FE6D0129B002B66
:10453000E1D051461A462046FFF780FE014600288A
:10454000DBD0ECE749464022204600F0F5FD01466D
:104550000028E4D141462022204600F0EDFD01462E
:104560000028DCD16946204600F010FE01460028F4
:10457000D5D1204600F0CCFD01460028CFD15946C8
:104580004022204600F0D8FD01460028C7D16946E8
:104590002022204600F0D0FD01460028BFD1414630
:1045A000204600F0F3FD01460028B8D138462A46DF
:1045B000414601F051FB761B2F44A4D151462046C1
:1045C000129AFFF73BFE01460028A8D10846D4F80E
:1045D00014310133C4F8143109B0BDE8F08F6FF025
:1045E0000201084670476FF0040198E75822002046
:1045F000002130B58DB0282202A8019101F051FBB5
:1046000002A800F047FF044610B120460DB030BDAF
:10461000174D4FF0FF31286800F042F9044620B1F1
:10462000144800F0D3F9012C18D0002000F068F9EC
:10463000D0B9114A02A901A800F0C4FC0446012027
:1046400000F05EF960B9286800F032F90028DCD08B
:104650000A4800F0BBF920460DB030BD0524F2E752
:10466000074800F0B3F9EEE7064800F0AFF9E0E7DD
:10467000D4100020785E0100D8220020D05E010016
:10468000B05E0100905E010030B583B000F05CF8D0
:1046900028B100F0ABF80324204603B030BD00F091
:1046A00077F8D8B900F02CF9E0B9224CD4F82839C1
:1046B0001B0EF02B0AD1D4F8242A1F4B9A4231D07A
:1046C00000F044F8072400F091F8E5E7062400F034
:1046D0003DF800F08BF8204603B030BD042420469E
:1046E00003B030BD00F032F800F080F8FFF780FF33
:1046F000044698B9114D2B68002BCDD102460146D6
:10470000FFF752FB50B968220D4901ABFFF77CFB64
:1047100020B920460B4B2B6003B030BD052420464A
:1047200003B030BD012000F0EBF80028DAD1C4F866
:104730000C0ADBE7001084500000E020F824002081
:10474000FC2400205AEA5A5A002070470020704783
:10475000430504D54FF0FF32034BC3F80821024B49
:10476000C3F8080A704700BF00108450014BC3F81B
:10477000040A70470010845008B100F06BB84FF481
:104780007500704708B100F04FB84FF475007047DE
:1047900010B5114800F070F800B110BD0F4800F0DE
:1047A0006BF80028F9D10E4C204600F065F800287F
:1047B000F3D10C4B0C481C6000F05EF80146002859
:1047C000EBD100F02DF8044608B1204610BD00F0F2
:1047D00079F82046FAE700BFE4100020E01000203E
:1047E000DC100020D4100020D810002008B50848A4
:1047F00000F04CF8074800F049F8074800F046F888
:10480000064800F043F8BDE8084000F00BB800BFD0
:10481000E4100020E0100020DC100020D810002060
:1048200000207047704700BF024610B4084CD4F80F
:10483000003A1342FBD021B1D4F804310B60C4F824
:104840000831034B0020C3F8082A10BC704700BF92
:1048500000108450044AD2F8003A1842FBD0C2F843
:10486000080A0020704700BF0010845001F0BEB954
:104870000A46002101F015BA08B5034B02681B680F
:1048800010689847002008BD1011002008B5034BA0
:1048900002685B6810689847002008BD101100206E
:1048A000024B02689B681068184700BF1011002077
:1048B00008B5034B0268DB6810689847002008BD04
:1048C0001011002070B5094C094D2069AB6898475C
:1048D00018B1084B08485B6898470021074AEB6805
:1048E00011602069BDE87040184700BFFC1000202F
:1048F00010110020F4100020E85E01006425002063
:10490000F8B51A4D1A4E0446B26828699047E8B9BE
:10491000184F3B684CB1A3B1012B19D0013B3B6050
:104920002869F36898470020F8BD43B90121124A6D
:10493000C2F800151149D1F81029002AFBD1013322
:104940003B60F368286998470020F8BD0C48F8BD23
:104950000A4AD2F81039002BFBD1074A6FF07E408B
:10496000C2F80035FFF702FF3B68D7E7FC100020D4
:104970001011002064250020000084500010845095
:10498000E98FFFFF014B1B68184700BF1011002083
:10499000014B9B68184700BF10110020014BDB68DA
:1049A000184700BF10110020BFF34F8F0549064B79
:1049B000CA6802F4E0621343CB60BFF34F8F00BFBD
:1049C000FDE700BF00ED00E00400FA0530B44FF051
:1049D000FE320025074B084C08494968C3F80024FB
:1049E000C3F80424C3F80824C3F80C24C4F8005501
:1049F00030BC08470010845000008450F4100020A0
:104A000010B5044650B1636813F0685F05D0064ADC
:104A1000934202D000236260236010BD034B044820
:104A20005B689847EFE700BF2C5F5CA9F41000209B
:104A3000085F0100C8B143680D4A934213D013F0D8
:104A4000685F0ED0012350E8002F194640E8001C93
:104A50009CF0000FF7D1012AF5D0BFF35F8F002043
:104A6000704704487047044870476FF4E04070474F
:104A70002C5F5CA9E98FFFFFEA8FFFFF034680B13F
:104A8000426809498A420AD012F0685F05D0BFF334
:104A90005F8F002210461A60704704487047044830
:104AA00070476FF4E04070472C5F5CA9E98FFFFF0F
:104AB000EA8FFFFF10B5044620B10023034A2360AC
:104AC000626010BD0248FFF781FFF6E73A00003A46
:104AD000305F01002DE9F047002878D00C4600290E
:104AE00075D01D46002B72D007461AB10122002353
:104AF0002A6003602B68002B64D02946204600F012
:104B0000B7FD804600285FD12146286800F096FD59
:104B10008046002858D12B68082B6CD0042B6DD010
:104B2000A3F10209B9FA89F94FEA59190121354E61
:104B3000C6F8C411C6F84011C6F8C411636AC6F8B5
:104B40003031D6F830219342F6D14FF0000A4FF0C1
:104B5000FF30C6F82CA1FFF7FBFD6FF01B0350469A
:104B6000C6F80031FFF702FEC6F80C91D6F8040A29
:104B700040F48060FFF7FAFD0A23C6F83831089B3D
:104B8000012B29D02369204AA2FB03231B09626A57
:104B9000404602FB03F303EB43031A4ADB039B0982
:104BA000C2F8D8310123C2F82C313B682A6823F0BF
:104BB0007F4343EA02633B602A6843EA02233B6087
:104BC000BDE8F087DFF844804046BDE8F087DFF8B5
:104BD00040804046BDE8F0874FF47F03D3F80C2CAB
:104BE000013206D0D3F80C3C074AA2FB03231B0971
:104BF000CDE71623CBE74FF0030997E74FF0020903
:104C000094E700BF00108450ABAAAAAA310CF100AF
:104C1000350CF10058B34B1EB3F5047F27D230B5E5
:104C20004FF0000ECD00744671464B0901F01F0C89
:104C300050F82330BCF11F0F23FA0CF306D003F019
:104C4000010319B901211C468E46EEE79C4201F191
:104C5000010106D01C464FF0010EA942E5D100200B
:104C600030BD0EF1010E9645F7D1024830BD014826
:104C7000704700BF360CF100C0B32DE9F0434C1E65
:104C8000B4F5047F1DD2E3B1DAB100252E46A84663
:104C90002C46CF0003F1FF394FEA541C04F01F0EDD
:104CA00050F82C10BEF11F0F21FA0EFC0CD00CF0A6
:104CB000010C4CB90126E04634463546ECE79642F5
:104CC00016D90C48BDE8F083AB420BD0C44508BFF1
:104CD0000136A945F3D001350134BC42DCD10020B6
:104CE000BDE8F0830125E0462E46F5E70148704710
:104CF0001D46F1E7370CF1002DE9F04F91B08346E6
:104D0000DDE91B460D46002E6ED10F691C600023A5
:104D10001A990B60002A00F02F819D4B6A6AD3F824
:104D20003811D3F830319A4269D10A2967D19BF8FA
:104D30000330089304F10803079304230593954B6C
:104D4000934CA3FB07239B0803EB4303A7EB43030D
:104D5000039306971A9B069E1E60002E00F0EA80C1
:104D600000F096FC00230993BBF1000F00F0D58002
:104D700098464FF0010ADDF81C90002D00F0CD8020
:104D8000089B002B3DD0284608A900F071FC0028A4
:104D900039D0814B984220D0089B082B00F0E4804A
:104DA00000225B000893294608AB58460092FFF7A3
:104DB00091FE7A4B984200F0D38070B9DBF8002066
:104DC000130A03F47F03134323F07F43CBF800302F
:104DD000059B013B0593BDD10020039000F058FCDA
:104DE000039811B0BDE8F08F4FF47F01D1F80C0C9F
:104DF00001300CBF4FF40477D1F80C7C86E768488B
:104E0000EBE76648C5E72946089800F017FC00283C
:104E1000BFD1089B082B00F0A980042B00F0A980CB
:104E2000A3F10203B3FA83F35B090493C4F8C4A1AA
:104E3000C4F840A1C4F8C4A16B6AC4F83031D4F8F6
:104E400030219342F6D100234FF0FF30C4F82C31CB
:104E5000FFF77EFC002318466FF01B03C4F80031F7
:104E6000FFF784FC049B4B4FC4F80C31D4F8040AC0
:104E700040F48060FFF77AFC0A23C4F838312B69CC
:104E800009A8A7FB03236A6A1B0902FB03F303EBD0
:104E90004303DB039B09C4F8D831C4F82CA1DBF829
:104EA0000030089923F07F420B0243EA0163134369
:104EB000CBF8003000F0B2FB099B03F01A03034368
:104EC0007FF46AAFA7FB0637D4F81431B8EB970F1D
:104ED0000A93D4F818310B93D4F81C310C93D4F8FE
:104EE00020310D93D4F824310E93D4F828310F9348
:104EF00001D1039B9BB9484618220AA9183EFFF727
:104F0000B5FC09F1180908F101089EB100F0C0FBD9
:104F100000230993002D7FF433AF224839E7484638
:104F20001A46F61A0AA9994408F10108FFF79EFCEF
:104F3000002EEBD1069F079E6A6939463046FFF77F
:104F400069FEAA6940B94FF4806339463046FFF7DD
:104F500093FE00283FF440AF00231A9A136018E72D
:104F60002B6A002B3FF439AF0F4836E70323049335
:104F70005CE70223049359E701222946584600962C
:104F800008ABFFF7A7FD00283FF4D4AE25E700BF2C
:104F900000108450ABAAAAAA020CF100310CF10057
:104FA000300CF100350CF100320CF10010B4DDE9E9
:104FB000013401940024DDF80CC0CDE902C410BC1A
:104FC000FFF79ABE30B51546012487B005AB0093B4
:104FD0000022CDE9015404ABFFF78EFE07B030BDCF
:104FE000F0B587B0002966D01E46002B63D014466A
:104FF000002A60D0314F0D4638684FF0FF31FFF77F
:105000004FFC00284DD10020FFF77AFC002844D146
:105010002B4800F03FFAD8B101204FF0FF35FFF7E1
:105020006FFC002835D14FF408712648FEF70EFFBB
:1050300004212548FEF70AFF21482821FEF706FF34
:105040003868FFF735FC00282FD1284607B0F0BD9F
:105050001C4A0346029205AA019204AA03900092F8
:10506000174902461848FFF7A1FF03460028D3D18D
:1050700028461D46059B22469C4228BF1A46049995
:1050800032600831FFF7F2FB0120FFF739FC0028FE
:10509000C9D00E48FFF79AFCC5E70D48FFF796FC0C
:1050A000B6E70C48FFF792FCADE70B48FFF78EFC24
:1050B000284607B0F0BD4FF0FF35C6E7D4100020FA
:1050C0007C250020A425002078250020B05E01006A
:1050D000905E0100785E0100545F010010B5044647
:1050E00028B12046BDE81040F421FFF7C1BB0448B9
:1050F000FFF76CFC2046BDE81040F421FFF7B8BB79
:105100006C5F010010B1F421FEF7A0BE704700BF34
:1051100008B521B1012908D06FF0360008BD012182
:1051200000F058F80028F7D108BD022100F052F82D
:105130000028F9D0F0E700BF30B505468818B0F573
:10514000801F0B461446A1B001D8802A0CD9B3F5B4
:10515000801F17D922461946284600F07DF80446DC
:1051600084B9204621B030BD6846FFF77FFB224658
:105170006946284600F070F8802104466846FFF72B
:1051800077FBEDE76FF03604EBE700BF70B5E8B1F1
:105190000E46D9B1044600F031F80546B0B923688F
:1051A000012B0BD0022B01D0284670BD1C223046AB
:1051B00004F10801FFF75AFB284670BD2022304653
:1051C00004F10801FFF752FB284670BD6FF0360569
:1051D000EAE700BF78B138B50D46F0210446FFF785
:1051E00047FB402320462560E36500F091FA003834
:1051F00018BF012038BD0120704700BFF0B5056E13
:10520000A5B0044604AEE5B900230127019330465A
:105210006760294602AA009300F046FA10B1012007
:1052200025B0F0BD2A46204602A900F099FA0028D0
:10523000F5D1204600F0AAFB0028F0D1206625B069
:10524000F0BD802D2A46304628BF802204F164013B
:10525000FFF70CFB256ED7E7002800F0AE802DE9A4
:10526000F04F1446A5B0002A3DD00F46002949D082
:10527000B2F5803F0546006E20D34FF6FF7805F16A
:10528000640AEB6D1A1AB2FBF3F103FB1122002A38
:1052900065D18342B9464FF6FF7672D0B6FBF3FB79
:1052A00003FB0BFBBBF1000F30D1002E45D1A4F561
:1052B0007F44FF3CB4F5803F4744E2D2EA6D161AC2
:1052C000B6FBF2F302FB1366A64228BF2646002E69
:1052D00075D1824200F08D80B4FBF2F602FB06F637
:1052E0002EB9002C79D1002025B0BDE8F08F002325
:1052F00031463846CDE9003302AA00F0D5F900283E
:1053000000F09580012025B0BDE8F08F00235946BC
:105310004846CDE9003302AA00F0C6F90028F1D1D1
:105320005A46284602A900F01BFA0028EAD1A6EB4B
:105330000B06286ED944002EB9D0193049463246A2
:1053400005EB8000FFF792FAA4F57F44286EFF3C3E
:105350003044B4F5803F4744286692D2AEE74245D8
:1053600028BF4246164639465044FFF77FFA286E5A
:10537000EB6D3044834207EB06092866A8EB06066E
:105380008CD1802B28BF802351461A4604A8FFF7F2
:105390006DFA0023E96D02AACDE9003304A800F0FC
:1053A00083F90028AED12846EA6D02A900F0D8F9A9
:1053B0000028A7D1EB6D286670E70120704705F142
:1053C0006403394632461844FFF750FA286EEA6DF6
:1053D0003044A41B374428667BE72B6E22461933E2
:1053E00005EB83003946FFF741FA2B6E23442B6609
:1053F00079E7802A28BF802205F1640104A8FFF71D
:1054000035FA0023E96D04A8CDE9003302AA00F0C3
:105410004BF900287FF476AF2846EA6D02A900F028
:105420009FF900287FF46EAFEA6D286654E7324694
:10543000284602A900F094F900287FF463AF3744AE
:10544000A41B4EE7F8B51C460546114816460F4604
:10545000FFF744FE21460E48FFF75AFE044620B1EE
:105460000B48FFF74FFE2046F8BD3A46294608484C
:10547000FFF762FE04460028F2D131460448FFF7E8
:1054800085FE04460248FFF73DFE2046F8BD00BFFA
:10549000C42700201C2370B582B001A905460193E2
:1054A00000F032F8044638B9019B1C2B07D0144C8D
:1054B0001C212846FFF7DCF9204602B070BDD5E973
:1054C0000112131E18BF0123003918BF0121012644
:1054D00028689B00EA6843EA4103002818BF43F0AC
:1054E0000103EE612AB9C5E90834002BE4D1054C6B
:1054F000DEE7204643F00803C5E9083402B070BD7A
:10550000370CF0000E0CF0000346002866D000298E
:1055100064D00A681C2A61D14FF47F023B49D2F85B
:10552000100C88425CD0D2F8101C013158D0D2F84F
:10553000101C4FF47F021960D2F8140C34498842D1
:1055400060D0D2F8141C01315CD0D2F8141C4FF496
:105550007F025960D2F8181C11F5947F4FD0D2F811
:10556000181C01314BD0D2F8181C4FF47F029960FF
:10557000D2F81C0C274988423ED0D2F81C1C0131BD
:105580003AD0D2F81C1C4FF47F02D960D2F8001C2C
:1055900070312FD0D2F8001C01312BD0D2F8001C72
:1055A0004FF47F021961D2F8041CAF3120D0D2F839
:1055B000041C01311CD0D2F8041C4FF47F02596145
:1055C000D2F8080C144988420DD0D2F8081C0131D9
:1055D00009D0D2F8082C00209A617047012070474A
:1055E00040F6FC01A5E740F2373200209A6170478F
:1055F0005121E2E79021D3E742F60411C3E740F6D8
:10560000D861B2E742F2D001A1E700BFFCF8FFFF8A
:10561000D020FFFF0429FFFF37F3FFFF014608B545
:105620004FF48060FFF7AEF80022034BC3F8C821A7
:10563000C3F82C2108BD00BF001084500138072892
:1056400005D8DFE800F0100E040A04040406074839
:105650007047CB6800204B6270478B6800204B621C
:1056600070474B68F6E70B68F4E700BF310CF100B8
:105670000B6802E0082B0B6006D8026A13424FEA5F
:105680004303F7D00020704700487047310CF10009
:105690000022044B4FF48060C3F82C21C3F8C421CE
:1056A000FFF756B800108450F0B5002483B0B0F175
:1056B000005F8DF8074025D38C468444BCF1804FB1
:1056C00004461FD817461D4601220DF1070300F0BE
:1056D00097F90646B0B99DF80730099A3C603B71CE
:1056E00092B14DB10246089928460DF1070300F02A
:1056F00087F938B99DF807303046099A156013715B
:1057000003B0F0BD4FF47506304603B0F0BD00BFE6
:10571000D8B108B50368012B04D0022B0FD043B1D8
:105720000B4808BD20220B490830FFF79FF80020E6
:1057300008BD142208490830FFF798F8F7E720223F
:1057400006490830FFF792F8F1E74FF4730070470D
:105750000100F3007C5F0100BC5F01009C5F010061
:105760002DE9F843002900F0F9800446002800F0F4
:10577000F98003680F469046002B00F0C380013B80
:10578000012B00F2D7804FF0FF3178484FF002092B
:10579000FFF786F8002840F0BF800020FFF7B0F840
:1057A0000646002840F0C280714AD2F81C39002B0E
:1057B000FBD16F4DD5F8203C002BFBD14FF0FF30D3
:1057C000FEF7C6FFD5F8040A20F04000FEF7CEFF32
:1057D00001230722C5F81838C5F80029C5F8C437D1
:1057E000A36CC5F8CC37E36CC5F8D037C5F8C097C3
:1057F00023685BB1013B012B18D8636AC5F85C369E
:10580000236AC5F85836E369C5F85436A269584B7F
:10581000C3F850266269C3F84C262269C3F84826AB
:10582000E268C3F84426A268C3F84026504AD2F87A
:105830001039002BFBD1B8F1000F5FD06368402016
:10584000012B08BFC2F884363A68494BC3F8282CAC
:10585000C3F82C8CFEF790FF0646454AD2F8103963
:10586000002BFBD1424AD2F8203C002BFBD123680D
:105870005BB1013B012B18D8D2F85C366362D2F8D9
:1058800058362362D2F85436E361394BD3F85026A8
:10589000A261D3F84C266261D3F848262261D3F87E
:1058A0004426E260D3F84036A36000230121304A49
:1058B000D2F8CC07A064D2F8D007E064C2F8C417CD
:1058C000C2F88436C2F8C837D2F81039002BFBD1A1
:1058D000C2F81838002E3BD1254BD3F8040A40F00B
:1058E0004000FEF743FF0120FFF70AF860BB1F48A6
:1058F000FEF7DEFF10BB3046BDE8F8830423C2F894
:10590000C837AAE74FF0FF3118484FF00109FEF7FA
:10591000C7FF00283FF441AF1648FFF757F80020B3
:10592000FEF7EEFF064600283FF43EAF1248FFF7B1
:105930004DF839E7114E3046BDE8F8831048FFF7BF
:1059400045F83046BDE8F8830E48FFF73FF8CEE74C
:10595000102104F10800FEF78BFFBDE70A4E304628
:10596000BDE8F8834FF47306C5E700BFE4100020DC
:1059700000108450785E0100905E01000100F30089
:10598000D05E0100B05E01000300F300A0B3034647
:1059900070B4D0E90240D3E9041226BA05BA0CBAB1
:1059A00010BAC3E90440D3E90612986A09BAC3E9F8
:1059B000026512BA996100BAD3E9084125BA0CBA56
:1059C000C3E90725D3E90B12C3E9094009BAD86B2B
:1059D00012BAD962D3E90D4125BAC3E90C250CBA34
:1059E00000BAD3E9101209BA12BAC3E90E40196419
:1059F00000205A6470BC70474FF47300704700BFBA
:105A000000201870704700BF08B5074B044613B15B
:105A10000021AFF30080054B1868836A03B19847F3
:105A2000204600F08DF800BF00000000D05F0100AC
:105A300070B50D4D00260D4C641BA410A64209D173
:105A40000B4D00260B4C00F0FDF9641BA410A64280
:105A500005D170BD55F8043B01369847EEE755F87F
:105A6000043B01369847F2E7A0110020A011002066
:105A7000A0110020A4110020431810B501D21F2A44
:105A800001D9002010BD013902F014030144102B8C
:105A900080EA01043CD009DC8BB1042BF1D11F2C2E
:105AA00040E840F315D941E840F10EE0142BE8D16D
:105AB0001F2C40E8C0F30CD941E8C0F105E01F2CD1
:105AC00040E800F305D941E800F11C460B468C4242
:105AD000D7D122F01402013A0A2AD2D801A151F8F2
:105AE00022F000BF335B01002D5B01001F5B010052
:105AF000835A0100835A0100835A0100835A01002E
:105B0000395B0100335B0100275B01001F5B010073
:105B10001F2C40E880F3DCD941E880F1D5E713F48D
:105B2000001FAFD1ADE713F4801FFAE75B02A9D5E0
:105B3000A7E713F4002FF4E713F4802FF1E700BF79
:105B4000FEE700BF002383F300887047FDF710BB1A
:105B5000EFF30880EFF309812DE9F00F6B467246F1
:105B6000FBF78AF808B0FFF7F1FFFEE7FDF700BB8F
:105B7000EFF30880EFF309812DE9F00F6B467246D1
:105B8000FBF77AF808B0FFF7F1FFFEE7FDF7F0BA90
:105B9000EFF30880EFF309812DE9F00F6B467246B1
:105BA000FBF76AF808B0FFF7F1FFFEE7FDF7E0BA90
:105BB000EFF30880EFF309812DE9F00F6B46724691
:105BC000FBF75AF808B0FFF7F1FFFEE7FDF7D0BA90
:105BD000EFF30880EFF309812DE9F00F6B46724671
:105BE000FBF74AF808B0FFF7F1FFFEE7814270B417
:105BF0000546144602D370BC00F02EB8821821442A
:105C00003CB141EA020313F003030FD1E01803286B
:105C100012D86FF00300A3084343002019441A442C
:105C20002344984210D1284670BC704711F8013DBA
:105C3000013C02F8013DE3E7581850F8046C98184D
:105C400040F8046C043BE1E70C1A14F8016C141AD8
:105C500004F8016C0130E4E770B504463AB141EA5A
:105C6000040313F003030CD1D518032D0FD822F031
:105C700003031C441944002302F0030293420CD195
:105C800070BD11F8013B013A04F8013BE6E7CD1A7B
:105C90002E68E51A2E60043BE6E75D5CE5540133AF
:105CA000ECE7F0B5044662B922F00303234402F0A6
:105CB00003021A44934214D1F0BD04F8011B013AC7
:105CC000F1E7A307F9D115460B0443EA01630B433F
:105CD00043EA01231619032DE6D9771B3B60043DE7
:105CE000F9E703F8011BE5E708B5EFF30583C3F314
:105CF00008030BB1FDF73CFABDE80840FDF7C0BA58
:105D000010B50446EFF30583C3F308030BB1FDF7A9
:105D10002FFA2046BDE81040FDF7B5BA2DE9F04155
:105D200004460D4616461F46EFF30583C3F30803EA
:105D30000BB1FDF71DFA3B46324629462046BDE829
:105D4000F041FCF7E9BC2DE9F04104460D4616464A
:105D50001F46EFF30583C3F308030BB1FDF708FA01
:105D60003B46324629462046BDE8F041FCF70EBDD1
:105D700008B5EFF30583C3F308030BB1FDF7F8F99A
:105D8000BDE80840FDF74FBA00207047704710B5D6
:105D9000044608B1FDF784FF2046BDE81040FDF73A
:105DA0006FBF10B50446406A10B1A16AFFF7EFFF5C
:105DB0000020C4E9090010BD38B50446FFF7F1FF23
:105DC000236A2C22012B0CBF05466FF0960500219B
:105DD0002046FFF766FF284638BD00207047704711
:105DE0000020704713B5002001AB1446FEF70CF8F5
:105DF00030B9019BA34218BF6FF0930002B010BDF1
:105E00006FF09200FAE7002070472DE9E04F274637
:105E1000A046A146A246A346A446A2B02DEC000A85
:105E200084F3008825462646A447EFF3148515F031
:105E3000080F18BFB0EE400A3DEC000A22B0BDE8E2
:105E4000E08F0000F8B500BFF8BC08BC9E46704764
:105E5000F8B500BFF8BC08BC9E467047FF8FFFFF37
:105E6000FF8FFFFFFE8FFFFFFE8FFFFFFD8FFFFF06
:105E7000FC8FFFFFFC8FFFFF4661696C20746F2071
:105E800061637175697265206D757465780A0000CB
:105E90004661696C20746F20696E63726561736519
:105EA00020504D20636F756E7465720A000000000B
:105EB0004661696C20746F20646563726561736507
:105EC00020504D20636F756E7465720A00000000EB
:105ED0004661696C20746F2072656C656173652022
:105EE0006D757465780A0000436F756C64206E6F81
:105EF00074206C6F636B20706F77657220736176AE
:105F000065206D75746578006D757465785F66726F
:105F100065652063616C6C65642077697468204EE8
:105F2000554C4C20706172616D65746572000000A3
:105F300043616E277420696E697469616C697A6562
:105F4000206D757465782C20776173204E554C4C0C
:105F50000D0A00004661696C20746F20756E6C6FCD
:105F6000636B206D757465780A0000000A637478AD
:105F7000206973204E554C4C0A00000067E6096A00
:105F800085AE67BB72F36E3C3AF54FA57F520E515A
:105F90008C68059BABD9831F19CDE05BD89E05C1EA
:105FA00007D57C3617DD703039590EF7310BC0FF3D
:105FB00011155868A78FF964A44FFABE01234567ED
:105FC00089ABCDEFFEDCBA9876543210F0E1D2C343
:105FD0004011002054464D5F43525950544F0054D5
:105FE000464D5F504C4154464F524D5F53455256BB
:105FF00049434500000000000000000000000000D0
:107C00007FE97FE9FBF7ECBD7FE97FE9FBF7F7BD93
:107C10007FE97FE9FBF71FBE7FE97FE9FBF712BE33
:107C20007FE97FE9FBF7FABD0000000000000000DB
:107C30000000000000000000000000000000000044
:107C40007AFFFFFF008000500000000014360100A2
:107C50000200000000000000000000000000000022
:107C6000000000000000000090ED00E000A00350C4
:107C70007FA60350008000506F8500501412002032
:107C8000A8110020440301008D5D0100895D010001
:107C9000A35C0100DC1000200C1100200411002066
:107CA00000110020FC1000209D49010091490100B5
:107CB0008549010000000000A94901003811002099
:107CC00030110020281100200000000020110020A9
:107CD000B54A0100014A0100354A01007D4A010010
:107CE000682500203A00003A6C2500203A00003A4E
:107CF000702500203A00003A742500203A00003A2E
:107D00000000000000000000000000000000000073
:107D10000000000000000000000000000000000063
:107D20000000000000000000000000000000000053
:107D30000000000000000000000000000000000043
:107D40000000000000000000000000000000000033
:107D50000000000000000000000000000000000023
:087D6000D5380100AD38010027
:10800000A805012071CB0100CD9A02005DCB0100D3
:108010005DCB01005DCB01005DCB01005DCB0100BC
:1080200000000000000000000000000029CD010059
:108030005DCB010000000000E1CC01005DCB010040
:10804000ADCE0100ADCE0100ADCE0100ADCE010040
:10805000ADCE0100ADCE0100ADCE0100ADCE010030
:10806000ADCE0100ADCE0100ADCE0100ADCE010020
:10807000ADCE0100ADCE0100ADCE0100ADCE010010
:10808000ADCE0100ADCE0100ADCE0100ADCE010000
:10809000ADCE0100ADCE0100ADCE0100ADCE0100F0
:1080A000ADCE0100ADCE0100ADCE0100ADCE0100E0
:1080B000ADCE0100ADCE0100ADCE0100ADCE0100D0
:1080C000ADCE0100ADCE0100ADCE0100ADCE0100C0
:1080D000ADCE0100ADCE0100ADCE0100ADCE0100B0
:1080E000ADCE0100ADCE0100ADCE0100ADCE0100A0
:1080F000ADCE0100ADCE0100ADCE0100ADCE010090
:10810000ADCE0100ADCE0100ADCE0100ADCE01007F
:10811000ADCE0100ADCE0100ADCE0100ADCE01006F
:10812000ADCE0100ADCE0100ADCE0100ADCE01005F
:10813000ADCE0100ADCE0100ADCE0100ADCE01004F
:10814000ADCE0100FFFFFFFF81F0004102E000BF64
:1081500083F0004330B54FEA41044FEA430594EA07
:10816000050F08BF90EA020F1FBF54EA000C55EA42
:10817000020C7FEA645C7FEA655C00F0E2804FEA13
:108180005454D4EB5555B8BF6D420CDD2C4480EAF5
:10819000020281EA030382EA000083EA010180EA25
:1081A000020281EA0303362D88BF30BD11F0004F73
:1081B0004FEA01314FF4801C4CEA113102D04042A9
:1081C00061EB410113F0004F4FEA03334CEA1333E4
:1081D00002D0524263EB430394EA050F00F0A780FC
:1081E000A4F10104D5F1200E0DDB02FA0EFC22FAF7
:1081F00005F2801841F1000103FA0EF2801843FAEB
:1082000005F359410EE0A5F120050EF1200E012ADB
:1082100003FA0EFC28BF4CF0020C43FA05F3C01819
:1082200051EBE37101F0004507D54FF0000EDCF192
:10823000000C7EEB00006EEB0101B1F5801F1BD33B
:10824000B1F5001F0CD349085FEA30004FEA3C0C3F
:1082500004F101044FEA445212F5800F80F09A8035
:10826000BCF1004F08BF5FEA500C50F1000041EB39
:10827000045141EA050130BD5FEA4C0C404141EB3D
:108280000101013C28BFB1F5801FE9D291F0000F38
:1082900004BF01460020B1FA81F308BF2033A3F1E7
:1082A0000B03B3F120020CDA0C3208DD02F1140CDE
:1082B000C2F10C0201FA0CF021FA02F10CE002F119
:1082C0001402D8BFC2F1200C01FA02F120FA0CFC12
:1082D000DCBF41EA0C019040E41AA2BF01EB04515B
:1082E000294330BD6FEA04041F3C1CDA0C340EDC59
:1082F00004F11404C4F1200220FA04F001FA02F39C
:1083000040EA030021FA04F345EA030130BDC4F159
:108310000C04C4F1200220FA02F001FA04F340EA4E
:108320000300294630BD21FA04F0294630BD94F0FF
:10833000000F83F4801306BF81F480110134013DE6
:108340004EE77FEA645C18BF7FEA655C29D094EA57
:10835000050F08BF90EA020F05D054EA000C04BFD5
:108360001946104630BD91EA030F1EBF00210020C0
:1083700030BD5FEA545C05D14000494128BF41F05F
:10838000004130BD14F580043CBF01F5801130BDC3
:1083900001F0004545F0FE4141F470014FF000004E
:1083A00030BD7FEA645C1ABF194610467FEA655CFF
:1083B0001CBF0B46024650EA013406BF52EA0335A1
:1083C00091EA030F41F4002130BD00BF90F0000F8F
:1083D00004BF0021704730B54FF4806404F13204CB
:1083E0004FF000054FF0000150E700BF90F0000F84
:1083F00004BF0021704730B54FF4806404F13204AB
:1084000010F0004548BF40424FF000013EE700BF7A
:1084100042004FEAE2014FEA31014FEA02701FBF0A
:1084200012F07F4393F07F4F81F06051704732F03C
:108430007F4208BF704793F07F4F04BF41F4002193
:10844000704730B54FF4607401F0004521F00041F1
:108450001CE700BF50EA010208BF704730B54FF07B
:1084600000050AE050EA010208BF704730B511F07C
:10847000004502D5404261EB41014FF4806404F1B4
:1084800032045FEA915C3FF4D8AE4FF003025FEA3A
:10849000DC0C18BF03325FEADC0C18BF033202EBBE
:1084A000DC02C2F1200300FA03FC20FA02F001FA18
:1084B00003FE40EA0E0021FA02F11444BDE600BFBB
:1084C00070B54FF0FF0C4CF4E06C1CEA11541DBF6A
:1084D0001CEA135594EA0C0F95EA0C0F00F0DEF835
:1084E0002C4481EA030621EA4C5123EA4C5350EA1A
:1084F000013518BF52EA033541F4801143F480136B
:1085000038D0A0FB02CE4FF00005E1FB02E506F0FB
:108510000042E0FB03E54FF00006E1FB03569CF050
:10852000000F18BF4EF0010EA4F1FF04B6F5007F56
:1085300064F5407404D25FEA4E0E6D4146EB0606C8
:1085400042EAC62141EA55514FEAC52040EA5E5051
:108550004FEACE2EB4F1FD0C88BFBCF5E06F1ED8FB
:10856000BEF1004F08BF5FEA500E50F1000041EB32
:10857000045170BD06F0004646EA010140EA0200DF
:1085800081EA0301B4EB5C04C2BFD4EB0C0541EA01
:10859000045170BD41F480114FF0000E013C00F316
:1085A000AB8014F1360FDEBF002001F0004170BD3A
:1085B000C4F10004203C35DA0C341BDC04F1140453
:1085C000C4F1200500FA05F320FA04F001FA05F2DF
:1085D00040EA020001F0004221F0004110EBD370AC
:1085E00021FA04F642EB06015EEA430E08BF20EAD8
:1085F000D37070BDC4F10C04C4F1200500FA04F37B
:1086000020FA05F001FA04F240EA020001F000410C
:1086100010EBD37041F100015EEA430E08BF20EA7F
:10862000D37070BDC4F1200500FA05F24EEA020EC7
:1086300020FA04F301FA05F243EA020321FA04F0F6
:1086400001F0004121FA04F220EA020000EBD370AD
:108650005EEA430E08BF20EAD37070BD94F0000FAD
:108660000FD101F00046400041EB010111F4801FE1
:1086700008BF013CF7D041EA060195F0000F18BF92
:10868000704703F00046520043EB030313F4801FCE
:1086900008BF013DF7D043EA0603704794EA0C0F88
:1086A0000CEA135518BF95EA0C0F0CD050EA41069E
:1086B00018BF52EA4306D1D181EA030101F000411B
:1086C0004FF0000070BD50EA410606BF1046194643
:1086D00052EA430619D094EA0C0F02D150EA01364F
:1086E00013D195EA0C0F05D152EA03361CBF104690
:1086F00019460AD181EA030101F0004141F0FE412F
:1087000041F470014FF0000070BD41F0FE4141F4B2
:10871000780170BD70B54FF0FF0C4CF4E06C1CEAB2
:1087200011541DBF1CEA135594EA0C0F95EA0C0F67
:1087300000F0A7F8A4EB050481EA030E52EA033522
:108740004FEA013100F088804FEA03334FF0805543
:1087500045EA131343EA12634FEA022245EA111570
:1087600045EA10654FEA00260EF000419D4208BF21
:10877000964244F1FD0404F5407402D25B084FEACE
:108780003202B61A65EB03055B084FEA32024FF47A
:1087900080104FF4002CB6EB020E75EB030E22BFD7
:1087A000B61A754640EA0C005B084FEA3202B6EB97
:1087B000020E75EB030E22BFB61A754640EA5C0046
:1087C0005B084FEA3202B6EB020E75EB030E22BFD6
:1087D000B61A754640EA9C005B084FEA3202B6EBD7
:1087E000020E75EB030E22BFB61A754640EADC0096
:1087F00055EA060E18D04FEA051545EA16754FEAF8
:1088000006164FEAC30343EA52734FEAC2025FEA15
:108810001C1CC0D111F4801F0BD141EA00014FF0A4
:1088200000004FF0004CB6E711F4801F04BF014375
:108830000020B4F1FD0C88BFBCF5E06F3FF6AFAE91
:10884000B5EB030C04BFB6EB020C5FEA500C50F121
:10885000000041EB045170BD0EF0004E4EEA1131A4
:1088600014EB5C04C2BFD4EB0C0541EA045170BDAB
:1088700041F480114FF0000E013C90E645EA060EEF
:108880008DE60CEA135594EA0C0F08BF95EA0C0F1D
:108890003FF43BAF94EA0C0F0AD150EA01347FF465
:1088A00034AF95EA0C0F7FF425AF104619462CE73C
:1088B00095EA0C0F06D152EA03353FF4FDAE10469F
:1088C000194622E750EA410618BF52EA43067FF4F0
:1088D000C5AE50EA41047FF40DAF52EA43057FF480
:1088E000EBAE12E74A0011D212F5001211D20DD5EB
:1088F0006FF47873B3EB62520ED44FEAC12343F0A6
:10890000004343EA505323FA02F070474FF000004F
:10891000704750EA013002D14FF0FF3070474FF0FE
:10892000000070474FEA4102B2F1E04324BFB3F5C3
:10893000001CDCF1FE5C0DD901F0004C4FEAC002D6
:108940004CEA5070B2F1004F40EB830008BF20F0BA
:108950000100704711F0804F21D113F13872BCBF74
:1089600001F00040704741F480114FEA5252C2F1C9
:108970001802C2F1200C10FA0CF320FA02F018BF12
:1089800040F001004FEAC1234FEAD32303FA0CFC65
:1089900040EA0C0023FA02F34FEA4303CCE77FEAF4
:1089A000625307D150EA01331EBF4FF0FE4040F43E
:1089B0004000704701F0004040F0FE4040F40000ED
:1089C000704700BF80F0004002E000BF81F000412E
:1089D00042001FBF5FEA410392EA030F7FEA226C65
:1089E0007FEA236C6AD04FEA1262D2EB1363C1BFF5
:1089F000D218414048404140B8BF5B42192B88BF64
:108A0000704710F0004F40F4000020F07F4018BF86
:108A1000404211F0004F41F4000121F07F4118BFA6
:108A2000494292EA030F3FD0A2F1010241FA03FC4E
:108A300010EB0C00C3F1200301FA03F100F0004336
:108A400002D5494260EB4000B0F5000F13D3B0F1FE
:108A5000807F06D340084FEA310102F10102FE2A6D
:108A600051D2B1F1004F40EBC25008BF20F00100DD
:108A700040EA03007047490040EB0000013A28BF7C
:108A8000B0F5000FEDD2B0FA80FCACF1080CB2EBFF
:108A90000C0200FA0CF0AABF00EBC250524218437D
:108AA000BCBFD0401843704792F0000F81F4000122
:108AB00006BF80F400000132013BB5E74FEA4103F5
:108AC0007FEA226C18BF7FEA236C21D092EA030F61
:108AD00004D092F0000F08BF0846704790EA010FDB
:108AE0001CBF0020704712F07F4F04D1400028BF08
:108AF00040F00040704712F100723CBF00F50000EA
:108B0000704700F0004343F0FE4040F4000070471F
:108B10007FEA226216BF08467FEA236301464202CB
:108B200006BF5FEA412390EA010F40F480007047DE
:108B30004FF0000304E000BF10F0004348BF404284
:108B40005FEA000C08BF704743F0964301464FF0C0
:108B500000001CE050EA010208BF70474FF000031C
:108B60000AE000BF50EA010208BF704711F000435D
:108B700002D5404261EB41015FEA010C02BF84462D
:108B80000146002043F0B64308BFA3F18053A3F58C
:108B90000003BCFA8CF2083AA3EBC25310DB01FAD3
:108BA00002FC634400FA02FCC2F12002BCF1004F57
:108BB00020FA02F243EB020008BF20F001007047E8
:108BC00002F1200201FA02FCC2F1200250EA4C003C
:108BD00021FA02F243EB020008BF20EADC70704782
:108BE0004FF0FF0C1CEAD0521EBF1CEAD15392EA90
:108BF0000C0F93EA0C0F6FD01A4480EA010C40026C
:108C000018BF5FEA41211ED04FF0006343EA5010C5
:108C100043EA5111A0FB01310CF00040B1F5000F07
:108C20003EBF490041EAD3715B0040EA010062F1B6
:108C30007F02FD2A1DD8B3F1004F40EBC25008BFA0
:108C400020F00100704790F0000F0CF0004C08BFBE
:108C500049024CEA502040EA51207F3AC2BFD2F18B
:108C6000FF0340EAC250704740F400004FF0000399
:108C7000013A5DDC12F1190FDCBF00F000407047D3
:108C8000C2F10002410021FA02F1C2F1200200FA11
:108C900002FC5FEA310040F1000053EA4C0308BFD8
:108CA00020EADC70704792F0000F00F0004C02BF29
:108CB000400010F4000F013AF9D040EA0C0093F0A4
:108CC000000F01F0004C02BF490011F4000F013BFE
:108CD000F9D041EA0C018FE70CEAD15392EA0C0F6C
:108CE00018BF93EA0C0F0AD030F0004C18BF31F0D7
:108CF000004CD8D180EA010000F00040704790F0AD
:108D0000000F17BF90F0004F084691F0000F91F050
:108D1000004F14D092EA0C0F01D142020FD193EA16
:108D20000C0F03D14B0218BF084608D180EA01009E
:108D300000F0004040F0FE4040F40000704740F07A
:108D4000FE4040F4400070474FF0FF0C1CEAD05248
:108D50001EBF1CEAD15392EA0C0F93EA0C0F69D0A4
:108D6000A2EB030280EA010C49024FEA402037D00F
:108D70004FF0805343EA111143EA10130CF0004006
:108D80008B4238BF5B0042F17D024FF4000C8B42F6
:108D900024BF5B1A40EA0C00B3EB510F24BFA3EBD6
:108DA000510340EA5C00B3EB910F24BFA3EB9103A6
:108DB00040EA9C00B3EBD10F24BFA3EBD10340EA00
:108DC000DC001B0118BF5FEA1C1CE0D1FD2A3FF646
:108DD00050AF8B4240EBC25008BF20F001007047FB
:108DE0000CF0004C4CEA50207F32C2BFD2F1FF039E
:108DF00040EAC250704740F400004FF00003013ACF
:108E000037E792F0000F00F0004C02BF400010F472
:108E1000000F013AF9D040EA0C0093F0000F01F086
:108E2000004C02BF490011F4000F013BF9D041EAA8
:108E30000C0195E70CEAD15392EA0C0F08D14202DB
:108E40007FF47DAF93EA0C0F7FF470AF084676E7AE
:108E500093EA0C0F04D14B023FF44CAF08466EE787
:108E600030F0004C18BF31F0004CCAD130F0004255
:108E70007FF45CAF31F000437FF43CAF5FE700BFAD
:108E80004FF0FF3C06E000BF4FF0010C02E000BFD6
:108E90004FF0010C4DF804CD4FEA40024FEA410378
:108EA0007FEA226C18BF7FEA236C11D001B052EA2E
:108EB000530C18BF90EA010F58BFB2EB030088BFF4
:108EC000C81738BF6FEAE17018BF40F00100704763
:108ED0007FEA226C02D15FEA402C05D17FEA236C45
:108EE000E4D15FEA412CE1D05DF8040B704700BF8C
:108EF000844608466146FFE70FB5FFF7C9FF002823
:108F000048BF10F1000F0FBD4DF808EDFFF7F4FF5B
:108F10000CBF012000205DF808FB00BF4DF808EDF4
:108F2000FFF7EAFF34BF012000205DF808FB00BF17
:108F30004DF808EDFFF7E0FF94BF012000205DF839
:108F400008FB00BF4DF808EDFFF7D2FF94BF0120EA
:108F500000205DF808FB00BF4DF808EDFFF7C8FFE3
:108F600034BF012000205DF808FB00BF4FEA40023B
:108F7000B2F1FE4F0FD34FF09E03B3EB12620DD947
:108F80004FEA002343F0004310F0004F23FA02F0B1
:108F900018BF404270474FF00000704712F1610F58
:108FA00001D1420205D110F0004008BF6FF000402F
:108FB00070474FF0000070477BB972B90029BEBFFF
:108FC00000204FF0004106E008BF00281CBF6FF0F2
:108FD00000414FF0FF3000F057B8ADF1080C6DE9DB
:108FE00004CE002909DB002B1ADB00F02BF9DDF899
:108FF00004E0DDE9022304B07047404261EB410127
:10900000002B1BDB00F01EF9DDF804E0DDE9022394
:1090100004B0404261EB4101524263EB43037047AD
:10902000524263EB430300F00DF9DDF804E0DDE9A3
:10903000022304B0404261EB41017047524263EBAE
:10904000430300F0FFF8DDF804E0DDE9022304B09B
:10905000524263EB4303704753B94AB9002908BF32
:1090600000281CBF4FF0FF314FF0FF3000F00CB86C
:10907000ADF1080C6DE904CE00F0E4F8DDF804E091
:10908000DDE9022304B07047704700BF4FF0FF3C9A
:1090900006E000BF4FF0010C02E000BF4FF0010CF2
:1090A0004DF804CD4FEA410C7FEA6C5C4FEA430C6B
:1090B00018BF7FEA6C5C1BD001B050EA410C0CBFBA
:1090C00052EA430C91EA030F02BF90EA020F00201C
:1090D000704710F1000F91EA030F58BF994208BF83
:1090E00090422CBFD8176FEAE37040F00100704740
:1090F0004FEA410C7FEA6C5C02D150EA013C07D197
:109100004FEA430C7FEA6C5CD6D152EA033CD3D0E1
:109110005DF8040B704700BF8446104662468C46DB
:109120001946634600E000BF01B5FFF7B7FF00280E
:1091300048BF10F1000F01BD4DF808EDFFF7F4FF37
:109140000CBF012000205DF808FB00BF4DF808EDC2
:10915000FFF7EAFF34BF012000205DF808FB00BFE5
:109160004DF808EDFFF7E0FF94BF012000205DF807
:1091700008FB00BF4DF808EDFFF7CEFF94BF0120BC
:1091800000205DF808FB00BF4DF808EDFFF7C4FFB5
:1091900034BF012000205DF808FB00BF4FEA410CFE
:1091A0007FEA6C5C02D150EA013C0AD14FEA430CE1
:1091B0007FEA6C5C02D152EA033C02D14FF000001E
:1091C00070474FF0010070474FEA410212F500125C
:1091D00015D211D56FF47873B3EB625212D94FEAFE
:1091E000C12343F0004343EA505311F0004F23FAE8
:1091F00002F018BF404270474FF00000704750EA3D
:10920000013005D111F0004008BF6FF000407047F9
:109210004FF00000704700BF4FEA40024FEA4103A1
:109220007FEA226C02D15FEA402C08D17FEA236CEE
:1092300002D15FEA412C02D14FF0000070474FF09D
:10924000010070472DE9F04786468C460846089E87
:10925000154674461946002B40F0C1808542B2FA8B
:1092600082F245D94AB1C2F1200300FA02FC9540CE
:1092700094402EFA03F343EA0C0C4FEA154EA8B2C1
:10928000230CBCFBFEF80EFB18CC08FB00F943EAEC
:109290000C43994528D9EB1808F1FF3704D29945BA
:1092A00002D9A8F102072B44A3EB0903A4B2B3FB34
:1092B000FEFC0EFB1C330CFB00F044EA0344A0420E
:1092C00014D92C190CF1FF3304D2A04202D9ACF10D
:1092D00002032C44241A43EA07401EB1D440002361
:1092E00034607360BDE8F0874746DDE76346F1E729
:1092F00092BB431B01214FEA154EAFB2200CB3FBCA
:10930000FEFC0EFB1C330CFB07F840EA03439845B8
:1093100061D9EB180CF1FF3004D2984502D9ACF1B9
:1093200002002B44A3EB0803A4B2B3FBFEFC0EFB2C
:109330001C330CFB07F744EA0344A7424DD92C1910
:109340000CF1FF3304D2A74202D9ACF102032C4442
:10935000E41B43EA0040C0E7C2F12003954094407B
:1093600020FA03F12EFA03F34FEA154E9040AFB204
:109370000343B1FBFEFC0EFB1C10190C0CFB07F8A1
:1093800041EA0041884522D969180CF1FF3004D226
:10939000884502D9ACF102002944A1EB08019BB237
:1093A000B1FBFEFC0EFB1C110CFB07F743EA01436B
:1093B0009F420ED9EB180CF1FF3104D29F4202D923
:1093C000ACF102012B44DB1B41EA004193E760460C
:1093D000E3E76146F7E76046A4E76346B8E7834200
:1093E00006D916B9002108467CE7C6E900E0F9E78E
:1093F000B3FA83F78FB9834201D3724508D8BEEB25
:10940000020460EB030301209C461EB9002169E7BA
:109410003846FAE7C6E9004CF8E7C7F1200CBB4034
:109420000EFA07F522FA0CF42EFA0CF1BA401C439E
:1094300020FA0CF3B8404FEA144901431FFA84FEA6
:10944000B3FBF9F809FB18300B0C08FB0EFA43EAE2
:1094500000439A4540D9E31808F1FF3004D29A45F9
:1094600002D9A8F102002344A3EB0A0389B2B3FB9B
:10947000F9F809FB183308FB0EFE41EA03418E455B
:109480002CD9611808F1FF3304D28E4502D9A8F116
:109490000203214443EA0040A1EB0E01A0FB029825
:1094A0004145CE46434602D306D14D4504D201384C
:1094B000B9EB020E68EB0403002EA7D0B5EB0E0249
:1094C00061EB030101FA0CFC22FA07F3F9404CEAC4
:1094D0000303C6E9003199E74046C5E74346D9E7AB
:1094E00010F8012B11F8013B012A28BF9A42F7D04E
:1094F000D01A7047034613F8012B002AFBD1181A23
:109500000138704700000000032973B50546144672
:1095100071D8002A40D0072A5CD15A681C681346CB
:109520003948D117C4FB0031012B71F1000225DB52
:1095300000F56E1000F65D70181841F1000130A3BF
:10954000D3E90023FFF738FD80B202281ED004289B
:109550001ED008281ED0102833D103232B492A6996
:1095600051F82310284611615268232114693022D2
:10957000A4461B0102B0BDE870406047244818189B
:1095800061F100011EA3D3E90023DBE70023E5E737
:109590000123E3E70223E1E71A881E4B33F8021B9D
:1095A0008A420BD12E692021736828469B680DF1F1
:1095B00007029847002807DA02B070BD01340B2C6F
:1095C000ECD16FF01500F7E79DF80720130704D4DE
:1095D000082C05D16FF08500EEE70A2C08BF09249E
:1095E000736802F00F0242EA041220212846DB6869
:1095F000D2B29847E0E702B0BDE8704005F070BC19
:109600003AA395000000000040420F00CCC50020A6
:10961000632EB5FFF4F402002DE9F04198460023D3
:1096200086B0CDE9043304230D4617460646019360
:10963000002800F0B580002900F0B280062104A8BF
:1096400012F041FC044648B103460121584A5948EA
:1096500012F099FD204606B0BDE8F081014604AA4B
:10966000304612F00BFC044648B10346524A012131
:10967000504812F088FD04A812F04FFCEAE76A4651
:10968000012104A812F0FBFC044610B103464B4A2A
:10969000EDE7009BB3B1042B1AD0052B0CBF0923B7
:1096A000FF232B70032101AB02AA04A812F013FDC3
:1096B000064678B10346424A01213E4812F063FD56
:1096C0003446D8E7002300202B706860A860D2E7FA
:1096D0000723E6E7019B002BF4D018336B4403F813
:1096E000100C02A9384614F098FD0222314602A857
:1096F0000EF08CFC2B78C0B2092B06D10F2824D990
:109700006FF0150423462F4AB1E70F28F8D8072B2E
:1097100022D12D4B2D4F33F81000D8B1FEF766FE45
:1097200021A3D3E90023FEF7CBFEFFF7FBF80421CA
:1097300068600DEB010302AA04A8019112F0CBFCB2
:10974000064660B10346224AB6E7224B224F33F861
:109750001000E2E72148EAE76FF07F04D2E7019BBF
:1097600002A918336B4403F8100C404614F055FD61
:109770000222314602A80EF049FCC3B20F2B07D9D2
:109780000121174A0B4812F0FEFC6FF0150472E736
:10979000581CC0B2FFF7D0F93946FFF721FA95E718
:1097A0006FF0150456E700BF7B14AE47E17A244002
:1097B000A410030014EB0200CD100300F610030008
:1097C00018110300441103002AF502000AD7A33F31
:1097D000681103000AF502000AD723400AD7A34004
:1097E0009311030000000000F8B506460F4600F094
:1097F0003BF81B4B04460D4693F90030013312D061
:109800003046394614F0C1FC68B13046394610A3E1
:10981000D3E90023FFF7B8FC40B110F0BEF90024F3
:109820002223104D036020462946F8BD0AA3D3E940
:10983000002330463946FFF789FC0028F3D010F0AA
:10984000ACF92223002400250360ECE7AFF300808D
:10985000EF39FAFE422E864051302DD5104987C08F
:10986000CBC700200000F07F2DE9FF4721F0004228
:10987000A94F04460D46BA424FEAD1762FD9A74FD9
:10988000BA4212D88EA3D3E90023FFF77DFCF0B9CA
:10989000204629468CA3D3E90023FFF757FC002874
:1098A00000F09C80002400250CE0C1F31303024665
:1098B000034305D00B46FEF74DFC04460D4601E080
:1098C000002EEFD12046294604B0BDE8F08780A3E2
:1098D000D3E9002310461946FEF7F2FDEDE7904B61
:1098E0009A4240F2A7808F4B9A4277D88E4BF40071
:1098F000C6F1010A03EBC603AAEB060AD3E900236B
:10990000FEF726FC894B804689462344D3E9003480
:10991000CDE90034DDE9002340464946FEF718FC56
:1099200004460D4622462B4620462946FEF7C8FD32
:1099300006460F4668A3D3E90023FEF7C1FD68A3DE
:10994000D3E90023FEF704FC32463B46FEF7B8FDA0
:1099500065A3D3E90023FEF7FDFB32463B46FEF745
:10996000AFFD63A3D3E90023FEF7F2FB32463B468B
:10997000FEF7A6FD60A3D3E90023FEF7EBFB32461A
:109980003B46FEF79DFD02460B4620462946FEF764
:10999000DFFB02460B4606460F4620462946FEF7E9
:1099A0008FFDCDE90201BAF1000F5AD100224FF02C
:1099B000804330463946FEF7CBFB02460B46DDE9D5
:1099C0000201FEF7A7FE22462B46FEF7C1FB024628
:1099D0000B4600205649FEF7BBFB6EE7554B204671
:1099E000294603EBC60646A3D3E90023FEF768FD2C
:1099F000D6E90023FEF7AEFBFFF7E6FB8246FEF753
:109A0000F5FC06460F4640A3D3E90023FEF758FDB8
:109A100002460B4620462946FEF79AFB80468946B9
:109A2000304639463AA3D3E90023FEF749FDCDE994
:109A300000016FE7404B9A420ED825A3D3E90023DB
:109A4000FEF788FB00223A4BFFF79EFB38B100225D
:109A5000374B204629462EE74FF0000A62E7824640
:109A600060E732463B4600204FF08041FEF770FB36
:109A700002460B46DDE90201FEF74CFE02460B46AC
:109A8000DDE90001FEF764FB42464B46FEF760FB52
:109A900002460B4600202649FEF75AFB6FF47F7200
:109AA000924502DB01EB0A5107E70AF57A7A0022B8
:109AB0004FF0B87301EB0A510EE700BFAFF300801F
:109AC000EF39FAFE422E864051302DD5104987C01D
:109AD0009C7500883CE4377ED0A4BE726937663E30
:109AE000F16BD2C541BDBB3E2CDE25AF6A56113F9E
:109AF00093BDBE166CC1663F3E5555555555C53F85
:109B0000FE822B654715F73F0000E0FE422EE63F40
:109B1000763C7935EF39EA3D412E8640FFFFEF7FF5
:109B2000422ED63FB1A2F03FE8EB0200D8EB020094
:109B30000000F03FF8EB0200FFFF2F3E00000000A6
:109B4000B1F5801F02460B462DE9F04F0D4687B058
:109B500024DA21F00044044308D10022002300202D
:109B6000C949FEF7D7FD07B0BDE8F08F002904DA38
:109B7000FEF7EEFA00220023F3E70022C34BFEF7C4
:109B80009FFC0B460D4602466FF03501C0488542EA
:109B900006DD10461946FEF7DDFAE4E70021F5E799
:109BA0002C15C5F3130510460022A4F2FF340C4413
:109BB00005F5152101F6647101F4801686F07F51D8
:109BC00004EB165481F4401141EA05031946B14BE8
:109BD000FEF7BEFAAB1C82468B46C3F3130300228A
:109BE000022B53DC0023FFF7A7FAD0B1002C00F0C2
:109BF00020812046FEF7FAFB06460F468EA3D3E9E6
:109C00000023FEF75DFC04460D46304639468CA322
:109C1000D3E90023FEF754FC02460B4620462946B2
:109C2000B9E789A3D3E9002350465946FEF748FC1B
:109C300002460B4600209849FEF78AFA06460F4670
:109C400052465B4650465946FEF73AFC02460B46E2
:109C500030463946FEF734FC06460F4614B9324604
:109C60003B46A0E02046FEF7C1FB8046894672A332
:109C7000D3E90023FEF724FC04460D46404649463E
:109C80006FA3D3E90023FEF71BFCA5E04FF0804350
:109C9000A5F5C226FEF75EFA02460B465046594627
:109CA000C5F5D725FEF736FDA6F27A465135CDE942
:109CB000000120463543FEF799FBDDE90023CDE99D
:109CC000020110461946FEF7FBFB02460B46CDE9A2
:109CD0000423FEF7F5FB804689465DA3D3E9002304
:109CE000FEF7EEFB5CA3D3E90023FEF733FA42460E
:109CF0004B46FEF7E5FB5AA3D3E90023FEF72AFA09
:109D000042464B46FEF7DCFB57A3D3E90023FEF7A0
:109D100021FADDE90423FEF7D3FB55A3D3E90023A1
:109D2000CDE9040140464946FEF7CAFB52A3D3E9F8
:109D30000023FEF70FFA42464B46FEF7C1FB50A345
:109D4000D3E90023FEF706FA42464B46FEF7B8FB7E
:109D500002460B46DDE90401FEF7FCF9002D8046C2
:109D6000894648DD00224C4B50465946FEF7A8FB79
:109D700052465B46FEF7A4FB02460B4606460F46DC
:109D800040464946FEF7E6F9DDE90023FEF798FB79
:109D90008046894664B902460B4630463946FEF78E
:109DA000D7F902460B4650465946FEF7D1F9DAE696
:109DB00021A3D3E90023DDE90201FEF781FB04467C
:109DC0000D461FA3D3E90023DDE90201FEF778FB6E
:109DD00042464B46FEF7BEF902460B463046394630
:109DE000FEF7B6F952465B46FEF7B2F902460B465D
:109DF00020462946D9E702460B4650465946FEF70B
:109E0000A7F9DDE90023FEF75BFB06460F46002CB1
:109E10003FF425AF08A3D3E90023DDE90201FEF7F3
:109E20004FFB04460D4606A3D3E90023DDE90201FA
:109E300029E70020002196E60000E0FE422EE63FE2
:109E4000763C7935EF39EA3D555555555555D53F51
:109E500044523EDF12F1C23FDE03CB966446C73F59
:109E6000599322942449D23F935555555555E53F72
:109E70009FC678D0099AC33FAF788E1DC571CC3F7D
:109E800004FA97999999D93F000050C300005043B4
:109E9000FFFFEF7F0000F03F0000E03FF8B502F168
:109EA000080323F0070300AFADEB030D054668463A
:109EB000144614F08EF900236E460DF804308AB073
:109EC0006A460849D661C2E9051507491162074982
:109ED00042F8101F4FF42351054802F0D5F8BD4653
:109EE000F8BD00BF50F502000002010304000002AB
:109EF00024EB02002DE9F04389B00B7806460C46AE
:109F000002AF092B00F2D680DFE813F00A00400010
:109F10004400C000D400D400D400C700D400CE0058
:109F2000CD6935B12B46644A012164480EF0BBFD72
:109F300028E00321624A61480FF001FD614B07F1FF
:109F40000C0493E80700604B84E807007C606C46D3
:109F50008AB0BB6002AA5D4B53615D4B93610523E0
:109F6000D3614FF4007313845A4B42F8103F4FF4FF
:109F7000135152482B4602F087F83046A546391D4A
:109F800010F0E2FC1C37BD46BDE8F083CB69524AB5
:109F90000321CAE74A69CB690321009247484F4A27
:109FA0000FF0E0FCD4F81480B8F1800F12D9DFF87C
:109FB000309149463046A8F1800210F072FD051E2E
:109FC00027D028DBA8EB0508B8F1800FF1D86FF097
:109FD000790901E04FF0000942463046404910F04F
:109FE00063FD0546B8B9237B012B06D1238B304690
:109FF000BB8107F10C0110F059FCB9F1000F16D02C
:10A0000063698022012100922C48364A0FF0AAFC95
:10A01000B8E76FF00405237B012B06D1238B304674
:10A02000BB8107F10C0110F041FC002D17DB6269C8
:10A030002B492D48FFF732FF05222C49284814F000
:10A04000F4F810B911F0F1FE9CE7062228492448E3
:10A0500014F0EBF8002895D111F0EAFE92E715F123
:10A060007A0FCDD02B460121224A14480EF01BFD59
:10A070000321214A11480FF062FC304610F03CFCED
:10A08000034600283FF47EAF1C4A4DE7CB690BB175
:10A090001B4A49E78B881B4A7AE7CB690BB11A4AFE
:10A0A00042E78B88194A73E7CB69002B3FF46AAF0C
:10A0B000174A39E7174A6BE755F5020024EB02000F
:10A0C0006DF5020080EB02000100D20483F502006E
:10A0D0009DF5020004000001A3F50200C0F5020096
:10A0E00076DD0020DEF502002DF6020038F60200D3
:10A0F0003EF6020045F6020065F6020082F6020016
:10A100009BF60200B1F60200C6F60200DCF6020081
:10A11000F1F6020009F702002DE9F0434FF00508BF
:10A1200089B0DFF8749000AF064614461D46C7E9B3
:10A1300005233974C7F80890C7F80C8004217818F3
:10A1400003F000F97B682A46BB83BB7F214623F0DE
:10A15000030312486C46BB77FFF7A0FE8AB06A463D
:10A160000F4BC2F81C80C2E905394FF40073138409
:10A170000C4B42F8103F00234FF413510A4801F0F2
:10A1800083FF07F10801A546304610F04BFB24374A
:10A19000BD46BDE8F08300BF27F702002DF702009F
:10A1A0003AF702000400000124EB02002DE9F04F11
:10A1B00001269DB002AF07F11408044610F0D9FA49
:10A1C00054220021404614F011F83B46424600213B
:10A1D000C7E9076645480FF0E2FC054688B103462B
:10A1E0003146434A43480EF05EFC434A31464148FB
:10A1F0000FF0A5FB6FF0090528466C37BD46BDE89A
:10A20000F08F4FF0080A3E68DFF8F09039482EB31F
:10A21000B369082B4AD1F36939495B6801204B6067
:10A2200045F6073308804B803E1D1023324604312B
:10A2300003F08CFAE94688B002AB324AC3E905263E
:10A240004FF400729A831A462F4B42F8103F0023B6
:10A250004FF4E651274801F017FFCD4638680FF05C
:10A26000A0FC274B17216363284B4046A364284A70
:10A270000AF0AAFA034668B30121264A1D480EF0E7
:10A2800012FC2548E062FFF735F9042284F85E20CD
:10A29000224A0023E26480222149C4E90E33C4E942
:10A2A00015122063226584F82430A5E7EB468AB0B6
:10A2B00002AAC2E90593182313620523C2F81CA061
:10A2C00042F8103F00234FF4215101F0DDFEDD463E
:10A2D00036689BE787F823000F231421114ACDF835
:10A2E00000800D480DF0A4FCCBE700BF4FF7020043
:10A2F0005DF7020024EB020074F70200B1F70200E0
:10A3000038DD00209BF7020003000001F59E0100EC
:10A31000D4F70200DCF7020062DD002076DE0020C8
:10A32000F6DD0020FDF702002123012110B5074AC8
:10A330000748FFF7F1FE034630B1BDE810400321A6
:10A34000044A05480EF0BFBB10BD00BF06F802006E
:10A3500070D3002028F8020024EB020098B50446D0
:10A360000321224A224800AF0EF0ABFB23781BB139
:10A37000032B20D0BD4698BD237A012B19D0052B85
:10A38000F8D11C4B6C4688B06A461B49C2E90513DC
:10A390004FF400739383194B42F8103F00234FF49E
:10A3A000E651134801F070FEA54615480CF03AFA44
:10A3B000E0E7144BE6E7217A134A144B6C4688B069
:10A3C000012908BF13466A461149C2E905134FF433
:10A3D00000739383094B42F8103F00234FF4E6517A
:10A3E000034801F051FEA546C4E700BF7FF8020014
:10A3F00024EB02005CF802008BF80200030000016D
:10A4000078C9002043F8020070F802007AF80200D0
:10A41000ABF802002DE9F047002582B0624C032121
:10A42000624A634802AF0EF04CFB2E46A146DFF8AD
:10A430008481DFF87CA194F8543053B1B4F85230E1
:10A44000B4F8562003210092504642460FF08AFA93
:10A45000013501360C2E04F10C04ECD12B460321FE
:10A46000554A53480EF02FFB0122E8214E480BF0CD
:10A470006BFB804640B103460121504A4C480EF028
:10A4800022FBBD46BDE8F08799F85030DB07F8D5D0
:10A4900011F0CBFCD9E9000100220023FDF75AFEA0
:10A4A0006D4688B002AC0426A246454BC4E90601BD
:10A4B00063614AF8106F4FF40351434652463C48DB
:10A4C00001F0E2FDD9E90201AD4600220023FDF7CB
:10A4D00041FE88B03B4BC4E90601636126614FF43D
:10A4E000035143465246324801F0CEFDAD460021AD
:10A4F000D9F81000FEF76CFA88B0334B6361FDF7B2
:10A5000087FF2661C4E906014FF4035143465246D2
:10A51000274801F0B9FDAD468AB099F8384099F85E
:10A52000390099F83A10B9F83C3002AA5362062370
:10A53000DFF898C0C2E90701C2E905C442F8103F3C
:10A54000234C43464FF44351194801F09DFD94F8C4
:10A550000080AD46B8F1000F93D113F028FC88B00D
:10A560000DF108094FF47A721A4BC9F81430A0FBA8
:10A57000020302FB0131C00B4FF47A72002340EA60
:10A580004140C90BFEF718FD4A46C9E9060142F8E9
:10A59000106F4FF403514346054801F075FD012348
:10A5A000AD4623706DE700BF30CA0020B8F8020046
:10A5B00024EB0200C5F80200D5F80200F6F802000C
:10A5C00019F902002FF9020045F902005DF90200B5
:10A5D000F6DE002081F90200072805D0092808D0FE
:10A5E000012808D1FFF716BF034A032103480EF0E4
:10A5F00068BA034AF9E770479EF9020024EB0200AB
:10A60000B0F90200F8B500AF6C4688B06A46724BEC
:10A610005361724B93614FF400739383704B42F814
:10A62000103F00234FF4E6516E4801F02DFDA54682
:10A6300005F068FF20B101216B4A6A480EF041FA2B
:10A6400003216A4A67480EF03CFA05F0B3F8034666
:10A6500060B1674A012163480EF035FA0121654A6D
:10A6600060480EF02EFA0020BD46F8BD0321624A74
:10A670005C480EF026FA614811F069FD034608B106
:10A680005F4AE7E74FF0FF324FF0FF335D480CF0D1
:10A69000EDF8544803215C4A0EF013FA5B480BF0C6
:10A6A000E3FBC8B15A4A01214E480EF00AFA594854
:10A6B00005F052FF20B10121574A4A480EF001FA35
:10A6C0005648FFF773FD0346002838D0544A01214D
:10A6D00044480EF0F8F9C6E70321524A41480EF00B
:10A6E000F0F90BF051FB044608B14F4ADBE711F0DB
:10A6F0009CFB00214FF480300CF09EFD204611F0B1
:10A7000097FBD4E701340AD03C230321474A35485C
:10A710000EF0D9F94FF4F01000210CF08DFD03215B
:10A72000434A30480EF0CDF93C4810F039F8034662
:10A7300040B1404A01212B480EF0C5F9E2E704463A
:10A740003D4DECE7294635480EF0AFF90346F8B920
:10A75000324E304610F06DF90246012128460FF0C6
:10A7600017FB002816DA0FF018FA344A03680121A3
:10A770001C480EF0A8F90321314A1A480EF0A1F93D
:10A78000264810F0B9F803460028BBD02D4AD1E77F
:10A790002D4A9CE7304610F027F9034620B110F10E
:10A7A0000B0F01D0294AE2E7EB88D90706D53046DE
:10A7B00010F056F9034608B1254AD8E7B5F9063036
:10A7C0001A0705D5234A012106480EF07AF9D2E787
:10A7D0009B06BED5204AF6E7CBF90200E7F9020056
:10A7E0000300000124EB0200FBF9020020FA020042
:10A7F0003BFA02000DFB02006DFA02005DA30100AE
:10A8000087FA020078C90020B0FA0200D9A5010039
:10A81000C9FA0200CB8A02002BFB020070D3002091
:10A8200054FB0200EAFA0200F8FA020079FB020087
:10A8300097FB0200BFFB020068D30020EFFB020081
:10A8400043FC02005DFC0200D9FB020003FC020095
:10A850001AFC020032FC02003AFC02002DE9F04F23
:10A8600091B0009302F004030293C2F3C2030133D8
:10A87000840705460E46DDF868900392059340F084
:10A88000BB81041D30B1072909D86FF01B0011B03E
:10A89000BDE8F08F01F00706341DC6F10806009BE5
:10A8A0004FF000084FF0040A591E4FF0FF3347469F
:10A8B0000193C3465346CDF810800DB1009A226033
:10A8C0000598002800F3E8809848009A824203D354
:10A8D00097488242C0F0E080039AA4EB050E9207ED
:10A8E0004FEA9E0000F103810F2F00F2B180002D8E
:10A8F00000F0058107F140020DEB020C019A0CF803
:10A90000200C0CF8102C049801300490E7E07A2811
:10A910005DD84B280ED8472859D829282DD8252866
:10A9200052D054D820287AD02338D0F1000B4BEBEA
:10A93000000B74E04C382E2849D8DFE800F070484E
:10A94000484848484848484848484B484848484884
:10A9500048484859484B4B595959704B6D487048B5
:10A96000184B184848827F4B48484B487F000020CE
:10A970004FF0000B4FF0040A38E001222A38C0B231
:10A9800002FA00F010EA0E0F49D110F0625C2FD1EC
:10A9900010EA020B43D06046013C5444B4FBFAF485
:10A9A0000AFB04F4002D61D0A3EB050CA444B445CC
:10A9B0003FF66BAF002868D1042B47D159F8043B10
:10A9C0002360042304342AE0019A013A01924FF0F3
:10A9D000000B24E011F8010C6C2834D1002011F890
:10A9E000023C83466C2BC5D14FF0080A5346D3E78F
:10A9F00009F1070929F00709073424F00704F9E8E9
:10AA000002AB35B106982044B0423FF63EAFC4E9F0
:10AA100000AB4FF0000B08344FF0080A534611F812
:10AA2000010F002878D0BBF1000F7FF470AF25280C
:10AA3000F5D14FF0010B019B013301934FF0040A54
:10AA4000ECE7584694E700208346A5E7082B02D0A0
:10AA50006FF015001BE709F1070929F00709F9E86C
:10AA60000223C4E9002308230834D8E768B9042B7B
:10AA700002D109F10409A4E7082BE9D109F107097A
:10AA800029F0070909F10809EDE7059A013A05924D
:10AA900059F8042B009210E7039A900720D54FF045
:10AAA000010CA4EB050E4FEA9E00BEF5007FCFD24D
:10AAB0000F2FCDD8F5B107F140020DEB020E019A30
:10AAC000C0B20EF8200C0EF8102CBCF1000F3FF4B1
:10AAD0001AAF60F07F000EF8200C08F10108013772
:10AAE000C5F108024FF6DA7E0434069297E74FF07C
:10AAF000000CDAE7BCF1000F01D00136EFE7029855
:10AB000002360028EBD10098CDE90631FEF7F2FCC1
:10AB1000DDE906310644E2E7631BB3F5806F97D2A7
:10AB200045B9A6F10804E018B1E600BFD8E6020076
:10AB30004C1F0300029A9B0828602B709DF8103070
:10AB4000C2B1EB7085F80280B8F1000F05D0002289
:10AB500008A8C5F1010C97420ED14FF0000AC5F1CB
:10AB600001030DF1200901930DF1300B574512D16E
:10AB7000601B8CE66B70E5E710F8013B190608D501
:10AB800004EB0C0EB64503F07F033FF67EAE04F8EF
:10AB9000013B0132DFE7B8F1000F03D099F9002043
:10ABA000002A17DB029BD3B11AF80B2004F8012B03
:10ABB0000022019B98182044B0423FF666AE99F8F7
:10ABC0000000009904F8010B2046039213F001FBEA
:10ABD000039A14440AF1010A09F10109C6E799F838
:10ABE000002055F822300093029B009845F822304F
:10ABF000FEF780FC421CDCE76FF00D0047E600BF6B
:10AC00002DE9F04F97B000AFD7F880B03B62CBF39F
:10AC1000C0030446894690F802A0FA62BB6141B9BC
:10AC2000457800780AEB800020444D4517D8A0EB0A
:10AC30000409E378FB61BAF1000F02D01BF0010FA9
:10AC400016D1FB6953BBFB6A1BB1494620463A6AE1
:10AC500098474D4628465C37BD46BDE8F08F461CF8
:10AC60003046FEF747FC0130304409F10109DCE7CA
:10AC7000626823787A62FA6A9900796104EB830149
:10AC8000002A40F001810E464FF000084D4601EBCE
:10AC90000A094E454CD101EB0A0610E01BF0020FE9
:10ACA000D1D023789A007A61626804EB83017A62DA
:10ACB000FA6A002A77D14D46904601EB0A061BF04E
:10ACC000050F0CBF02230123FB62FB6906EB430A5D
:10ACD0000BF00203BB625645BCD016F8021B16F8F7
:10ACE000013C54F82390AF4B994502D3AE4B9945A4
:10ACF00036D3BB69002B40D0786A0EF0CBF9002820
:10AD00003BD0E9468AB06A46A84B53617B6AC2E9E8
:10AD100006314FF400731384A54B42F8103F002313
:10AD20004FF41251A34801F0AFF9023DCD46D2E7EE
:10AD300016F8013BF96254F82300FEF7DBFBD7F865
:10AD40008430F96A01304BB1D7F8883098453EBF5E
:10AD5000D7F8843023F8180008F10108054498E773
:10AD6000BB6923B1786A0EF095F90028C9D11BF0B0
:10AD7000010F05D1FB6AED1AADE7BB6A002BAAD023
:10AD80004846FEF7B7FBD7F8843053B1D7F8883080
:10AD900098453FBFD7F88420431C22F8183008F1AB
:10ADA0000108054497E7BAF1000F73D01BF00406C1
:10ADB00073D0D046002607F1480052463B61B96285
:10ADC00013F007FAB96A3B6901EB0A02BA62FA6941
:10ADD000F9695200FA60BA6A02EB41023A610BF07B
:10ADE0000202BA603A69B96A8A4258D162781BF0A5
:10ADF000020F18BF00217A6208BF4FEA5801B2184B
:10AE00001BF0010FD2B240F09F801BF0040F14BF63
:10AE100040460020BB616270A070E17020463A6A33
:10AE20007969FB6A9847051EFFF614AFBB69414676
:10AE300023707B6A3A6A6370FB6984F802A0E3704E
:10AE400007F14800FB6A9847B0F10008C0F2B480EF
:10AE50007B69A9EB0A01C91AFB683A6AC91AD7E9E2
:10AE60000A0398470028C0F2A9804FF0000BA844BD
:10AE700008EB000507F1380AB34567D300213A6AA9
:10AE80000846FB6A9847E5E656464FF0000807F18A
:10AE9000380092E75646D04696E7B04694E7BA6A3D
:10AEA00012F8021B12F8015CBA6254F825003D4A00
:10AEB000904202D33C4A90421ED3BA6932B1786ABA
:10AEC0007B600EF0E7F87B6800288BD1BA6802BB84
:10AED00008F1280207F1300C08F10100944407F151
:10AEE000580208F1020852FA80F00CF8101C5FFAC0
:10AEF00088F800F8105C75E7BA693AB1786A7B6047
:10AF00000EF0C8F87B6800287FF46CAF1BF0010FCF
:10AF100009D006F1280207F13000711C161806F856
:10AF2000205CCEB25EE71BF0040F3FF45BAF08F18C
:10AF3000280207F1300008F1010102EB000808F8CF
:10AF4000105C5FFA81F84DE7002063E71BF80A30D8
:10AF500054F8239087F83730D7F88430FBB133F8B2
:10AF60001B8001213A6AFB6A07F1370098470028E5
:10AF700024DB0544B8F1000F06D14846FEF7BAFAC3
:10AF800000F101081FFA88F8414648463A6AFB6A10
:10AF90009847002812DB05440BF1010B6CE7D7F84A
:10AFA0008480DEE7D8E602004C1F03008BFC020021
:10AFB00004000001CCEA020045464BE6054649E69E
:10AFC000014B1860704700BF80C5002030B50025D8
:10AFD00087B0CDE903010446009503A9054805950E
:10AFE00000F010F9DDE904309842B8BF255407B0ED
:10AFF00030BD00BFE3900200032808B506D90EF06B
:10B00000CCFD092303604FF0FF3008BD2822044B1C
:10B0100002FB0033D3E8AF3F002BF0D00020F4E771
:10B02000E0D3002070B504460E461546FFF7E4FF56
:10B0300000280DDB28236343064AD1184968316094
:10B0400015B10C3313442B6028235C43105970BD99
:10B050000020FCE7D8D3002070B500254FF0FF3367
:10B060004FF0FF3217480BF0F7FA174BD3E8AF2F2A
:10B070007AB10135042D03F12803F7D10EF08DFDCF
:10B0800017234FF0FF3503600E480BF05DFB284699
:10B0900070BD28246C43D3E8EF0F0130C3E8E10F03
:10B0A0000029F8D1094E331932515A6004F10C00CD
:10B0B000304412F013FC04F12000304412F00FFD74
:10B0C000E2E700BFD0C80020E0D30020D8D30020A2
:10B0D00010B40446104628225443084B1A1919513B
:10B0E000506040B1C26832B10C34234440F20512C2
:10B0F00010BC0EF02DB810BC704700BFD8D3002094
:10B100002823434330B50D4908330B44D3E8AF2F10
:10B1100092B1541ED3E8EF5F954204D1C3E8EC4FDF
:10B12000BCF1000FF6D1F1D1012A05D128235843F3
:10B1300000230A180B50536030BD00BFD8D3002045
:10B14000F0B5024601680A270020074E0B461C781E
:10B150000131355D6D0701D41360F0BD07FB00437D
:10B16000A3F13000F2E700BFD91D03002DE9F84F2D
:10B1700015469A46D378224A6F2B12F803B08046C0
:10B180000F460BF0030B29D024D8582B0CBF1026E8
:10B190000A26DDF828903246002340463946FDF75E
:10B1A0005BFF092AD4B21ED83034B045E4B277F13F
:10B1B000000709F8014D01D3D14511D82B789B0622
:10B1C00005D5082E15D1AB7843F00803AB7048467F
:10B1D000BDE8F88F03F0F703702BD7E70826D8E710
:10B1E00080460F46D7E7BBF1010F0CBF3734573409
:10B1F000DBE7102EEBD1AB7843F01003E6E700BF9E
:10B20000D91D03002DE9F04F8A4616461C4600253D
:10B2100097B00390307808B928464AE3731C252874
:10B22000049307D05146039B98470028C0F24183FE
:10B230000135F0E11822002110A812F0D7FF737831
:10B24000252B00F0A380002398469E469C46184676
:10B25000711C0F4611F8012B2B2A00F0C68000F25A
:10B26000BD80202A00F0C480232A00F0C4802BB1C6
:10B270009DF8483043F040038DF84830B8F1000F96
:10B2800005D09DF8483043F020038DF84830BEF1DA
:10B29000000F05D09DF8483043F010038DF848307A
:10B2A000BCF1000F05D09DF8483043F008038DF83D
:10B2B000483028B19DF8483043F004038DF84830F9
:10B2C0009DF8483003F04401442903D16FF38613FD
:10B2D0008DF848309DF848302A2A43F080030997BA
:10B2E0008DF8483040F08C809DF8493043F00103E0
:10B2F0008DF849307B1C1A782E2A0CBF01210021C1
:10B300009DF8492061F341028DF849200CD15A1C67
:10B3100009925A782A2A40F083809DF84920023306
:10B3200042F004028DF849201A786C2A00F0A480BB
:10B3300000F28680682A00F08C806A2A00F0A580DE
:10B340004C2A00F0AA801A4612F8013B782B04928E
:10B350008DF84B309DF8492000F217816D2B00F2DB
:10B36000A980692B00F21181572B00F2BE80412B7E
:10B3700003D0453B022B00F2088104229DF84A309D
:10B3800062F302038DF84A300123CAE0B21C049232
:10B390008DF84B309DF84930D90740F1FD8054F8C5
:10B3A000048BB8F1000F07DA9DF84820C8F10008B7
:10B3B00042F004028DF848205A0740F1F68054F814
:10B3C00004BBBBF1000F80F2F5809DF849306FF3AC
:10B3D00041038DF849304FF0FF3BEBE02D2A0DD0B3
:10B3E000302A7FF444AF012333E74FF0010C30E7FC
:10B3F0004FF0010E2DE74FF001082AE7012028E762
:10B4000009A8FFF79DFE099BBB423FF474AF9DF86E
:10B4100048201390C00F60F341028DF848206AE77E
:10B4200009A8FFF78DFE9DF848301490C3F3400241
:10B4300042EAD07262F341038DF84830099B73E70A
:10B44000742A26D07A2A7FF47EAF06219DF84920FF
:10B450000CE05A78682A9DF8492006D1012161F351
:10B46000C6028DF8492002336DE7022161F3C6025E
:10B470008DF84920013366E75A786C2A9DF84920F7
:10B4800001D10421EBE70321F0E705219DF84920D4
:10B49000ECE707219DF84920E8E7BDF8482022F4B1
:10B4A000F04222F0020242F4804242F00202ADF881
:10B4B0004820DFE76E3BD9B201238B4040F2824146
:10B4C0000B4238D113F0240F52D1DF075DD5032191
:10B4D0009DF84A3061F302038DF84A3002F0780398
:10B4E000A3F14000434243411BE00120A3F1580176
:10B4F000C9B200FA01F111F4624F7FF43EAF40F699
:10B50000010739421DD111F4043F3ED09DF84A3065
:10B5100060F3020302F07802402A8DF84A3034D0FA
:10B5200000239DF84820C2F340010B4363F341021E
:10B530008DF848202EE702219DF84A3061F302037E
:10B54000E8E702209DF84A1002F0780260F3020159
:10B55000402A8DF84A1002BF9DF8481041F00101C1
:10B560008DF84810632BDBD1131E18BF0123D8E7D9
:10B5700003219DF84A3012F0780F61F302038DF831
:10B580004A3014BF01230023CBE79DF8483043F035
:10B5900001038DF84830C3E79DF94820002AACBF6D
:10B5A0004FF0FF38DDF84C8006E79F077FF513AFBB
:10B5B000DDF850B00023CDE913339DF84A309DF8F3
:10B5C000491003F00703012BC1F3C30133D1CB1E94
:10B5D000042B04D8DFE803F021464621210023682C
:10B5E00001294FEAE372CDE910321CD19DF94030B8
:10B5F000DA17CDE9103204349DF8483013F0030710
:10B6000050D032465146049B03980DF0B0FD0028FF
:10B61000C0F24F810544049EFCE554F8043BDA1760
:10B62000CDE91032E8E70229E5D11AB243F3C0337D
:10B63000CDE91023DFE7022B24D1CB1E042B04D845
:10B64000DFE803F018101018180001294FF000026D
:10B6500054F8043B14D00229CDE91032CCD19BB26E
:10B660001093C9E7073424F00704F4E80223CDE976
:10B670001023C1E754F8043B109300231193BBE758
:10B68000DBB2CDE7042B08D1073424F00704D4E95A
:10B6900000230834CDE91023AEE7032BACD154F8D6
:10B6A000043BDDE79DF84B007828B4D862281DD80C
:10B6B00025283FF4B7AD5828ADD1DDE910010DF1D3
:10B6C0003E03009312AA0AABFFF750FDBBF1000F37
:10B6D000814680F29880B9F1000F9CD00DF13E06B2
:10B6E000A6EB0903002F50D001334EE06338152834
:10B6F00091D801A252F820F079B70100DDB701001E
:10B7000017B6010017B6010017B6010017B6010001
:10B71000DDB7010017B6010017B6010017B601002A
:10B7200017B6010067B8010001B8010029B801008F
:10B7300017B6010017B6010051B7010017B6010096
:10B7400001B8010017B6010017B6010001B80100E9
:10B75000BBF1000FDDF840900ADB5946484612F075
:10B7600089FDB9F1000F3FF456AF09EB000676E012
:10B770004846FDF7BFFEF8E7109B00278DF82830FC
:10B7800001230DF129060DF128099DF84A1011F049
:10B790001002069200F081800233139A134405923E
:10B7A0004A0644BF14995B18B8F1000F40F38E802D
:10B7B000A8EB03089DF848305807C3F3800B00F14D
:10B7C0008580590678D53FB151463846039B984746
:10B7D00000286EDB5F46013530236EE01E075ABF3E
:10B7E000C3F300135F012B27DDE91023002BBFF605
:10B7F00064AF524263EB43032D27CDE910235CE78E
:10B8000000275AE700279DF848100DF13E03A3EBEF
:10B8100009036FF386119B458DF848107FF65BAFE7
:10B82000ABEB0303139356E7109880B30DF13E067C
:10B830000AAB0021009612AAFFF798FCBDF84A3027
:10B84000BBF1000F03F0EF0343F4F04343F01003A8
:10B850008146ADF84A30D5DA00283FF4DCAE002747
:10B86000A6EB090391E7109B07293FF6D4AEDFE86A
:10B8700001F00C04060C08080C0C1D70CBE61D80B2
:10B88000C9E6EA17C3E90052C5E61D60C3E6314EBA
:10B8900007460523A6F1050977E7080748BF0133E6
:10B8A0007BE7184607935146039B98470028079B60
:10B8B00004DA17B0BDE8F08F2023C34659460029AB
:10B8C0000BF1FF3BEDDC4544D8466D1A37B15146CC
:10B8D0003846039B98470028EBDB01359DF84A303A
:10B8E000DA0601D41B0706D551463020039B984742
:10B8F0000028DEDB0135069B3BB151469DF84B002D
:10B90000039B98470028D4DB0135059F2F4406E0B0
:10B9100051463020039B98470028CADB01357B1B2A
:10B92000002BF5DC33464A46514603980DF01FFCC8
:10B930000028BEDB0544A844A8EB0503002B7FF7D5
:10B940006AAE51462020039B98470028B1DB0135A1
:10B95000F2E700BF44FD02002DE9F047058B0446E5
:10B960002807904611D4022905F0070540F0CC8045
:10B9700020460DF067FE78B10138218B042811D8DC
:10B98000DFE800F0C2106D85950001290CBF45F07D
:10B99000100545F02005258388F31188BFF36F8FCC
:10B9A000BDE8F08701F0070AAA4500F0A58000274E
:10B9B000B9463E46A368002B00F0BC8041F0080168
:10B9C000218388F31188BFF36F8FA168002900F0ED
:10B9D000BA800D68002900F0B680334652462046F2
:10B9E000D1F80480C047002D76D02B6829461D462B
:10B9F000F0E701F007035A1F012A1BD8002221F0AB
:10BA00000701062B276889B2C4E9002209D13B4609
:10BA100003E0628B013262831B68002BF9D141F095
:10BA20000201204621830DF00DFE00287AD041F05E
:10BA3000200176E0042B0AD121F0070189B22046CB
:10BA400021830DF0FFFD10B141F020012183218BF6
:10BA500001F0070AAA454FD00027B946AAE7236993
:10BA600021F0070141F00601062DD3F80090218353
:10BA70002DD1B9F1000F3FD041F00801218388F3A7
:10BA80001188BFF36F8F20463949C84729E021F05C
:10BA90000701236941F0040189B2042DD3F8049011
:10BAA0002183E6D000274FF0040A3E4682E721F0CA
:10BAB0000701236941F0050189B2052DD3F80890EB
:10BAC0002183D6D000274FF0050A3E4672E70027B3
:10BAD0004FF0060A3E466DE72B4687E7B9F1000FA7
:10BAE000D1D1EFF31188202383F31288BFF36F8F36
:10BAF000238B23F008032383258BEA062ED525F01C
:10BB00001003238305F007056669218B002EBFF61D
:10BB100070AF00232768C4E9003321F0070141F02A
:10BB200001012183218B4FF0000901F0070AAA458A
:10BB30007FF440AF002F9CD041F00801218388F3AF
:10BB40001188BFF36F8F002FC8D03D683946334648
:10BB5000524620460DF0A2FD2F46F4E7AB067FF5D6
:10BB60001BAF25F02003238305F0070500E700BF86
:10BB7000C99602002DE9F047044607464FF0010937
:10BB8000DFF8508014B93846BDE8F08794FAA4F580
:10BB9000B5FA85F509FA05F32E0108EB05156FEAEC
:10BBA000030A24EA03042B7B002BEBD058F8063061
:10BBB0001B694BB94644736804222846196807EA92
:10BBC0000A0700F04DFADDE7284698470028D9D14A
:10BBD000F0E700BF64EB020030B5002289B00F49E6
:10BBE0000F4812F02BF9002200230024CDE9062390
:10BBF0000E230C4DCDE903344FF440722846CDE9B5
:10BC00000144094B094900940BF066F8084928469D
:10BC100011F06FFF204609B030BD00BF35BC0100F8
:10BC2000A8CF002018CB00200DBF010068E4002041
:10BC300045FD020001480AF0F5BD00BF60C90020C3
:10BC40002DE9F04780461F480F460DF0F6FD0646E9
:10BC5000002830D000252846BDE8F087237B6BB153
:10BC60002368DB680BB12046984723681B69D3B96A
:10BC7000636804222046196800F0F2F90136103496
:10BC80004C45EBD3B8F1000FE5D0002DE2D02846AB
:10BC9000FFF770FF0546002FF7D000214FF4A47086
:10BCA0000BF0CAFAF1E7204698470028E0D00AFADC
:10BCB00006F31D43E2E705464FF0010A024CDFF8A8
:10BCC0000C90DDE788D4002064EB020074EB0200E6
:10BCD000014B53F8200070471CEC020008B50346E6
:10BCE00008462BB1044A136000F05EFC002008BD3A
:10BCF0006FF01500FBE700BF84C5002010B5044CB1
:10BD0000237813B903480AF08DFD0123237010BD79
:10BD1000F7DE002060C9002010B5044606480DF08B
:10BD20008CFD3CB1054BD3E8EF1F0139C3E8E21F9E
:10BD3000002AF8D110BD00BF80D4002084D4002098
:10BD400000200146034BD3E8EF0FC3E8E21F002AAF
:10BD5000F9D1704780D4002070B5FFF7F1FF054698
:10BD6000074C084EB44200D370BD63685B792BB1B9
:10BD700023685B6813B12946204698471034F1E7E1
:10BD800064EB020074EB020010B5044C0449204639
:10BD90000DF000FB034B1C6010BD00BF3CC8002031
:10BDA00008EC020078D4002008B50023074A4FF4BD
:10BDB00000411370064A07481360074A1360FFF7F3
:10BDC0008DFFBDE80840FFF7DFBF00BFF8DE0020B1
:10BDD00080D400203798020084D40020014600223D
:10BDE000002301480DF0F7BA3CC8002001480DF0CF
:10BDF0008DBB00BF3CC80020024B014618680DF007
:10BE0000D9BB00BF78D4002001480DF00EBC00BFA4
:10BE10003CC8002070B5264B1878002847D0FFF7A3
:10BE2000E5FF054670B1234BD3E8EF1F0139C3E8A6
:10BE3000E21F002AF8D1204C204EB4422DD32846D0
:10BE4000FFF7DAFF1E4B1F4C1B68002B19DD11F0AA
:10BE5000AEFF4FF47A72A0FB020302FB0131C30B69
:10BE600043EA4143D4E900209B1A40F2E9324FEA09
:10BE7000D13161EB0001934271F1000101D3FFF771
:10BE80006BFFD4E9003213F57A7342F10002C4E982
:10BE90000032BDE87040FFF7B7BF63685B7923B13C
:10BEA0002368294620461B6898471034C5E770BDB3
:10BEB000F7DE002084D4002064EB020074EB020063
:10BEC00080D40020A0CF002070B50D4D297861B935
:10BED0000120FFF7B5FE0B4C0B4EB44206D3FFF723
:10BEE00099FF0028FBD101232B7070BD63685B793B
:10BEF0001BB1236820469B6898471034EDE700BFCC
:10BF0000F8DE002064EB020074EB020000212DE952
:10BF1000F0470846FFF794FE044648B340F26768CE
:10BF20004FF000090BF0A6F91A4B186030B11A4B0C
:10BF30001B68092B02DD19480AF074FC0025184F14
:10BF4000DFF858A044B12046FFF714FE044618B9A4
:10BF50004FF0FF384FF0FF39FFF75CFF064628B976
:10BF6000B5B942464B4650460AF080FC3546E9E7F3
:10BF70004FF0FF384FF0FF39D4E72B689B691BB1B6
:10BF800000222846114698471035BD42F5D3E8E710
:10BF9000044DFAE77CD4002084D4002060C900203E
:10BFA00074EB020064EB020013B518480DF045FC79
:10BFB000174B1B7873B1EFF31184202383F312889E
:10BFC000BFF36F8FFFF726FF84F31188BFF36F8FE6
:10BFD00002B010BD0F4B1B68002BF9D050B90022E6
:10BFE00000230D48CDE900234FF4004200230BF05D
:10BFF000A9FBEDE70928EBD1074811F02BFF074813
:10C0000002B0BDE810400AF00DBC00BF84D400208F
:10C01000F8DE00207CD40020A8CF002060C90020DA
:10C0200010B5064B04461B6898472146A06004489B
:10C030000DF04DFABDE81040FFF7B6BF84C50020F3
:10C040003CC80020044A054B9B1AB1EBD30F34BF08
:10C0500052F8310000207047C4EA020064EB02008D
:10C06000084B10B4C31A44681B1101332371436891
:10C070009A7101224368196043685A7110BCFFF736
:10C080003DBE00BF64EB02002DE9F04F8FB0C1F35D
:10C090004A2804AF0D469146B8607B600C0DB8F19C
:10C0A000000F63D000264FF0040B4FF00A0A07F18F
:10C0B0001403C7F80C80C7E907667E620193CDF8C8
:10C0C00008B0CDF800A007F11C0332464846F968D5
:10C0D000FEF796FDB0F5006F03461CD36C468AB0A0
:10C0E000D9F8041004AB26481A46C3E9050140F20A
:10C0F000FF71D9614FF400711984224B42F8103F4F
:10C100004FF4125133462048FFF7BEFFA5462C37A7
:10C11000BD46BDE8F08FC0F30A0804F117001844CB
:10C1200020F0070080083B60FFF758FE68F35325B6
:10C13000044690B13B6800F11001C7E9083607F1E9
:10C140001403F961CDE900A3CDF808B048460F4AC1
:10C15000F96807F11C03FEF753FD68F353252A46DF
:10C1600020467B68B9680DF09AFBD0E704F1170010
:10C1700020F007008008FFF731FE0446EDE700BF1E
:10C180005AFD020004000001FCEA0200739802005C
:10C190002DE9F04F87B00446DDE9105ADDE9126958
:10C1A0000F4693469846A6B31021334652460020C8
:10C1B000CDF80090CDF81490FEF750FB014605F144
:10C1C00017000844144B04F007040BF0070BE400BD
:10C1D00020F0070003EA412344EA8B1480081C4343
:10C1E0000391FFF7FBFD44EA0554054640B13EB11B
:10C1F000334652460399CDF800901030FEF72EFBDF
:10C20000434622463946284607B0BDE8F04F0DF0B8
:10C2100046BB3146D3E700BF00FE0F00406820B1A7
:10C22000034BC01A40F3CF0070474FF0FF30704708
:10C23000C4EA02000EB403B503AB53F8042B014665
:10C24000044801930DF0A8FB02B05DF804EB03B0C5
:10C25000704700BFC1990200CA0605D48B064CBFC7
:10C2600002490349FFF7E6BF704700BFB919030051
:10C27000B81903002DE9F04F89B09A46149B9DF838
:10C280004CB00693159B04460593169B0D469046AD
:10C29000179E0493BBF1000F00F09D8006F480739D
:10C2A00007930DF0E4FA06F00209024600283ED09A
:10C2B00020469249FFF7BEFF0746B9F1000F08D0AC
:10C2C00016F0440F35D12A4620468D49FFF7B2FFBC
:10C2D000074406F0010353B18A4B204653F82B2044
:10C2E000894B8A49002A08BF1A46FFF7A3FF06F4C4
:10C2F0008073002B49D006F00803002B63D1B8F1FE
:10C30000000F66D0424620468149FFF793FF05465D
:10C31000069B3D44002B6DD1049B002B73D1F3078A
:10C3200000F1E58031462046FFF796FFD9E0074649
:10C33000C3E7784B18680028CAD0774B4FF47A7956
:10C340001B684FF46161B5FBF3F5B5FBF0F300FB3F
:10C35000135509FB05F5B3FBF1F2B5FBF0FE4FF009
:10C360003C0C01FB123100FB1E55B1FBFCF309FB39
:10C3700005F5B5FBF0F50CFB131120460091CDE956
:10C3800001E56649FFF756FFA2E706F00803EBB1A7
:10C39000634B204653F82B206249FFF74BFF0546BD
:10C3A000B8F1000F05D0424620465949FFF742FF39
:10C3B0000544BAF1000FABD0524620465A49FFF768
:10C3C00039FF0544A4E74FF0000AE1E706F008054D
:10C3D000E6E745469CE7BAF1010F069B06D1002B24
:10C3E00065D1049B002B7CD000250CE0002BF8D0FD
:10C3F0004E485DE04E48069B22464E490CF019FE21
:10C40000049B002B69D0DFF83081DFF83091049F66
:10C410003146102F204628BF10274FF0000AFFF7A3
:10C420001BFF554546DC059B494620461A78FFF719
:10C4300001FF4FF0010A1AF0070F03D141462046D1
:10C44000FFF7F8FE57453CD9059B4946204613F8AF
:10C450000A20FFF7EFFE0AF1010ABAF1100FEAD144
:10C460004FF0000A20463649FFF7E4FE5246059B8E
:10C4700020469A5C334B995C11F0970F08BF2E222F
:10C480003149FFF7D7FE0AF1010ABAF1100F1DD0AA
:10C490001AF0070F03D141462046FFF7CBFE574560
:10C4A0005246E4D841462046FFF7C4FEEBE7204859
:10C4B0005D46A0E741462046FFF7BCFE0AF1010AAF
:10C4C000AFE720462149FFF7B5FEC4E7059B3B4493
:10C4D0000593049BDB1B049399D1BBF1000F7FF400
:10C4E0001EAF204609B0BDE8F04F0DF05CBA204603
:10C4F000054A0649FFF79EFE14E700BF9EFD0200B5
:10C50000A2FD02002CEC020099FD0200580B030072
:10C51000C7FD020090D400208CD40020ABFD0200A7
:10C5200040EC0200CBFD0200D1FD0200EF990200B9
:10C53000C199020099990200DEFD0200D6FD0200B9
:10C54000E0FD0200D91D0300B30E0300DCFD020074
:10C5500042F20F7373B58B4228BF0B460568044641
:10C56000052168460D4A0CF0DCFD06466368284646
:10C570000B225B680A490DF001FA6368324669468E
:10C5800028465B680DF0FAF963681B2228465B6851
:10C5900004490DF0F3F902B070BD00BF40F802008D
:10C5A000FEFD0200E2FD020000210123064A904246
:10C5B00006D8064A01B901231360054B186070477D
:10C5C000012140085B00F2E740420F008CD40020BC
:10C5D00090D40020F8B50D460446064F4618B442E4
:10C5E00001D12846F8BD14F8011BBB6801485B68FF
:10C5F0009847F4E7F8E70200014B0360002070471A
:10C6000088EC020008B504480CF07EFDBDE8084047
:10C6100002480CF079BD00BF44FE020079FE020022
:10C620002DE9F04706460C4600AF002936D0D1E987
:10C630000012E9468AB06D46A3684FF0050AA84685
:10C640001F48C5E90723C5E9050148F810AF0023D5
:10C6500042464FF421511B48FFF716FDD4E903125F
:10C66000CD466369AD461848C5E90723C5E905010C
:10C67000C5F810A0002342464FF421511148FFF79E
:10C6800003FDCD46E3690121104A0E480DF060F923
:10C69000A36901210E4A0B480DF05AF9012E07D16A
:10C6A000EFF305830B4A31460648103B0DF050F975
:10C6B0002146304609F022FEBD46BDE8F08700BFA6
:10C6C000A7FE020044EB0200D6FE020005FF0200B6
:10C6D00014FF020042FF020030BFFFF7FDBF00BFA2
:10C6E000074A936893F90E10002907DB52699342B9
:10C6F0001FBF044A536843F080535360704700BF24
:10C70000F4DC002000ED00E070B52A4C06460D4632
:10C7100029482A490DF0E1F9A36ADB0647D52648E6
:10C7200027490DF0DAF91120A36A1C0704D5224825
:10C7300024490DF0D2F912201E4CA36A990712D594
:10C7400021491D480DF0C9F9636BA26A120609D58B
:10C7500001211E4A18480DF0FBF81EB1A36A23F010
:10C760008003A3621320134CA36ADE0704D512488A
:10C7700017490DF0B2F91420A36A9C0604D50E489F
:10C7800014490DF0AAF915200A4B9A6AD10658BF30
:10C790009A6A9A6A920642BF5A6A22F400525A6210
:10C7A0009A6A42F0FF029A6200232B7070BD10203B
:10C7B000BAE700BF00ED00E044EB020055FF0200C5
:10C7C0006BFF02009EFF0200B1FF0200C9FF0200E2
:10C7D000DFFF0200FEFF020010B5244C244925486B
:10C7E0000DF07BF9A36A99013ED5224822490DF04C
:10C7F00074F91E20A36ADA0104D51E481F490DF002
:10C800006CF91F20194CA36ADB0204D519481C4996
:10C810000DF063F90220A36A1C0304D515481949D9
:10C820000DF05BF92120114CA36A590304D511487E
:10C8300015490DF052F92220A36A9A0304D50D4838
:10C8400012490DF04AF92320084CA36ADB0304D5F2
:10C8500008480F490DF041F92420A36A6FEA034309
:10C860006FEA1343A36210BD1D20C3E700ED00E093
:10C870002D00030044EB02004500030058000300B4
:10C88000720003009C000300BA000300DF000300F5
:10C89000F900030070B5294C06460D462848294981
:10C8A0000DF01BF9A36AD9043CD5254826490DF0A3
:10C8B00014F91720A36A1A0504D5214823490DF05D
:10C8C0000CF918201D4CA36A9B0512D51C48204961
:10C8D0000DF003F9A36BA26A100409D501211D4ACA
:10C8E00017480DF035F81EB1A36A23F40043A36284
:10C8F0001920124CA36A590504D5114816490DF0A8
:10C90000ECF81A20A36ADA050ED50D4813490DF08C
:10C91000E4F81B20094A936A43F47F43936200239F
:10C920002B7070BD1620C5E7A36A9B04F2D504489E
:10C930000B490DF0D2F81C20ECE700BF00ED00E041
:10C9400044EB0200240103003A0103009EFF0200B1
:10C950004B0103006401030079010300940103000B
:10C96000FEFF02002DE9F0478AB0694B0446D3F878
:10C9700004A089461646002500AFCAF3080885F3CF
:10C980001188BFF36F8F02F07F43B3F17F4F1ED149
:10C99000D3071CD4500603D4110708D4012508E09E
:10C9A0005C495D480DF099F816F0040600D04C463D
:10C9B00000250023FB71A8F10303092B00F28680F8
:10C9C000DFE803F0077C7F798484848484822C46AA
:10C9D000EFE7524950480DF080F800234C4EFB71B0
:10C9E000F36A9A0705D54E494B480DF076F80023B7
:10C9F00029E0F36A002B01DA4A49F5E7F36A5B00A4
:10CA0000F5D5494944480DF068F87369A26943F4C3
:10CA100080737361BFF34F8FBFF36F8F736932F809
:10CA2000022C23F480737361BFF34F8FBFF36F8FBA
:10CA30004DF602739A4228D1236801213B4A3648B9
:10CA40000CF086FF2368FA79DAB907F1080604F1D9
:10CA5000200C324620686168083403C264451646DB
:10CA6000F7D17A6A002D4ED0C2F3080121B96FEADE
:10CA700052226FEA42227A62184607F10801FFF754
:10CA8000CFFD2837BD46BDE8F087B36ADBB22BB1D6
:10CA90000120F91DFFF738FE0346D4E7B36A13F40B
:10CAA0007F4F04D00120F91DFFF7F4FEF4E7B36ACD
:10CAB000B3F5803F9BD3FFF78FFEEDE70020F91D14
:10CAC000E8E70020F91DEFE719498DE7194A6E469E
:10CAD0001AF4F87F8AB0184B18BF13466A461749F4
:10CAE000C2E90513A8F11003D3614FF40073138456
:10CAF000134B42F8103F00234FF411510648FFF743
:10CB0000C3FAB54673E722F4FF7222F00102B2E7DE
:10CB100000ED00E0DA01030044EB0200FD01030038
:10CB20001402030035020300430203006202030003
:10CB30007E020300C1010300AC010300A202030056
:10CB400004000001044B5A6942F010025A615A690C
:10CB500042F480625A61704700ED00E0EFF3088014
:10CB6000EFF3098101B57246FFF7FCFE01BD00BF7E
:10CB7000002080F31488BFF36F8F002080F30A88B1
:10CB800080F30B880FF079FB00200E490860BFF39B
:10CB90004F8F0D4880F3088800F02CF8202080F398
:10CBA00011880A484FF40061401880F30988EFF3B8
:10CBB00014800221084380F31488BFF36F8F00F0C4
:10CBC00009F9000094ED00E0A805012068EC0020C0
:10CBD000002318460649D1F89020C2F30722934259
:10CBE00000DB7047C1F89830C1F8A0000133F6E7C8
:10CBF00000ED00E010B572B6002484F31388FFF74F
:10CC0000E7FF23464FF0FF300C4A03F120010133C8
:10CC1000102B42F82100F8D100234FF0FF30074AD3
:10CC200003F160010133102B42F82100F8D162B604
:10CC3000BFF34F8FBFF36F8F10BD00BF00E100E067
:10CC4000084B9B6883420BD1EFF3058343B1064B3E
:10CC50005A6842F080525A605A6A22F400425A627C
:10CC600011F048B8F4DC002000ED00E06FF00A019C
:10CC7000084A9368D967084998674B6843F080531E
:10CC80004B60002383F31188BFF36F8F9368D86FD5
:10CC9000704700BFF4DC002000ED00E00E4A93680E
:10CCA00083F88100EFF31183202383F31288BFF30D
:10CCB0006F8F4FF00061536920F0FF009360074AC7
:10CCC0005160002193F8812010439A6F996782F395
:10CCD0001188BFF36F8F7047F4DC002000ED00E097
:10CCE00010498A6882F881E04FF030001044EFF379
:10CCF000098C80E8F01F74467046FFF7CFFFA64608
:10CD000008498A68864602F1300090E8F01F8CF3EB
:10CD1000098802F1000004B50CF0E9FEBDE804400A
:10CD200070470000F4DC00201EF0040F0CBFEFF38E
:10CD30000880EFF30980816911F8021C0229FFD0F5
:10CD400001B50CF0BFFE01BD40B2002807DB012396
:10CD50004109034A00F01F00834042F82130704728
:10CD600000E100E040B200280CDB01220649430943
:10CD700000F01F008240203341F82320BFF34F8F83
:10CD8000BFF36F8F704700BF00E100E0054B420921
:10CD900053F82220012300F01F0003FA00F0104096
:10CDA000704700BF00E100E040B2002801F101013E
:10CDB000ACBF00F16040064B4FEA4111C9B2ABBFB6
:10CDC00000F5614000F00F0080F80013195470471F
:10CDD00014ED00E00B4A08B50B4B22F07F029A607D
:10CDE000BFF34F8FBFF36F8FD3F8882022F4700208
:10CDF000C3F8882009F06CFB0AF0DAFA00F04AF870
:10CE000009F0A6FB0080010000ED00E042F8203CA4
:10CE1000009B0D4942F81C3C019B21F0010142F8A6
:10CE2000183C029B42F8081C42F8143C4FF08073F7
:10CE300042F8043C002383674FF43C43203A0265E8
:10CE4000C0F88030704700BF3D9102000B4B0E468A
:10CE500098601546836E83F30B882C4686F3098809
:10CE60004FF00000064B984720464FF000014FF06E
:10CE700000024FF00003034C204700BFF4DC002009
:10CE8000F79A02003D9102001022014B1A6170478F
:10CE900000ED00E0002320210348C2180133412B9C
:10CEA00082F80013F9D1704700E100E008B5EFF314
:10CEB0000583064A103B02EBC30152F83300496870
:10CEC0008847BDE80840FFF70BBC00BFACE8020094
:10CED0001FB5094C094A23460121094800F012F9FF
:10CEE00000230393074B0121E41A01A80193029444
:10CEF00000F012F904B010BD0000042080C500202D
:10CF000088EC020030CA002010B50C7A0B6804F0DF
:10CF10001F0223F01F031A43CB68640923F01F0389
:10CF2000054943EA440343F00103C1F89800C1F8FE
:10CF30009C20C1F8A03010BD00ED00E010B50A4BF8
:10CF4000D3F89030C3F30723013B984208D901215D
:10CF50000346064A06480CF0FBFC6FF0150010BDB6
:10CF6000FFF7D2FFFBE700BF00ED00E0B9020300CE
:10CF70001CEB02002DE9F04F8946144606464FF09F
:10CF80000008514D85B0C84527DAD6F804A0BAF19B
:10CF9000000F44D0BAF11F0F17D91AF01F0F14D188
:10CFA000D6F800B01BF01F0F0FD158460CF0C6FD8D
:10CFB00007460AEB0B0001380CF0C0FD874210D089
:10CFC0006FF01507414A3B4601E04346404A0121C4
:10CFD00040480CF0BDFC6FF01504204605B0BDE8DC
:10CFE000F08F17F1160FEDD0BC42EBDDC5F898704D
:10CFF000D5F89C10C5F89870D5F8A03021F01F0125
:10D0000043F01F0BD6E900321A44994202F1FF3A6D
:10D010001DD1D34507D13146F8B20CF098FD08F187
:10D0200001080C36AFE73146C5F89870D5F89C304A
:10D0300022F01F0203F01F031343C5F89C30E0B237
:10D040000CF085FD10F1160FC5D0441CE7E7C5F8BC
:10D050009870D5F8A020013B23F01F0302F01F02B7
:10D060001343D3453146E0B2C5F8A030E8D00CF008
:10D070006EFD10F1160FAED0C5F89870D5F89C2053
:10D080009DF808300BF1FF3B62F304038DF8083084
:10D09000D5F8A0309DF808205B0863F347128DF89F
:10D0A0000820D6E900321344009323F01F035B44A9
:10D0B000A3EB0A03013023F01F036946C0B20393B8
:10D0C000FFF73CFFBEE700BF00ED00E002030300F6
:10D0D000DF0203001CEB02000522044BC3F894207E
:10D0E000BFF34F8FBFF36F8F704700BF00ED00E0BD
:10D0F000BFF35F8F0022024BC3F89420704700BF3C
:10D1000000ED00E010B5034C2278FFF733FF2070EC
:10D1100010BD00BFFADE00202DE9F74F294D8A46E9
:10D1200006464FF00008AB46274FD0451BDAD6F82D
:10D130000490B9F1000F3FD03168084601910CF01E
:10D14000FDFC0199044609EB010001380CF0F6FCE6
:10D1500084424FF014021D4B08D002FB08F36FF01D
:10D1600015024BF8032003B0BDE8F08F14F1160F41
:10D170002C60F8D01978A142F5DD02FB08B0C7F8A1
:10D180009840C7F89840D7F89C4000F10801007B10
:10D1900064F304000871D7F8A0000C79400860F32C
:10D1A00047140C71D7F89C1021F01F016960D7F863
:10D1B000A01021F01F01296108F1010814350C3677
:10D1C000B3E700BFC0D4002000ED00E0FADE00208D
:10D1D000F0B54149414CD1F890302568C3F307239D
:10D1E0009D4287B075D80020FFF782FF3C4BC1F805
:10D1F000C030854216D13B4C01A82570FFF7FCF9E1
:10D2000000250646384FAE4213D10020237832491C
:10D21000D1F89020C2F30722934254DBFFF75CFF62
:10D2200000202FE0616801EB0011FFF76DFE013077
:10D23000DFE70199280101EB0513DA683A40B2F5FE
:10D24000001F21D0B2F5800F2BD0B2F5801F38D14E
:10D250005A689B680958013B22F01F0003440120D3
:10D26000844623F01F0340EA4C10CDE902218DF8DB
:10D27000100002A920780593FFF760FE00281DDA50
:10D280006FF0150007B0F0BD5A689B680958013B64
:10D2900022F01F0003444FF0020C012023F01F0373
:10D2A000E1E75A689B680958013B22F01F000344DC
:10D2B0004FF0000C062023F01F03D4E7237801333E
:10D2C000237001359FE7C1F89830C1F8A000013301
:10D2D0009EE74FF0FF30D5E700ED00E094EC020050
:10D2E000AAFF4400FADE00200000F0FF014B1860A6
:10D2F000704700BF90C5002010B5074C2368C218C6
:10D300000648C0F1005101F580218A4236BF2260F3
:10D310004FF0FF30C01810BDD4D4002028120120D7
:10D320000122024B0020C3F84025704700900340C3
:10D3300020B1034B800143F001031847704700BF41
:10D34000D0EB0200F7B506460D460D488AB2836859
:10D3500031461B689847002810DA00240CE02F1B88
:10D36000042F28BF04270EF0F9FA3A46019001A9CC
:10D37000301910F02EFF3C44A542F0D803B0F0BDA8
:10D38000E4E702002DE9F04105460E461746104C31
:10D39000DFF84080444507D30CF0FFFB6A230360AD
:10D3A0004FF0FF30BDE8F0812368AB4200D063B995
:10D3B0003A4631462846A368984730B13A46314646
:10D3C0002846E368BDE8F04118471034E2E700BFA3
:10D3D000B4EA0200C4EA02002DE9F04F4FF0000861
:10D3E00046469DB0CDE9060108A814461D4610F03A
:10D3F000E0FCDDE90823DDE9069BCDE904230DAB64
:10D400000A93CDF80C80BBF1000F22D1002E6ED014
:10D41000B5F1FF3F08BFB4F1FF3F17BF4FF47A7279
:10D420004FF0FF34A4FB024302FB05331CBFE40BA7
:10D4300044EA4344079B4FF4827200934146069BA3
:10D44000039801940CF0AFFB074638461DB0BDE8C9
:10D45000F08FD9F80000002829DB0CAA0BA9FDF7F2
:10D46000E1FD074618B34FF0FF324FF0FF330C9841
:10D470000CF0A8FB1CAB01930AAB00934FF4817234
:10D480004B4639460B980CF08EFB10F1780F824614
:10D4900012D10022002308A810F08BFCDDE908342B
:10D4A000CDE9043400240C980CF08EFB254609F1DC
:10D4B00008090BF1FF3BA6E71AF1120F0C980BD1EC
:10D4C000039B1BB10CF080FB0126F0E70B9BB846D9
:10D4D00003930CF079FBF7E70CF076FBBAF1000F41
:10D4E000E5DA0CF05AFBCAF10003036021E0DDE944
:10D4F000042308A810F081FCDDE9084522462B46EC
:10D50000DFF8C8800A990DAC091B891008FB01F1EE
:10D5100020460AF051F900F10B030B2B054604D805
:10D520002B4F1F4117F0010706D00CF036FB6D4260
:10D5300005604FF0FF3788E7B9460A94DDE90645F4
:10D540008DB9B9F1000F80D0002F7FF47EAFDDE9F7
:10D55000042308A810F051FCDDE908452B462543BB
:10D560002246CFD171E72068E680002827DB0CAA8D
:10D570000BA9FDF757FD824618B92023E380013738
:10D580001DE04FF0FF324FF0FF330C980CF01AFB08
:10D590000AAB514640F2031200930B9823460CF05D
:10D5A00002FB82460C980CF00FFB1AF10B0F09D00E
:10D5B000BAF1000F95D1B4F90630002BDFD1083451
:10D5C000013DBDE74FF00109F9E700BFCDCCCCCC60
:10D5D0007EF7FFFF014B1860704700BFD8D40020D2
:10D5E00010B4034C24682468A44610BC604700BFF4
:10D5F000D8D40020014B1B685B681847D8D40020A2
:10D600002DE9F0410D460646E8B1E1B10846FBF7C9
:10D6100071FF08281AD8104FDFF84080441C474596
:10D6200007D322462946301D10F0D3FD0020BDE867
:10D63000F081B74205D022462946381D10F0B9FDC9
:10D6400038B13C37EBE76FF01500F0E76FF05A00A8
:10D65000EDE76FF07700EAE7C0C90020FCC90020C1
:10D66000F0B54FF0FF324FF0FF33274885B00CF094
:10D67000E1FB0025254C264EB44205D3224805B0D7
:10D68000BDE8F0400CF0F4BBC4E9015523682573F4
:10D690001B689F6897B13B6883B104F1100010F0DC
:10D6A0001DF904F1240010F019F93B682046984751
:10D6B00094F8383023F0030384F83830237903BB1F
:10D6C0002046CDE901338DF80C300CF04CFC40B114
:10D6D000104A01A81368591C116008210E4A0BF06A
:10D6E00020FD9DF8043043B90C4A01A81368591C69
:10D6F000116008210A4A0BF014FD204601A9FFF72A
:10D700007FFF3C34B8E700BF0CC90020C0C900202F
:10D71000FCC90020E0D400204F030300DCD400202B
:10D720005603030038B5074C074DAC4200D338BD53
:10D73000032120460CF087FB10B920460CF0E1FBDA
:10D740003C34F2E7C0C90020FCC900202DE9F04FAD
:10D75000002489B0022883460E46CDE90644029291
:10D760005FD10B6804913BB94A6852B94FF6FF7319
:10D770004C89E11A4C424C4106A80146002213464E
:10D7800008E01C46F8E70D78013301350D70DDB275
:10D79000082D03D036F81350002DF4D00132082A9A
:10D7A00001F10101EBD14FF0FF374FF0010A0023E7
:10D7B00010F8012B524588BF5FB203F10103DBB2C1
:10D7C00088BF9246082BF3D199463A220023BAF13A
:10D7D000010F08BF4FF0FF37CDE900230022029868
:10D7E00000252B46B9F1040F5ED10199C95C0346AF
:10D7F00041BB302103F8021B0099417018460135E6
:10D80000EDB24D452B46EDDB029B98420BD0BBF1B0
:10D81000010F4FF0000340F09C8000F8013C02989B
:10D8200002E0012803D0002009B0BDE8F08F2E23CC
:10D830004FF004094FF0FF378246264601910093CE
:10D840000494CBE74FF0000C4FF00908CDF814C05A
:10D85000DFF804C1B1FBFCFE03910CFB1E11DDF8E7
:10D8600014E0C64503DCDDF80CE0E64509D3DDF83D
:10D870000CE0CDF81480BEFBFCFE0EF1300E03F878
:10D8800001EB4FF00A0E08F1FF38B8F1FF3FBCFB87
:10D89000FEFCDFD14FF0000119701B1A50FA83F023
:10D8A000009B00F8013BAAE774B1052D0CD906F1E5
:10D8B0000C0301933A2300F8013B2E234FF0040997
:10D8C0004FF0010B00938BE79F420DD102B915B9C0
:10D8D0003A2300F8013B3A2300F8013B0AF1FF33F9
:10D8E0002B440022DDB28AE712B13A2300F8013B53
:10D8F000049B33F8152052BA12F47F4FC2F307236A
:10D900005FFA82F816D00F2BD9B20AD90023612210
:10D910000CF036FB0123612241460CF031FB012261
:10D920006DE7092B04D83031C9B200F8011BF1E7CB
:10D930005731F9E7B8F10F0FEDD8B8F1090F94BFDF
:10D9400008F1300808F157085FFA88F800F8018BF1
:10D95000E5E7037063E700BF00CA9A3B2DE9F04793
:10D960000F6890F860503C4B3C4A064690F85E00C9
:10D970000537042814BF104618460F600C460CF0FB
:10D98000E2FBC5F34005034638B9D4E900209042D4
:10D9900096F85E1004D16FF00B031846BDE8F087CF
:10D9A000501C20601170D4E900829045F3D008F13A
:10D9B0000102226088F800302146B6F85C000CF0C5
:10D9C000B0FB03460028E8D106F12C000CF0BBFBAD
:10D9D00003460028E1D1306C6D00E8B1214696F88D
:10D9E00060A090F808900CF0AEFB0AF0010A034624
:10D9F0000028D2D1736C21465BB318460CF0A3FB10
:10DA000003460028C9D145F004054FEAC90345EA99
:10DA10004A1503F018031D43B06B38B121460CF0D2
:10DA200092FB03460028B8D145F08005F06B38B171
:10DA300021460CF088FB03460028AED145F0400596
:10DA400088F8005022463946BDE8F04710200CF017
:10DA500095BB0CF066FBD3E7BCEC0200C4EC020003
:10DA6000D0E900239B1A012B81BF054B1B88138033
:10DA7000036883BF0233436000206FF00B007047E0
:10DA80005C030300D0E900239B1A012B81BF054BE7
:10DA90001B881380036883BF0233436000206FF04C
:10DAA0000B0070475E030300142290F824305343A8
:10DAB000014AD358184700BFCCEC020030B41425FB
:10DAC00090F82440024B05FB043330BC5B681847D8
:10DAD000CCEC020010B4142490F82420024B04FB78
:10DAE000023310BC9B681847CCEC020070B41426BB
:10DAF00090F82450034C06FB0544E468A44670BC2F
:10DB0000604700BFCCEC0200084B70B5C31A0D464D
:10DB100007499B1004465943402206480CF0E2FF97
:10DB20002B4601462046BDE870401847F8D4002037
:10DB3000B76DDBB6BCE70200402373B50B4C009316
:10DB4000041B0B460D460A49A41061430646094AC8
:10DB500009480CF0F2FF011E05DA30462B4602B0F0
:10DB6000BDE87040184702B070BD00BFF8D4002077
:10DB7000B76DDBB6A3AB0200BCE7020010B5EFF354
:10DB80001184202383F31288BFF36F8F074A136831
:10DB900023F00201DB07116002D401200EF078FBB4
:10DBA00084F31188BFF36F8F10BD00BF48D50020EC
:10DBB00070B50022012104460520FFF7F5F80F4853
:10DBC00005F0F0F80E4B984215D105F0FBF82669E8
:10DBD0000C4930460BF085FD00280BDB0125356430
:10DBE0002469084904F11C000BF07BFD002801DBCF
:10DBF0000020E56470BD6FF00400FBE70DDD01005F
:10DC00000000AD0BE0EC02007FB500220123CDE95E
:10DC1000022304ABCDE90433094A6B46CDF800D0AA
:10DC2000CDF804D00CF0B6FF002805DB4FF480429D
:10DC30000023684608F01AFE07B05DF804FB00BF39
:10DC4000C1AB02000C22104B014602FB0033002046
:10DC500030B4D3E90E529863EFF31180202484F39B
:10DC60001288BFF36F8F1C6C04F0C00444F00204F0
:10DC70001C6480F31188BFF36F8F1DB12B4630BC3D
:10DC80000248184730BC7047F8D40020BCE70200B7
:10DC900010B4EFF31182202383F31288BFF36F8F48
:10DCA0001748016841F002040460C80707D482F3F2
:10DCB0001188BFF36F8F012010BC05F097B8114990
:10DCC000D1F80C04D1F80C14C907F0D5EFF311808A
:10DCD00083F31288BFF36F8F0B490B6C03F0C00303
:10DCE00043F002030B6480F31188BFF36F8F82F35C
:10DCF0001188BFF36F8F002010BCFFF7A3BF00BFD8
:10DD000048D5002000500040F8D4002010B1012870
:10DD100004D07047034B1B6C5B0701D1FFF792BF28
:10DD2000704700BFF8D400202DE9F04101220746DA
:10DD30003449D1E8EF3FC1E8E02F0028F9D133B9E9
:10DD4000314932484B60CB608A600BF0DDFC7B1EB2
:10DD5000012B28D8012F06D12D4BD3F81C3403F00A
:10DD60000303022B1FD00FF0BEFE0546E8B9294B76
:10DD70001B78D3B102220646254BC3F80823244C56
:10DD8000DFF89480D4F81824D4F81834D20315D5C9
:10DD900003F00303022B01D0012F0FD16DB386F3E3
:10DDA0001188BFF36F8FBDE8F081EFF31186202358
:10DDB00083F31288BFF36F8F0125E0E7C5B13046CA
:10DDC0000BF0ADFED4F81835DBB2012BDAD1D4F864
:10DDD0000421002AD6D00022C4F80421D4F804215A
:10DDE0000222C4F818252022C8F88021A360C9E7C0
:10DDF0000021212009F020FAE4E70222044BC3F8B5
:10DE00000423D0E7F4D40020E4D4002014D500206B
:10DE10000050004064E4002000E100E008B507483D
:10DE20000FF0ABFC38B10648FFF760FA0448FDF785
:10DE3000C7F8002008BD6FF01200FBE7F8E702000A
:10DE400045DE01000A2838B50446074D04D1AB6809
:10DE50000D2128465B689847AB6803485B68E1B2D0
:10DE60009847204638BD00BFF8E7020038B545683E
:10DE70002B69B3B11035284605F0ECFB044680B998
:10DE80000146284605F0AAFB084B98420BD12246D2
:10DE90002846074905F078FB224605213120FEF788
:10DEA00083FF002038BD6FF00400FBE70000AD0BDE
:10DEB000B5DE0100430970B507D10B4B596821B19C
:10DEC00001250C68094E854001B970BD8A682A4059
:10DED00002D030464B6898471CB1236821461C4647
:10DEE000F2E72346FAE700BF4CD50020D0E7020056
:10DEF0002DE9F04340F206354668D00648BF0320BE
:10DF0000337B02EA050558BFC2F3401087B001F029
:10DF10001F07B5F5837F144647EA43178DF80300C2
:10DF200041D00FD8062D18D007D8B5B1022D3CD05E
:10DF30006FF0150007B0BDE8F083B5F5807FF7D12D
:10DF400001250AE040F20222954230D0B5F5407F2B
:10DF50002FD0B5F5007FEBD1022522032BD501236D
:10DF600072688B409360326962BB07F01F037F09C0
:10DF700075D13D4A84F4803102EB8302D2F800323D
:10DF8000C1F30041C4F3404423F4E16344EA410493
:10DF900023F007031C4344EA800444EA0524C2F842
:10DFA00000420020C6E70725D7E70425D5E7052569
:10DFB000D3E70325D1E7630341BF012372688B4098
:10DFC000D360D0E71036394630460DF1020205F035
:10DFD000E9FA14F4403F80460CD1394630460EF041
:10DFE000F5F9224B9845DCD130469DF8021005F03A
:10DFF0003FFBD6E74FF0000901AB3946304603AA94
:10E00000CDE90439CDE90199CDF80C9005F028F956
:10E01000164B98428CD114F4003315D09DF8033080
:10E0200084F48034C4F300448DF80E3039464B46F6
:10E03000304603AA8DF80C508DF80D4005F00CFA0F
:10E040000A4B9842CDD073E7CDE9043339460DF140
:10E050000303304603AA039305F002F9F0E7803387
:10E0600052F82330FFDE00BF002584400000AD0BD6
:10E07000F0B5406801F01F04057B87B044EA451401
:10E080000569002D5FD0B2F5001F00F1100506D123
:10E09000214628460EF09CF9002007B0F0BD00276D
:10E0A000B2F5800F01AE0197776037D1B3F1007FF1
:10E0B00014BF052304238DF804300023CDE9046345
:10E0C0000393836823FA01F111F0010118D1B2F131
:10E0D000A07F15D104F01F03620903F1800338D13A
:10E0E0001D4A52F82330DB070AD40DF103063246ED
:10E0F0002146284605F056FA184B984219D0029648
:10E100002146284603AA05F0ABF8154B98421DD1CD
:10E1100001222146284605F0C3FABDE7B3F1C06FDE
:10E1200005D0B3F1007F14BF01230223C3E703230B
:10E13000C1E73146284605F0A7FA094B9842DED0E0
:10E140006FF00B00A9E76FF08500A6E76FF01500F0
:10E15000A3E751F82330FFDE002584400400AD0B17
:10E160000000AD0B08B5CA0743680AD4C1F34201E9
:10E17000012909D002290ED00121094A09480BF0D2
:10E18000DEFB6FF0150005E04FF0CC721B6800203D
:10E19000C3F8242508BD4FF0C8621B68F7E700BF2D
:10E1A000A9030300ECEA0200F8B5446800AFE36994
:10E1B000054606699847206A0CF069FD00281FDBB8
:10E1C00033462046124A04F1080105F0AFFB114B1B
:10E1D000984217D06C4688B02B686A460E49C2E94F
:10E1E00005134FF4007393830C4B42F8103F0C4817
:10E1F00000234FF4E251FDF747FF6FF00400A546FE
:10E20000BD46F8BD204605F0CBFB0020F8E700BF77
:10E2100061E201000000AD0BBB030300030000013D
:10E22000ECEA020070B5446823682046D3F808552C
:10E23000D3F80C6505F0C4FB3146284605F056FEC0
:10E240000546206A0CF023FD204605F0A9FB034B90
:10E250009D4214BF6FF00F00002070BD0000AD0B99
:10E260000378012B08D0022B08D04BB9054B0B6368
:10E2700001F1180008F0D6BA034BF8E7034BF6E7B4
:10E28000034BF4E70000AD0B0100AE0B0200AE0B38
:10E290000100AD0B2DE9F04F8DB002AFBA60142232
:10E2A0001D46D0F804B0D0F81080BBF818300646F0
:10E2B0000C46B8180021D8F834A0FB600FF096FF88
:10E2C0007D754FF0FF324FF0FF33404608F0CEFA35
:10E2D00008F118037B604FF000090022002308F1C9
:10E2E000180008F0C3FA4D46BB68994501D30024D5
:10E2F0003FE0207A020700F1AA80BB6809F101091A
:10E30000994521680AD2830708D4237D80EA030255
:10E3100002F0010203F004031A4307D025B901F00B
:10E320006043B3F1005F36D0002300E00123626850
:10E33000D7F80CE005EB020CF4451ED96C468CB006
:10E34000316802ABDA61FA684248C3E9082140F259
:10E3500003521A851A46C3E905053F4B42F8103FA0
:10E3600000234FF451513D48FDF78EFEA5466FF056
:10E370001B04404608F056FA22E0C00705D40AEB19
:10E3800005003B600FF025FF3B6862682A4495B2A8
:10E39000002B47D1CDB9002523683B626368227A00
:10E3A000BB6102F001013975BBF82410994210D20B
:10E3B0002B4A0091294801210BF0D4FA6FF01B047D
:10E3C00020462C37BD46BDE8F08F2B46C7F820A06D
:10E3D000E5E782F00202C2F340025846520107F11B
:10E3E000140105F00BFB1F4B984205D00B339842EC
:10E3F0000CD16FF00F04BCE74FF480420023786823
:10E4000008F034FA28B13046FFF70CFF6FF004042F
:10E41000AFE7D8F83030134A9342F7D1237ADB07BD
:10E4200002D400250C345FE73B6A9A45F9D12346B4
:10E4300008E0A91AD8688DB21AFA81F13B600FF092
:10E44000C8FE3B685A680C3B9542F2D2E9E76FF090
:10E4500085048EE7DB03030006000001ECEA0200FE
:10E46000A60403000000AD0B2DE9F0414568044609
:10E47000066928680FF081F918B96FF01200BDE83D
:10E48000F08130460FF02AFA7461AB68BBB9042200
:10E490000B2120466B7C0CF042FC0028EFDB0622AF
:10E4A0000B212046AB7C0CF03AFC0028E7DB012373
:10E4B0002046BDE8F0411A460B210CF030BC052384
:10E4C000062120462A7C0CF02AFC0028D7DBA8680D
:10E4D0000FF053F90028D0D0EB89A868297B43F4CA
:10E4E00080320127D0F810C013F0010FDCF80030A3
:10E4F00007FA01F714BF3B43BB43D0F808E0CCF860
:10E500000030DEF8003098470028B8DB01272B7B6D
:10E51000144A07FA03F3C6E90723A86806F11801AD
:10E520008368DB6913B96FF05700A8E73A4698474C
:10E530000028A4DB0C4BB362A868297B82680369BE
:10E540009669002EEFD01B688F401F4214BF4FF01A
:10E5500000734FF080634FF0A072B047002896DA46
:10E560008DE700BFAFAC02006DE50100262300225D
:10E570002DE9F04F044650F8100C91B0D0F80490FB
:10E580001146009306AB0CF0A6FB002805DA2046E6
:10E5900008F0CAFA11B0BDE8F08F0026234F97F8B3
:10E5A000008097F801A008F140036B4413F8273C62
:10E5B0001AEA030F13D0216931B1012354F8100C6A
:10E5C0000D6803FA06FB11BB08F101025346002156
:10E5D00054F8100CD2B20CF0A2FB0028D7DB0136A5
:10E5E0000E2E07F10207DAD1D9F8080099F80C507D
:10E5F0000669836805A95B6898470028C7D1059B11
:10E6000032685A400123AB401A42C3D0BFE78A6840
:10E610001BEA020203D04B680390984703981DB190
:10E620002B6829461D46CEE72B46FAE70F05030067
:10E630002DE9F04740F2FF15524E534FDFF84CC121
:10E6400000EB8101814202D10020BDE8F08704681F
:10E6500014F4804FC4F3C32EC4F3080340F0828047
:10E66000640CAB4208BF4FF0FF3316F80EE0192CD4
:10E670007BD8DFE804F00D131A1D7A7A7A7A7A7A59
:10E680007A204D7A7A7A7A7A7A7A7A7A5065686BD1
:10E69000C2F80C355C1C5CD10430D3E7C2F81435E9
:10E6A0005C1CF9D04FF0000910E0C2F80835F1E722
:10E6B000C2F81035F4E7C2F80835BEF1000FEFD10B
:10E6C0005C1CE9D04FF000094FF0060ED0F800A016
:10E6D0000AF40044002C16BF4FF00009C8464FF062
:10E6E000010803F01F045B0947D107EB8404D4F849
:10E6F0000032CAF3412A03EA0C0343EA8A0343EADD
:10E700000E2343EA090343EA4803C4F80032C3E78F
:10E71000C2F80C35D1E7C2F86035B3F1FF3F0468A9
:10E72000BAD0C4F30044A4B95FEA531820D101243D
:10E73000DFF854809C40C8F80C404FF00109C5E751
:10E74000C2F86435E9E7C2F86835E6E7C2F86C3527
:10E75000E3E75C090ED10124DFF82C809C40C8F867
:10E760000840EAE76FF015006FE76FF085006CE78F
:10E77000E460FFDE00239B60FBE70023803453F856
:10E780002430F6E72B05030000258440F0F8FCFF59
:10E7900038B570B14FF400450021064C0023E0FB72
:10E7A0000541054A2046FAF757FCBDE8384008F015
:10E7B00043BD38BD3F420F0040420F00F8B54468EA
:10E7C00000AF05460CF012FBA06A28B900212846CC
:10E7D0000CF081FBBD46F8BD0EF0CFFF0346B0B98B
:10E7E000A26A6C4688B011686A461548C2E90501FC
:10E7F0004FF400719183134942F8101F12484FF4EF
:10E80000E251FDF741FC6FF01200A546E2E7E38D0F
:10E81000A06A94F82C1043F400320124066913F026
:10E82000010F336804FA01F414BF2343A343D0F863
:10E8300008C03360DCF8003098470028C6DAC9E722
:10E8400033050300030000014CEB020017289FBFB3
:10E85000054B584300F5742000F510709ABF08600E
:10E8600000206FF015007047A086010010B5134C12
:10E87000A1421DDD124B98421ADCA04206DD9942EE
:10E8800006DD17236FF02100138010BD0023F9E788
:10E890006FF43A63A0F55B2018440A4BB0FBF3F029
:10E8A0001080584300F5742000F51070884202D99A
:10E8B0006FF01500E9E70020E7E700BF3F420F00D7
:10E8C000A05A3200A086010037B50D46212D114611
:10E8D0001C46406814D03A2D27D10A2A25D104229B
:10E8E000032100680DF107030CF012FA20B99DF81E
:10E8F0000720C4E90020002003B030BD1046F8E72F
:10E90000022A12D1052200680DF107030CF000FA6B
:10E910000028F1DB9DF80720002AEFD012F00A0F43
:10E9200014BF012200220248E3E76FF08500E3E70D
:10E9300020A1070070B50C2914464568036900F052
:10E94000928029398AB2142A00F29880142900F2A0
:10E950009580DFE801F00B5093811B939393939381
:10E96000939393939393937693707400188841F2E2
:10E97000883358434FF47A738012B0FBF3F203FBF1
:10E980001200584322606060002070BD9888FAF73A
:10E99000CFF801464FF08940FAF7D6F94FF07E5193
:10E9A000FAF714F8F9F734FD08F0ACFFF9F7BAFFFD
:10E9B0000646A88EFAF7BCF801463046FAF7C4F9C5
:10E9C00001463048FAF702F801464FF07E50FAF758
:10E9D000BBF92D49F9F7FAFF0546FAF7C7FA4FF0E8
:10E9E0007E512060284608F0C7FF2849FAF7F8F85A
:10E9F000FAF7BCFAC7E75A889B7A0D2B0ED80B2B77
:10EA00000ED8042B11D00020504348BF00F2FF3035
:10EA100080124FF47A7390FBF3F2B0E70F2BF2D130
:10EA2000E8684FF44873404202E04FF47A73286973
:10EA300090FBF3F0E8E71B7A00202360A3E75B7A02
:10EA4000FAE7EA68124B92FBF3F22260E86890FB67
:10EA5000F3F203FB120096E72A690D4B92FBF3F2E7
:10EA600022602869F3E7D8880A4B58430A4B90FB89
:10EA7000F3F000F5C02000F2AE50CAE76FF0850059
:10EA800083E700BF0FCF5B3B339388430024744977
:10EA900040420F0078783C0078ECFFFF2DE9F04F02
:10EAA000446887B020680EF068FE002800F05F819F
:10EAB00094F836300A22013305212068DBB20CF0CD
:10EAC0002EF90646002854D110254FF07E58DFF865
:10EAD000A4A2DFF8A49204F114076FF0004357F8E2
:10EAE000040F98420BD10235EDB2182DF5D16FF01D
:10EAF000004ADFF88892A24F04F124083EE0FAF7BA
:10EB00001BF85146FAF720F94946F9F761FF01462B
:10EB10004046FAF719F99B49F9F758FF8346A08E4A
:10EB2000FAF706F801465846FAF75AF8F9F770FC72
:10EB3000266BFAF759FE02460B463046CDE9022312
:10EB4000F9F744FCDDE90223F9F7BAFCF9F7CAFE4C
:10EB500006448302B3FBF6F303F0030200920321A1
:10EB60002A462068C3F387030CF0E8F8064600281D
:10EB7000B9D0304607B0BDE8F08F1A2558F8043FE9
:10EB800053450DD11A2DF8D162687F4811460DF119
:10EB900016030CF0AFFD163020D16FF01506E8E734
:10EBA00041F28832A9EB03035A434BBF774B784BB2
:10EBB0009B189B184CBF93FBF7F3B3FBF7F39BB287
:10EBC00003F00302009203212A462068C3F387035F
:10EBD0000CF0B4F806460028D4D0CAE70C22032172
:10EBE0009DF8163020680CF09AF806460028C0D12F
:10EBF000A268654811460DF116030CF07BFD163036
:10EC0000CBD00D2203219DF8163020680CF087F838
:10EC100006460028ADD1E2685E480DF11603A2F564
:10EC2000FA610CF0D6FC1630B7D0BDF816300321CF
:10EC300003F00102009220680822C3F347030CF09E
:10EC40007DF80646002894D1226953480DF1160339
:10EC5000A2F69E410CF0BDFC16309ED0BDF81630D9
:10EC6000032103F00102009220680A22C3F3470344
:10EC70000CF064F8064600287FF47BAF62694748D1
:10EC800011460DF116030CF035FD163085D0022229
:10EC90009DF81630114620680CF041F80646002811
:10ECA0007FF467AF0E22032194F8373020680CF010
:10ECB00036F8064600287FF45CAF0F22032194F853
:10ECC000383020680CF02BF8064600287FF451AF4E
:10ECD00001232422052120680CF021F80646002893
:10ECE0007FF447AF02460123052120680CF017F896
:10ECF000064600287FF43DAF012500952B462A46A5
:10ED0000052120680CF01AF8064600287FF431AF80
:10ED10002B460C22052120680CF001F8064600283D
:10ED20007FF427AF94F83A30BBB994F83B3033B155
:10ED300001230622032120680BF0F1FFA8B994F803
:10ED40003930002B3FF415AF012304220321206842
:10ED500007B0BDE8F04F0BF0E2BF2B465022032175
:10ED600020680BF0DCFF0028DFD0064601E76FF0DB
:10ED70001206FEE600007A4433938843AE0506008F
:10ED800078783C000FCF5B3BD8EF0200C4C3E1FFB3
:10ED90003C3C1E00CCEF0200C0EF0200A8EF0200D6
:10EDA00013B50A2A446833D1212917D03A292FD123
:10EDB0001B6820683BB901230522032102B0BDE88E
:10EDC00010400BF0ACBF0123002203210BF0A7FF82
:10EDD00000BB0123042203212068EFE7D3E90012DE
:10EDE0000D4B0E4803FB01220DF1060311460CF0FA
:10EDF00081FC10F1160F0DD0012202219DF8063082
:10EE000020680BF08CFF28B9012302460221E3E7BA
:10EE10006FF0850002B010BD40420F00A8EF020065
:10EE200070B5032904691CD80F4B58560F4B5E561A
:10EE30000F49B04202F1080201DD002070BD031D40
:10EE400004EB4303B3F9013025691B116B4393FBBA
:10EE5000F1F501FB153342F8085C42F8043C01303F
:10EE6000E7E76FF08500E9E7B9060300B5060300A0
:10EE700040420F0038B5056927216B6805F108028B
:10EE80001C680723A047041E06DA0221054A06482B
:10EE90000AF055FD204638BD2B7A13F00F0F18BF2E
:10EEA0000024F7E78A050300F4EA02003B2908B5CD
:10EEB00003D1BDE80840FFF7DDBF0329F9D00C29D5
:10EEC00007D105480221054A0AF039FD6FF0850097
:10EED00008BD6FF03C00FBE7F4EA0200A90503005F
:10EEE00008B50221034A04480AF029FD6FF08500A5
:10EEF00008BD00BFCA050300F4EA02002DE9F04195
:10EF000084B0D0F8048000AFD8F800300546066918
:10EF10009847041E17DB73680F2128469B68FA1D6B
:10EF20009847041E05DA384A012138480AF007FDDF
:10EF300009E0FB79332B0BD00121354A33480AF025
:10EF400007FD6FF0150420461037BD46BDE8F0817F
:10EF500098F80C20D3070BD544F6161142F28B4CCF
:10EF600049F22D2E2B4BC3E900C12B49C3E902E125
:10EF700094070AD573681E211C69802328461A4607
:10EF8000A047041E01DA254ACEE74FF00008072308
:10EF9000C7F8098087F80D803B72736820215C6890
:10EFA0002846062307F10802A047041E01DA1C4A7E
:10EFB000BAE7184B42461B68232133617368284621
:10EFC000DB689847041E01DA164AADE76C468AB042
:10EFD0006A4633691449C2E9088351610220042159
:10EFE0000623C2E9060142F8103F4FF4435143465D
:10EFF0000648FDF749F87368A546472220212846B0
:10F00000DB68984704469EE7F4050300F4EA020033
:10F010000C060300CCC5002094B6010023060300B3
:10F0200049060300690603009106030010B5436812
:10F03000046958680EF0A1FB38B906480121064A58
:10F040000AF07DFC6FF0120010BD044B00206360DD
:10F05000FAE700BFF4EA0200CE0603001CF002004B
:10F060002DE9F74306464FF0000800220121082051
:10F07000FDF79AFE0820FDF767FE776835693C6862
:10F080004146C4F800852E60D7F80C9001AA484686
:10F090000BF099FE002837DB019BD9F80020197985
:10F0A0001868FFF7C5FA00282EDB6B7A3169012B4F
:10F0B00003D0032B26D14FF01008AB7A032B21D1BC
:10F0C00095F80BC0BCF1000F02D0BCF1010F19D1B3
:10F0D0002A7A12B1022A15D10E226B687068B3F534
:10F0E000164F00687BD02DD8B3F5165F7AD016D8AE
:10F0F000B3F5966F78D00AD8B3F5967F77D0B3F58D
:10F10000167F77D06FF0850003B0BDE8F083B3F5CC
:10F11000166F72D0B3F5965FF4D15C4B3EE0B3F559
:10F12000E14F6DD007D8B3F5615F6BD0B3F5964F63
:10F13000E8D1574B32E047F6122E7345E2D14FF437
:10F1400000032BE0B3F5613F5ED013D8B3F5963FD3
:10F150005DD009D84DF6C02E73455AD0B3F5614F36
:10F16000D0D14FF46B0319E0B3F5E13FCAD14FF0B2
:10F17000EB7313E0B3F5612F4ED009D8DFF814E13B
:10F1800073454CD0B3F5E12FBCD14FF0E86305E0F7
:10F19000DFF804E17345B5D14FF08053C0F8243552
:10F1A000736848EA0C081B6842EA0802C3F86C2539
:10F1B0000B1DD5E9010183E803007B6899073DD564
:10F1C00005F1180003F0A0FE344B98422AD03448D1
:10F1D0000121344A0AF0B3FB6FF0040094E74FF4C6
:10F1E0001D03DBE7304BD9E74FF49E23D6E74FF4FE
:10F1F000A033D3E74FF41C33D0E74FF41D23CDE702
:10F200002A4BCBE72A4BC9E74FF06C73C6E7294B73
:10F21000C4E74FF46503C1E74FF07063BEE74FF0FA
:10F220008063BBE7287E04F10C0204F590710DF0B9
:10F2300028F801202B7E984003F056FD0823C4F8DF
:10F2400000353B7A53B9C4F81031D4F810316B69EA
:10F25000C4F834350123C4F8383523607B680020B6
:10F260009A075CBF4FF48073C4F804337B68DB06F5
:10F2700044BF4FF48003C4F804332B69C4F8443509
:10F280000123C4F84805A360E3603DE700B0130024
:10F2900000A04E0090D0030040420F000000AD0BD4
:10F2A0005CEB0200E60603000050270000C075007A
:10F2B00000F03A0000903A012DE9F04104460D4675
:10F2C00007690EF010FC4FF02008B0B92C4B1B78EA
:10F2D0009BB1642660680CF0EEFAF0B901200CF0E6
:10F2E000CEFF013EF6D10021212007F0A5FFF0E777
:10F2F00086F31188BFF36F8FF5E7EFF31186314680
:10F3000088F31288BFF36F8F60680CF0D4FA80B96D
:10F3100086F31188BFF36F8FEFE7EFF31186314665
:10F3200088F31288BFF36F8F60680CF0C4FA00286E
:10F33000DED03B691D70626838691368C3F8440504
:10F340000120C3F848050020C3F82001D3F820515C
:10F35000C3F858015268D3F85801D20608D50820DE
:10F3600062681268C2F800054FF48002C3F80423F3
:10F3700001229A6081F31188BFF36F8FBDE8F0819D
:10F3800064E400200123834070B5DC430B4AD2E8DB
:10F39000EF1F01EA0405C2E8E65F002EF7D14FF443
:10F3A000803282400648C0F80823BFF35F8FBFF366
:10F3B0006F8F0B4214BF0120002070BDF4D50020D8
:10F3C0000050014070B40E4922F07F46D1E900346C
:10F3D000D01AC31844F10004C1E90034A6F50013A3
:10F3E000B3F5400F09D2074B1B681A0A1B069C197C
:10F3F000054B42F10005C3E9004570BC08F0B2B806
:10F40000F0CF0020F8D50020F8CF0020D9B101239B
:10F410000D4A8340D2E8EFCF4CEA030CC2E8E1CFBB
:10F420000029F7D14FF48033084A8340C2F80433EF
:10F43000074BD3E8AF3FC340DB0742BF4FF4001296
:10F44000044BC3F800217047F4D500200050014060
:10F45000F0D5002000E100E00D4B1868010A00061D
:10F46000BFF35F8F0B4BD3F80435181841F100013F
:10F47000B3F5801F0AD2084BD3E90023904271EB09
:10F48000030303D210F1807041F10001704700BF07
:10F49000F8D5002000500140F8CF00202DE9F04FB2
:10F4A00085B016461F4604469DF840A0FFF76AFF48
:10F4B0000190FFF7D1FFB04271EB070352D23B4BF3
:10F4C000301A67EB0101984271F100014DD2384BBF
:10F4D00003EB0413D3E902239F4208BF964258D09E
:10F4E0004FF48038334908FA04F8204626F07F4B61
:10F4F000C1F848830CF026FA4FF00309584604F18E
:10F500005005AD00ADB205F1804504F5A87305F5D1
:10F51000A8350293029A20F07F4341F82230C1F8C7
:10F520004483D1F80435244AC01A033820F07F40C0
:10F5300090422ED9286868B1D1F80435A3EB0B00AE
:10F5400020F07F40B0F5000F039322D920460CF045
:10F55000F9F9039BBAF1000F07D109EB030009F198
:10F560000109D7E7BAF1000F09D06FF01505204661
:10F570000199FFF74BFF284605B0BDE8F08F012346
:10F580000E4AA340D2E8EF0F1843C2E8E10F00296A
:10F59000F8D107490E982301C8500F9B01EB0412C4
:10F5A0000025C2E902675360E1E700BF0100800067
:10F5B000E0CF002000500140FDFF7F00F0D500208B
:10F5C0007FB500254FF0FF304FF0FF31194C1A4B3B
:10F5D0000226C4F80833C4F84833184BC4F8085559
:10F5E000C3E902014FF480334FF40012C4F804332E
:10F5F000134B0121C4F804631520C3F880212A4667
:10F60000FDF7D2FB1520FDF79FFB01230D4AA360F8
:10F61000236013600C4B0D4A009328460023CDE96C
:10F620000155FFF73BFF3046FEF77EFB284604B04E
:10F6300070BD00BF0050014003000F00E0CF00206C
:10F6400000E100E0F4D50020C5F30100FFFF7F00DA
:10F650002DE9F7432E4BD3F8042390070BD5D3F8AD
:10F66000042142B10022C3F804212A4AD3F804310C
:10F67000136801331360264AD2F80433D90326D520
:10F68000254BD3E8EF1F21F00100C3E8E40F002C65
:10F69000F7D1CB0702D4D2F84031C3B100251C4CBE
:10F6A000C4F84051D4F84031FFF7D6FEEFF3118291
:10F6B000202383F31288BFF36F8F184BD3E90267BF
:10F6C000B042B94106D282F31188BFF36F8F03B005
:10F6D000BDE8F0834FF0FF38D3E900104FF0FF3959
:10F6E0001D60C3E902894FF48033C4F84833C4F87D
:10F6F0004051D4F8403182F31188BFF36F8F002955
:10F70000E5D0009032463B4628468847DFE700BFF9
:10F7100000500140F8D50020F0D50020E0CF0020B7
:10F7200030B5431C124C85B005D08442A8BF0446B6
:10F73000012CB8BF0124FFF78FFE0E4B0C4DD3E90F
:10F740000013401AB0F5000F0FD22218AA4228BFAA
:10F750002A46002052180849CDE90100009143F1E2
:10F760000003FFF79BFE05B030BD2A46F1E700BF5E
:10F77000FFFF7F00F0CF0020C5F3010008B5FFF7C1
:10F780006BFE024B1B68C01A08BD00BFF0CF002003
:10F7900070B50546054C064EB44200D370BDD4E9A1
:10F7A0000031284698470834F6E700BF341F0300AD
:10F7B000341F030070B5002201212A20FDF7F4FA5E
:10F7C0000B4806F081FC044628B101210346094A92
:10F7D00009480AF0BDF8094D094EB54201D320464B
:10F7E00070BDD5E90031204698470835F5E700BFE0
:10F7F00068F002001F0703003CEB0200341F030007
:10F80000441F0300F0B50F4B01461A680E4B0B2541
:10F81000002618461F46B84201D3013D04D11846C0
:10F82000013A19605A60F0BD04688C42FBD03CB1CB
:10F830004468141BA642BCBF034626460830EAE7CC
:10F840000346ECE7B8D60020C4D600200020054BC4
:10F85000C3E90000044BD3E8EF2FC3E8E10F002910
:10F86000F9D17047BCD60020B8D600202DE9F0476A
:10F8700088B005460E460DF079FF20B96FF06D0097
:10F8800008B0BDE8F0870EF092FA33680446002B0A
:10F890000F4604D107F04EFC6FF00A00F0E7BCBF42
:10F8A0004FF0FF3333600122002101A80EF099F8D8
:10F8B000E8460795EFF3118A202383F31288BFF3FC
:10F8C0006F8F07F0D7FCFFF79DFFDFF818914268B4
:10F8D000D9F800309A426CD10023434D00936B68F5
:10F8E000002B6DD1C5E900888AF31188BFF36F8FB3
:10F8F00033685A1C69D04FF4004E40F2E7300021C3
:10F9000023EAE37C4FF47A720023CCFB0E01F9F773
:10F91000A3FB02460B4601A806F0A8FFEFF3118AED
:10F92000202383F31288BFF36F8F00222B685BB113
:10F93000434554D10099002A4BD16A6829609A4204
:10F9400000D169600023009307F094FCFFF75AFF91
:10F95000D9F8003043608AF31188BFF36F8F0DF040
:10F9600005FF00288AD035686B1C27D00EF01FFADF
:10F970004FF47A7EA0FB0E320EFB0121A4FB0E4257
:10F980000EFB0722DB0BE40B43EA414344EA42440B
:10F990001B1B4FEAD1314FEAE57C61EBD231ED1A06
:10F9A0006CEB010CBCF1000FB8BF002535602DB920
:10F9B00072E743608AF31188BFF36F8F00205FE71F
:10F9C000C3F80080C5F804808EE74FF0FF3213467D
:10F9D000A1E711606968994208BF6A60B2E71A46F8
:10F9E0001B68A4E7B8D60020BCD6002030B4046859
:10F9F0002CB10D4B9C4202D3A8339C420BD30B4C31
:10FA00002378062B0BD85D1C2570074C03EB4303B2
:10FA100004EBC3030360006830BC0DF0E2BF6FF07D
:10FA20000B0030BC704700BF10D600200EDF002056
:10FA300002682AB1094B9A4202D314339A4206D380
:10FA4000074B1A7832B901221A70044B0360006820
:10FA50000DF044BF6FF00B00704700BFFCD50020D5
:10FA60000DDF002038B505460A4BD3E8EF1F013102
:10FA7000C3E8E21F002AF8D1074B1C6804B938BD5F
:10FA8000E369AB4201D005B113B9201D06F0CAFEEF
:10FA90002468F3E7B8D60020BCD600200146002237
:10FAA000002301480DF0E1BE14D7002001460148B3
:10FAB0000DF0E5BE14D700200146002200230148C6
:10FAC0000DF0D3BE28D70020014601480DF0D7BE67
:10FAD00028D7002008B54FF48062064906480DF08B
:10FAE0007BFEBDE808404FF40252044904480DF083
:10FAF00073BE00BF0FDF002014D70020E884002071
:10FB000028D7002010B5044B1C6804B910BD201D77
:10FB100006F088FE2468F8E7BCD6002070B50546DC
:10FB2000054C064EB44200D370BDD4E900312846DE
:10FB300098470834F6E700BF241F0300341F030072
:10FB4000014804F0D7BD00BF1DFB0100292800F0CB
:10FB500099800ADC01284FD0062800F09580002803
:10FB600000F08E804FF0FF307047B0F58D7F04D0ED
:10FB7000B0F5007FF6D11E2948E04B1E142BF1D8BA
:10FB800001A050F823F000BFDFFB0100DFFB010004
:10FB9000DFFB0100DFFB0100DFFB0100DFFB0100F9
:10FBA00065FB010065FB010065FB010065FB0100D1
:10FBB00065FB0100DFFB0100DFFB0100E5FB01004D
:10FBC000E9FB010065FB010065FB0100DDFB0100B5
:10FBD000EDFB0100F1FB0100F5FB01000E2100200F
:10FBE000116070470F21FAE71021F8E71121F6E7BD
:10FBF0001221F4E71321F2E736293FDC202907DC44
:10FC00001429ECD038DC0229E9D00429E7D0A9E78F
:10FC1000A1F12103152BA5D801A050F823F000BFB6
:10FC2000DFFB0100DFFB010065FB010065FB01005C
:10FC300065FB010065FB010065FB0100DFFB0100C6
:10FC400065FB010065FB010065FB010065FB010030
:10FC500065FB010065FB010065FB010065FB010020
:10FC600065FB0100DFFB0100DFFB0100DFFB0100A2
:10FC7000DFFB0100DFFB01001529C7E73D29C5E7D0
:10FC80001F29C3E72029C1E73729BFE74FF0FF321B
:10FC9000064B00201A609A611A639A641A669A6782
:10FCA000C3F89020C3F8A820704700BF40D70020B9
:10FCB0000B490346087880B90A49097839B1A2F599
:10FCC000807102290AD9A2F58872012A06D9013B5E
:10FCD000022B8CBF0020012070470020704700BF1E
:10FCE00090E300208FE3002070B400231825016802
:10FCF000084C05FB03F2A658B14206D1B0F9061034
:10FD00000832A01870BC07F0AFBD0133082BF0D14A
:10FD100070BC704740D700202DE9F3470746904656
:10FD20000C4679B300231A46C868834234D1802A2E
:10FD300071D800254FF0FF324FF0FF3338480BF0F9
:10FD400006FFA946374EE368AB422CD8002635465D
:10FD5000DFF8D0A0B14511DD85B96368384601935D
:10FD60002368A9EB060200930AEB060143460BF059
:10FD7000F2FE051EEEDD2E44B145EEDC28480BF008
:10FD8000E8FE05E009F009FF16234FF0FF35036098
:10FD9000284602B0BDE8F087A16801EBC3014968BD
:10FDA00001330A44C1E7A36806EB090003EBC5026F
:10FDB00053F8351052680EF00CFAA3684FEAC50AE2
:10FDC00053445B6801359944BDE7A3684FEAC60A0E
:10FDD00003EBC6035B683BB14FF00009A36803EB7C
:10FDE0000A025268914504D30136E368B342ECD865
:10FDF000CEE753F80A1063684944019323683846F4
:10FE00000093A2EB090243460BF0A5FE011E05DBA1
:10FE100089440D44E2E700263546E6E70D46B7E79C
:10FE200020C900200FE300204FF0FF324FF0FF33D6
:10FE300070B505460B480BF08AFE002318200A4ACD
:10FE400000FB03F156588C18013605D15550054872
:10FE50000BF07FFE204670BD0133082BF0D100244B
:10FE6000F5E700BFBCC8002040D7002038B5094DD9
:10FE700004464FF0FF3228464FF0FF330BF067FE89
:10FE800000234FF0FF32C4E900232846BDE8384084
:10FE90000BF05FBEBCC8002010B50446094B0A4AEF
:10FEA000186003680948DA61FDF794FB23680C3396
:10FEB000D3E8EF1F41F00801C3E8E21F002AF7D1A1
:10FEC00010BD00BF3CD70020DDFF010094F0020010
:10FED000F0B5A1F58173046887B0032B57D8DFE82C
:10FEE00003F0024077530127D2E9016113683A4ACF
:10FEF000B3F904300492ADF814308DF816703368FD
:10FF0000994204D109F049FE0C23036014E000F18A
:10FF1000080528460EF000F92B46002239463068C5
:10FF20000EF0D1F80823204600933C22394604AB5A
:10FF300005F012FA044610B14FF0FF340EE03368BA
:10FF400014333360CDE90200284602AA03A90EF05B
:10FF5000E8F8039B002B18BF6FF07704204607B02A
:10FF6000F0BDD2E900421368143313600023CDE9D9
:10FF7000033303AA04A908300EF0D3F8049B0BB195
:10FF8000039BE3800024E9E713684360FAE7032951
:10FF900012D0042918D1156835F4804303D009F034
:10FFA000FCFD1623036004212046C5F3803207B010
:10FFB000BDE8F0400DF0A4B9204600220DF0A0F9F4
:10FFC000840304F48044C9E709F0E7FD16239CE7A5
:10FFD0006FF05E04C2E700BFE9FC01002DE9F041CB
:10FFE0000D1E0746904612DA07F068F81C4E0123F2
:10FFF00033704246384625F04041FDF7C3F90023EF
:020000040002F8
:100000003370044607F06EF82046BDE8F0816B00BF
:1000100003D507F053F8134EE9E7FBF71DF8041E6C
:1000200009DB2946424638460CF0E9FC051E05DA94
:100030002046FBF765F84FF0FF34E5E7FFF7F4FEE5
:10004000014638B909F0A9FD0C230360284605F0E4
:1000500051F9EDE72046044AFBF73AF8D4E700BF30
:1000600090E300208FE300209CF002002DE9F04F88
:1000700014460E4600218BB00546202202A81F46DA
:1000800001910EF0B3F85CB163680293E3680493E6
:10009000A368039323690593236A03B1089302AC11
:1000A0004FF0FF324FF0FF333B480BF050FD31462D
:1000B0002246284601AB04F031FE064648B9804688
:1000C00081464FF0180A019D38604DB901980CF037
:1000D00078FC31480BF03DFD30460BB0BDE8F08FA9
:1000E00054200EF03DF8044600284FD0C0F8009090
:1000F000C0F820902B684360AB68C3606B68836076
:10010000EB680361D5F804B0BBF1010F15D10820ED
:100110000EF026F8E061002835D00823A3616B6952
:100120005A88A0F800B042805B684360B8F1000FC5
:100130002FD13C60A046ED69C7E7BBF1020F09D0A3
:100140000EF007F86FF0050638680BF0F3FC00239B
:100150003B60BBE718200EF003F8E06198B1C4F8EB
:1001600018A06A695388111D4380034602F1140CDC
:1001700023F804BB51F804EB614543F804EBF9D1D3
:10018000137D0375D2E720460DF0E3FF6FF00906FB
:10019000DAE7C8F80040CDE7E4C800202DE9F043D5
:1001A00089B007460C461546FAF756FF0646002E5C
:1001B00038681DDBFCB10DB32B6801AA082B18BFF2
:1001C00016230DF10809019349460CF092FDB0F198
:1001D00000080ADBFFF728FE074690B909F0DDFCAE
:1001E0000C230360404605F085F83046FAF788FF97
:1001F0004FF0FF3618E02246A146E5E72A46A94619
:10020000E2E764B15DB1B9F80020012A10D10823FA
:100210002B60BDF80A3022806380039B63603946FF
:100220003046164AFAF754FF304609B0BDE8F0836D
:10023000022A17D118232B60BDF80A3003AD638062
:1002400023460DF11C0C23F8042B2A4603CA6245F1
:1002500018605960154603F10803F6D19DF81C306B
:100260002375DCE709F099FC86230360404605F01E
:1002700041F83846FFF7FAFDB7E700BF9CF00200EF
:1002800007B5D0E90032012100920348034A09F082
:1002900069FB03B05DF804FB3CEB0200620703005E
:1002A00008B5034903480BF0BCFD6FF0150008BD0D
:1002B0008B070300DCEA020008B5034903480BF092
:1002C000B0FD002008BD00BFA6070300DCEA020065
:1002D00013B50B480469836801A95B689847002837
:1002E00005D008DA02B0BDE81040FFF7E5BF23688B
:1002F00001985840C00F003818BF012002B010BD4F
:10030000D0E7020010F0010210B50ED111F0010487
:1003100009D0192106480BF074FD044618B10549AF
:1003200005480BF07EFD204610BD0122F1E700BF1D
:10033000D0E70200BB070300DCEA0200002814BF7C
:100340004FF098624FF4001210B5114B19699B6879
:100350009C699CB1130206D50B68002BACBF4FF013
:1003600098624FF0307202F0C0631F21084802F417
:10037000C002A047044618B9204610BD6FF05704CC
:1003800001212346034A044809F0E2FAF4E700BFDA
:10039000D0E70200D1070300DCEA020038B5EFF332
:1003A0001185202383F31288BFF36F8F0E4C2378BF
:1003B000ABB90E4B984200D050B90020FFF7BEFFFA
:1003C00018B10B490B480BF02CFD00220A4B1A7098
:1003D0000123212223700948002306F047FC85F3FE
:1003E0001188BFF36F8F38BD92E30020D0E7020081
:1003F000F1070300DCEA020091E3002000D00020B6
:100400002DE9F041334F3B7853B10020FFF796FFC1
:1004100028B131493148BDE8F0410BF002BD3870D8
:10042000FFF756FF04462E4BD3E8EF2FC3E8E14F0A
:100430000029F9D12B4BDFF8B0801A7842BBD8F8ED
:100440000060A64219D0294B66401B680BB13146AB
:1004500098474FF0FF334FF0FF32254806F0FCF885
:10046000244B1D6835B1043D2B6831462046984722
:100470006D68F7E71E4806F067F9C8F8004054B108
:10048000BDE8F0414FF4A47200231B4806F0EEBB18
:1004900000221A70F1E7EFF31186202383F312880C
:1004A000BFF36F8F154B1D78012D05D086F3118892
:1004B000BFF36F8FBDE8F08128461C70FFF73EFF49
:1004C0003D7086F31188BFF36F8F0028F2D00C497E
:1004D000A0E700BF91E300200D080300DCEA020062
:1004E00030D80020ACC7002004D8002034D8002029
:1004F00008D800201CD8002000D0002092E3002063
:100500002608030010B54FF4003108480BF064FCD6
:10051000044620B9BDE810400F21FFF7F3BE04499F
:1005200004480BF07EFC204610BD00BFE0F0020046
:100530003E080300DCEA0200054BD3E8AF3F00B100
:100540000360044811B102685A400A6003607047B2
:1005500030D8002000D80020F8B5264B1860264877
:100560000DF0BCF9254926480BF036FC044628B1AD
:10057000244925480BF055FC2046F8BD234FBD68A3
:10058000AE691EB96FF057042149F2E703464FF4F4
:1005900000121F213846B04704460028F4D11D49F7
:1005A0001D4B4B604FF000438B60EB69F3B10122B0
:1005B000384698470446D8B9184919480DF083FAC7
:1005C0000122184B16481A700023002206F01AFB6D
:1005D00021462046FFF7B0FFFFF77AFE124BD3E823
:1005E000EF2FC3E8E10F0029C6D0F8E76FF05704FA
:1005F0000E49BEE734D8002008D8002010000100C2
:10060000E8F0020058080300DCEA0200D0E702002C
:100610007508030024D800209D0302000104020095
:1006200000D0002092E3002030D800209008030082
:100630000A4610B518B1BDE81040FFF731BE1921C8
:1006400005480BF0DEFB044618B1044904480BF0E2
:10065000E8FB204610BD00BFD0E70200BB07030047
:10066000DCEA020008B5064804F03EF8034620B173
:100670000121044A044809F06BF9002008BD00BFBD
:100680008D060200B8080300C4EA02002DE9F84311
:1006900004460026244DDFF8949000AF4D4521D349
:1006A000EEB12046F8F726FF0022411D0023204826
:1006B0000DF0DBF8054650BB6E4688B06A461D4B10
:1006C000C2E905344FF4007393831B4B42F8103F8B
:1006D0004FF4E45103461948FBF7D6FCB546BD4636
:1006E000BDE8F88395F8088018F0010F0BD1296850
:1006F00019B120460DF0CAFD28B118F0020F04D040
:1007000020466B6898470C35C8E70126FBE7214671
:1007100004300DF082FD294609480DF057F90948CB
:1007200006F002FADBE700BFCCC7002020C800209B
:1007300094C80020E508030003000001C4EA020099
:10074000A8C9002004C600202DE9F843134E144F19
:10075000DFF8508000220023304606F031F80546CD
:10076000B8B9BDE8F883237ADA070AD49B0708D41E
:10077000216819B148460DF089FD10B148466368FB
:1007800098470C34BC42EED3294640460DF077F82A
:10079000E0E7054C05F10409F4E700BFA8C9002013
:1007A00020C8002094C80020CCC70020094B1B5C47
:1007B00003F00303022B08BF2038C0B2A0F14103AD
:1007C000192B04D9A0F15F0358425841704701200A
:1007D000704700BFD91D0300A0F12C03DBB2112B21
:1007E0009DBF0348D84000F001000020704700BFC3
:1007F00001400200F8B505460024094E56F8047B76
:100800003846F8F777FE3946024628460DF00DFDCA
:1008100020B10134042CF1D10020F8BD0120FCE707
:10082000F0F002002DE9F0430468A3B0237880467D
:100830000E4615460094002B00F0CF80684B1B78C5
:10084000062B13D10020621C00921146074612F8B5
:10085000010BFFF7ABFF0028F7D107B100910B1B8D
:100860002246314628460BF090FB46E0013B082B20
:1008700043D8DFE803F064495AA20D421C3F05004B
:1008800022460021134612F8010B60B10121F9E75D
:1008900022460021534F134612F8010B385C10F02A
:1008A000440F40F0988001B100931B1BD8E76846C5
:1008B0000BF0D6FA0022009B4A481F4613F8011B92
:1008C000415C490710D102B100973B1B22463146DB
:1008D00028460BF05AFB3B783D2B07D17B783F2B0A
:1008E0000BD10237009708E00122E6E73F2B04D145
:1008F0000137F7E728460BF01EFB0020009BC8F8E5
:10090000003023B0BDE8F08327463A7810460BF05C
:100910009EFA3B46013708B9002AF6D122463146F5
:1009200028461B1B0BF031FBDCE727463A783B4699
:10093000222A07F10107F1D0002AF7D1EEE720467D
:100940000A2201A907F062FB0124019B0290009397
:10095000009B1878292825D020B303F10109FFF75F
:100960003BFFCDF8009008B9274619E00A2201A9FB
:10097000484607F04BFB22AB671C03EB840444F8AA
:10098000800C4846F8F7B6FDDDF80490044648466A
:10099000F8F7B0FD844206D0202FCDF8009002D0A9
:1009A0003C46D5E72746BB003146284602AA0BF055
:1009B0000FFB009B013300939FE70A22204602A908
:1009C00007F0A8FA0B4602990246009128463146E4
:1009D0000BF0C6FA91E701215DE74FF0FF3090E799
:1009E00094E30020D91D030010B50446F8F782FDFA
:1009F000012821D923781249CA5C02F00302022A95
:100A000008BF203B412B17D16378CA5C02F0030278
:100A1000022A08BF203B542B0ED1A27802F0F70324
:100A2000232B0BD0252A09D010460BF010FA10B951
:100A3000B2FA82F0400910BD0020FCE70120FAE77D
:100A4000D91D03002DE9F04107460468DFF89081C5
:100A500000293DD120780BF0EEF9624E054660B3D7
:100A6000062305222046604933700DF0DEFBF8B105
:100A7000052220465D490DF0D8FBC8B10B22204667
:100A80005B490DF0D2FB98B10A22204659490DF07E
:100A9000CCFB68B10B22204657490DF0C6FB38B19C
:100AA0000722204655490DF0C0FBB0FA80F56D09CC
:100AB00088F8005000203C604EE098F8003053B9B0
:100AC0002046FFF791FF002848D007233370F1E755
:100AD00098F800301BB10222424B1A70EAE7002955
:100AE00043DD224615781646284601320BF0AFF951
:100AF0000028F7D13046F8F7FDFC032830D92B4603
:100B00003F4A515D01F00301022908BFA5F120030E
:100B1000412B25D17378D15C01F00301022908BF74
:100B2000203B542B1CD1B378D15C01F00301022986
:100B300008BF203B2B2B0AD0252B11D1F378D25C98
:100B400002F00302022A08BF203B582B08D00922DA
:100B50006FF00100234B1A70BDE8F0810223B5E766
:100B600020780BF068F9002836D12278244B9B5C62
:100B70005B070AD42D2A08D02B2A06D0222A07D1B7
:100B80000322184B01341A7094E70422154BA4E792
:100B9000282A04D10122134B14441A708AE7104604
:100BA0000BF055F988B10F490B78042B0AD1224676
:100BB000144612F8010B0BF04AF90028F8D105236E
:100BC0000B7077E7082B3FF475AF1046FFF704FE74
:100BD00010B10822034B80E74FF0FF30BCE700BFA5
:100BE00093E3002094E300201C0903002209030082
:100BF00028090300340903003F0903004B090300DF
:100C0000D91D03002DE9F74F894616461F46804639
:100C1000002800F09980002A00F096805368002B8D
:100C200000F09280002410460BF060F942463368D1
:100C3000CDF804809F4228BF1F46454B1C70454B92
:100C40001C70114608780BF002F925460132044663
:100C50000028F6D105B101910025DFF8FCB0019B19
:100C60001A78002A50D0AF424ED91BF802202946EC
:100C7000120748BF013301A848BF0193FFF7E2FE06
:100C8000431C41D0023008BF00253246294601A846
:100C900008BFCDF80480FFF7C5FD013034D0019ABC
:100CA0001078FFF799FDB0B150780BF0D0F878B11B
:100CB0000135BD4241D0294601A8FFF7C3FE0130EE
:100CC00022D03246294601A8FFF7ACFD01301BD0E7
:100CD000019B01330193019A10780BF0B8F838B3F7
:100CE000013211789246084601320BF0B0F8002824
:100CF000F7D139B108460BF09EF818B95046FFF706
:100D000079FDA8B1CDF804A0019DC4B92B78CBB171
:100D10002846FFF76FFD002814BF00206FF00A007F
:100D2000B9F1000F01D0C9F8005003B0BDE8F08F51
:100D30000135BD4208BF012491E70446E4E76FF0A6
:100D40000600EDE72046EBE76FF01500EDE700BF8A
:100D500094E3002093E30020D91D030010B504465E
:100D600092B04822002168460DF040FA0D4B2168F0
:100D70001A6891421A4603D161685B6899420ED0A5
:100D800094E80300012382E803008DF8003002ABF1
:100D900094E8030083E80300684600F0EDFD12B01C
:100DA00010BD00BF3CD800202DE9F74F05230422D9
:100DB0006E460025CDE90023154FDFF85880DFF897
:100DC000589056F804BB154BBBF1040F14BF3C46BA
:100DD0004446204614BFCA469A46F8F78BFB0428BF
:100DE00010D121465046F8F77BFB58B122465946B0
:100DF0000B4803F085FC034620B10121094A0A484B
:100E00000BF0A3F915B103B0BDE8F08F0125D8E7C9
:100E10004CE4002051E4002038E400203DE40020B0
:100E2000760903008709030014EB020008B50B489C
:100E300003F066FC034638B10121094A09480BF06A
:100E400084F96FF00D0008BD074803F059FC002835
:100E5000F9D003460221054AF0E700BFB1090300BB
:100E6000BC09030014EB020076100300F209030032
:100E700010B5044692B04822002168460DF0B6F93C
:100E80000122204602A900F049FE034630B10121AB
:100E9000064A07480BF059F912B010BD0323684603
:100EA0008DF8003000F068FDF6E700BF280A030067
:100EB00014EB02000023064A13601371054A136005
:100EC0001371054A13601371044A1360137170475C
:100ED00047E400203DE4002042E4002038E4002004
:100EE00010B5044692B04822002168460DF07EF904
:100EF000204602A900F07AFF034630B101210A4AD8
:100F00000A480BF022F912B010BD029B039AA3F518
:100F10009C53083B1343F6D1062368468DF80030F6
:100F200000F02AFDEFE700BF4F0A030014EB0200B8
:100F300010B5044692B04822002168460DF056F9DB
:100F4000204602A901F0A0FB034630B10121104A5E
:100F500010480BF0FAF812B010BD9DF808305A1E78
:100F6000032A01D9072BF6D1DDE90421A2F59C5310
:100F7000083B0B4308D00A4308D00A2368468DF883
:100F8000003000F0F9FCE6E70823F7E70923F5E76E
:100F9000830A030014EB020010B5044692B0482205
:100FA000002168460DF022F9204602A901F0CAFB93
:100FB000034630B10121064A06480BF0C6F812B0CC
:100FC00010BD0B2368468DF8003000F0D5FCF6E725
:100FD000BF0A030014EB02001FB50024074B4FF4B7
:100FE0008062029302AB009305490E2305480394E7
:100FF00005F0A0FD204604B010BD00BFEF0A0300BD
:1010000068E8002060D00020072810B5144605D0FD
:1010100009280CD0BDE81040FFF74CBF07480DF081
:10102000FCF821460648BDE810400DF0F6B805482A
:101030000DF0F3F821460448F5E700BF47E400202F
:101040003DE4002042E4002038E4002010B596B0D2
:1010500004464822002104A80DF0C8F800236A467F
:1010600000938DF8043002938DF80C30204602ABCB
:1010700006A9F8F7D1FA034630B101210C4A0D4810
:101080000BF063F816B010BD69469DF8180002AA6F
:10109000FFF7BAFF9DF818301BB1074907480CF05D
:1010A00002FD022304A88DF8103000F065FCE9E78A
:1010B000FD0A030014EB020024C6002060D00020CB
:1010C00008B550B9054B1B783BB1FFF7F3FEBDE8FF
:1010D0000840034903480CF0E6BC08BD56E4002074
:1010E00014C6002060D0002008B50121034A04483E
:1010F0000BF029F86FF0150008BD00BF190B0300B5
:1011000014EB02002DE9F0410025A4B002AF044623
:101110004822002107F140000DF068F830222946EE
:1011200007F11000BD710DF061F84FF0FF3307F1CA
:101130000808C7E90233FB1D009301212046CDF8C2
:10114000048007F11003BA1D00F034FDB8B16E46FB
:101150008AB002AA3D4BD461C2E9053040F20133A6
:1011600013843B4B42F8103F4FF411512B46394842
:10117000FAF78AFFB5468837BD46BDE8F081BB79EE
:1011800003F0FB03012B04D1BB69013356D10423C7
:10119000BB7100F0BDFB0028EDD12F4ABB7911785F
:1011A000994208D087F8400007F14000137087F893
:1011B000483000F0E1FB294BB9699A68914203D1AC
:1011C000DB68FA699A421DD00423244D07F110040C
:1011D00087F840300FCC0FC50FCC0FC594E80F0037
:1011E00085E80F0007F1480607F110050FCD0FC67F
:1011F0000FCD0FC694E80F0086E80F0007F14000FE
:1012000000F0BAFB164AFB791178994209D01370A5
:10121000052207F1400087F8402087F8483000F0A9
:10122000ABFBBB7903F0FB03012BA4D1BB680133FB
:1012300008D10C490C480CF036FC9CE70B4805F033
:10124000F1FAA6E74046FFF789FD94E72F0B03006C
:101250000400000114EB020035E4002030D000202F
:1012600057E4002034C6002060D0002048C9002088
:1012700030B5A5B000214822054668460CF0B6FFFF
:1012800000F046FB0146A0B9374C2378032B3AD92E
:1012900048220DEB02000CF0A9FF607870B13021FC
:1012A0000CF062FF044650B9304A012130480AF080
:1012B0004AFF304805F0B6FA25B030BD044629464D
:1012C000294814AA239400F061FFC11D034607D0EA
:1012D00001280BD90121284A25480AF036FF0BE0E6
:1012E0000A230221254A22480AF02FFF072312A8C9
:1012F0008DF8483000F040FB20460CF02AFF219882
:101300000CF027FFD5E7284600F0C4FD044630B1B5
:1013100010210CF029FF044608B9194AC5E72846F0
:1013200002A90F9400F0D6FDC21D034607D0012884
:1013300010D90121104A0E480AF007FF10E00221DF
:10134000104A0B480AF0FFFE0A2302210E4A084801
:101350000AF0FBFE072368468DF8003000F00CFB16
:10136000002CA6D02046CBE736E400205B0B030020
:1013700014EB020090C90020E90B0300870B030067
:10138000130C0300400C0300AF0B030038B50C46F0
:10139000054640B931B30846F8F7ACF8082816D02E
:1013A0006FF0150012E0F8F7A5F80828F8D18CB115
:1013B0002046F8F79FF80828F2D129460B480CF090
:1013C0002CFF21460A480CF028FF002038BD074BAF
:1013D0001D70F6E7294605480CF01FFF0022044B5C
:1013E0001A70F2E7014B1970F8E700BFAFC7002091
:1013F000B8C7002010B538B31448F8F77BF8044696
:101400001348F8F777F8082C15D108280ED1104AA0
:101410000E49104803F074F938B1034601210E4813
:101420000E4A0AF092FE6FF00D0010BD07490C48FD
:1014300003F066F9F0E7082802D105490948F7E703
:10144000094803F05DF9E7E70848FAE7AFC700206D
:10145000B8C70020670C030014EB0200AE0C0300B9
:101460007E0C0300900C0300A30C0300811003000A
:101470000023F0B58DB00D460646CDE90333CDE926
:101480000633CDE909338DF814308DF820308DF80E
:101490002C3000285ED000295CD0304CA0212046A2
:1014A0002F4A237003F090F9034648B101212D4AD9
:1014B0002D480AF04AFE6FF00D0420460DB0F0BD35
:1014C00020462C210CF09CFE044648B96FF04C04D9
:1014D000F3E734B90121254A23480AF034FEF5E741
:1014E0000C27601C2C210CF08BFE013F0446F0D130
:1014F0000028EFD0811C082203A80CF0A8FE601C75
:101500002C210CF07DFE04460028E3D0811C08222B
:1015100006A80CF09CFE2C21601C0CF071FE00282B
:10152000D8D0811C082209A80CF091FE01AB09AAB1
:1015300006A903A800F064FA044630B1034601216D
:101540000B4A09480AF001FEB7E7019B3360029B92
:101550002B60B2E76FF01504AFE700BF95E3002002
:10156000DD0C0300EA0C030014EB0200070D03007E
:10157000210D03004FF0FF3307B5684601A9CDE9FF
:101580000033FFF775FF48B14D300AD00121064AFC
:10159000064803B05DF804EB0AF0D5BD6846FFF7D6
:1015A000DDFB03B05DF804FB4E0D030014EB0200FD
:1015B000002208B511460346034803F0A1F80028AD
:1015C00018BF6FF00D0008BD6C0D03002DE9F74F3B
:1015D00005230422CDE90023224B187090B922483C
:1015E00003F08EF8034648B1204A214801210AF051
:1015F000ACFD6FF00D0003B0BDE8F08FFFF75AFCB3
:101600000020F8E76D4600241A4E1B4FDFF86C806F
:1016100055F8049B1A4BB9F1040F14BFB246BA46F1
:10162000504614BFC3469B46F7F764FF042813D106
:1016300051465846F7F754FF40B1524649461148C3
:1016400003F05EF8034618B10F4ACEE7FFF7ACFB94
:10165000002CD5D10124DBE749460C4803F050F8B3
:10166000F0E700BF56E40020810D03008D0D03005C
:1016700014EB0200C1C70020C6C7002042E40020CE
:1016800047E40020B80D0300DB0D0300CC0D030080
:10169000014B1878FFF79ABF56E40020002313B5DA
:1016A00004460193D0B101AB0E490F480DF102027F
:1016B00003F050F9031E08DC0C4801210C4A0AF023
:1016C00044FD6FF00D0002B010BD019B00200133FE
:1016D0000CBF04239DF802302370F4E76FF015006F
:1016E000F1E700BF050E0300220E030014EB020019
:1016F0002C0E030038B5431E062B05460C4608D9B0
:101700000346124A124801210AF01FFD6FF015002E
:1017100038BD042902D90B460E4AF3E70E4B5A5C3A
:101720000E4B53F820100E4802F0EAFF40B103467A
:10173000012107480B4A0AF008FD6FF00D00E7E7AA
:10174000094B1D70094B1C70E2E700BF590E0300E6
:1017500014EB02007B0E03007110030000F1020085
:10176000A00E0300B60E0300AEC70020ADC70020D8
:1017700013B50446B0B10D490D480DF1060203F052
:10178000E9F80128034608D00A4801210A4A0AF06C
:10179000DCFC6FF00D0002B010BDBDF8063000207B
:1017A0002370F8E76FF01500F5E700BFDB0E0300CC
:1017B000E60E030014EB0200EF0E0300042838B518
:1017C000044619D804281CD8DFE800F0240A241B9A
:1017D00024000123154AAB4013421BD1012D10D127
:1017E000FFF724FB0346A8B10121114A11480AF072
:1017F000ACFC6FF00D0038BDA0F11405EDB2182D52
:10180000E7D90C48234601210B4A0AF09EFC6FF0F1
:101810001500F0E72146094802F072FF0028EAD0DF
:101820000121074A03480AF08EFCE2E7010C30016F
:101830002A0F030014EB0200540F0300700F030083
:101840007B0F0300F7B507460124294ED6E8EF3F8A
:10185000C6E8E24F002AF9D1002B46D10DF107006E
:10186000FFF71CFF054660B12146224A22480AF0D4
:101870006AFC6FF00D049DF80600FFF79FFF2546F8
:1018800029E09DF8073003F0FB03012B23D00DF175
:101890000600FFF76DFF0028EBD1184805F00CF8A3
:1018A0002046FFF78BFF04460028E4D19FB14FF09C
:1018B00096720023114804F0D9FF10F10B0F044673
:1018C00007D103210E4A0C480AF03DFC6FF0730467
:1018D000D1E70028CFD10023D6E8EF2FC6E8E13FBB
:1018E0000029F9D1284603B0F0BD6FF07605F9E77D
:1018F00038D80020B40F030014EB020048C90020C0
:10190000DE0F0300014804F01FBF00BFF8C800202D
:10191000024B1868B0FA80F04009704744D80020A4
:1019200070B50646124D4FF0FF324FF0FF331148AD
:1019300004F092FE2C6844B908200CF011FC48B960
:10194000FFF7E0FF6FF068000DE063689E4207D08C
:101950002468F0E7046046606B682BB9C5E90000B5
:10196000FFF7D0FF002070BD18606860F8E700BF87
:1019700044D80020F8C8002038B50F4C054623682D
:10198000C3B14FF0FF334FF0FF320C4804F064FE58
:1019900023680BB11C681BB9BDE83840FFF7B2BF24
:1019A00028465B6898471CB1226823461446F2E734
:1019B0002246FAE738BD00BF44D80020F8C800200E
:1019C00070B50E461446054600B132B901210A4AE7
:1019D0000A480AF0D6FB002070BD1046F7F78AFDD2
:1019E000B042F8D83246214628460CF0E2FBB0FA65
:1019F00080F04009F0E700BF8B10030014EB0200F9
:101A00002DE9F3411D46002307460E461446019377
:101A1000F7F770FD08281CD13046F7F76BFD082852
:101A200017D124B12046F7F765FD082811D1328877
:101A3000B378ADF804200021022201A88DF8063009
:101A400006F0E4FA072809D92C4A01212C480AF0AB
:101A500098FB6FF0150002B0BDE8F081294B02221F
:101A600053F820800021F01C06F0D0FAB8F1000FE6
:101A700012D14FF0FF332B609CB12288A378ADF8D0
:101A800004200021022201A88DF8063006F0BEFADB
:101A9000072815D91C4AD8E708FB00F02860013058
:101AA000EAD03A88BB78ADF804200021022201A8D0
:101AB0008DF8063006F0AAFA07280FD9134AC4E7B2
:101AC000134B53F820600EB9124ABEE702220021E0
:101AD000E01C06F09BFA70432860E2E70E4B0222FE
:101AE00053F820400021F81C06F090FA1CB1444342
:101AF00000206C60AFE74FF0FF34F9E7B01103004E
:101B000014EB020048F10200E5110300311203005A
:101B100068F102001112030068F102000023F0B521
:101B200085B007460D4602A804211646CDE90233CA
:101B30000AF0C9F9044640B103460121184A194880
:101B40000AF021FB204605B0F0BD014602AA384646
:101B50000AF094F9044648B10346134A012111489A
:101B60000AF011FB02A80AF0D8F9EBE7314601AA06
:101B700002A80AF084FA044610B103460B4AEDE7C6
:101B8000019B1BB1012B03D12B70EBE70346FBE755
:101B90000121074A03480AF0F6FA6FF01504E1E75D
:101BA000A410030014EB0200541203007F12030080
:101BB000A81203002DE9F0471D46002390B00393BF
:101BC000ADF810308DF812301646DDE9189807226E
:101BD000092382460F4605A80B21CDE900230AF010
:101BE00072F9044648B103460121784A78480AF060
:101BF000CAFA204610B0BDE8F087014605AA504653
:101C00000AF03CF9044648B10346724A0121704883
:101C10000AF0B9FA05A80AF080F9EAE701466B462E
:101C200003AA05A80AF057FA044610B103466A4A07
:101C3000ECE76A4A009903A8FFF7C2FE00284BD0E0
:101C40000DAAC7F1020105A80AF019FA041E6AD10B
:101C50000D9C052C44DC002C5ADB002E3ED1002DBF
:101C600068D125460024B9F1000F43D125F00405C1
:101C7000012DCFD1B8F1000FCCD000230825CDE93C
:101C80000733CDE90A338DF824308DF830304FF02A
:101C9000FF330295C8E90033002F40F08D802946BC
:101CA0000DEB050307AA05A80AF015FA0921044659
:101CB0000AAA02AB05A80AF00EFA50EA04020BD1F8
:101CC00043460AA907A8FFF79BFE034620B101215E
:101CD000434A3F480AF057FA00249BE73470BEE7B6
:101CE0005A2C15D106B13470002D5AD1B9F1000F1C
:101CF000F2D05A250AAAC7F1050105A80AF0BFF9D2
:101D0000002857D19DF82830002489F80030ADE72D
:101D100023460121334A2E480AF035FA6FF01504A4
:101D20002346314A72E7FBDB06B13470002D98D0B0
:101D30005A2C36D005A80AF0F1F9032836D9C7F194
:101D4000030101AB0DAA05A80AF0C5F90146D0B9F7
:101D5000019B102240336B4403F80C0C0DA806F0D5
:101D600055F90923E8600193C7F1040101AB0DAAFD
:101D700005A80AF0B0F9014640B14FF0FF33AB605F
:101D8000254604466FE74FF0FF30EAE7019B10223B
:101D900040336B4403F80C0C0DA806F037F9A8602B
:101DA0005FE74FF0FF33C5E902339FE74FF0FF30A5
:101DB000E860F4E70023A7E7072102AB07AA05A81C
:101DC0000AF089F92946044672E700BFA41003000F
:101DD00014EB0200C4120300F112030039100300D7
:101DE000210D03001A1303002C0E0300002373B50A
:101DF00006460D46CDE9003300293BD0002839D0F6
:101E0000042168460AF05FF8044640B10346012108
:101E10001A4A1B480AF0B7F9204602B070BD0146C5
:101E20006A4630460AF02AF8044648B10346154A85
:101E3000012113480AF0A7F968460AF06EF8EBE7AB
:101E40002A46022168460AF032F9044610B10346D8
:101E50000D4AEDE70D49D5E9003299424FF00803EC
:101E60009341E9D202210A4A05480AF08AF96FF043
:101E70001504E1E76FF01504CEE700BFA4100300DE
:101E800014EB0200421303006F13030000E09950AB
:101E90009C13030008B530B901210C4A0C480AF024
:101EA00070F9002008BD0023013810F8012F2C2AFA
:101EB00001D10133F9E7002AF7D10A2BF1D9A3F1B7
:101EC00009000523B0FBF3F0ECE700BFC9130300E2
:101ED00014EB02002DE9F0430B230D4600210746C9
:101EE0008DB0CDE909110493CDF82B10421E12F8E4
:101EF000013F2C2B01D10131F9E7002BF7D185F8F7
:101F000030304FF0FF330331AB6007A809F0DBFF3F
:101F1000044648B103460121974A98480AF033F92C
:101F200020460DB0BDE8F083014607AA384609F007
:101F3000A5FF044658B1C31D15D00346904A0121A0
:101F40008E480AF020F907A809F0E7FFE8E70646FF
:101F5000002104AB09AA07A80AF0BDF8044620B185
:101F60000346884AEBE70126F2E7874A049909A865
:101F7000FFF726FD002800F0A580012101AA07A88F
:101F80000AF07DF804460028DDD1019B002B40F0CB
:101F9000F080022102AA07A80AF01DF904460028D1
:101FA000D1D1029B4FF00708B3F1805FA4BF4FF07F
:101FB000FF330293029B0321AB6005AA03AB07A882
:101FC000CDF80C800AF087F804460028BBD1039BAB
:101FD0000A2130336B4403F81C0C2A1D0DF1170045
:101FE0000AF0D3F804460028ADD18DF817002A4630
:101FF0000A2105A80AF0C9F804460028A3D1042143
:1020000002AA07A80AF0E7F8044600289BD1029B21
:102010000521EB6002AA07A80AF031F8044600285F
:1020200091D1029B0621AB8205F1100207A80AF0AC
:1020300026F80446002886D1414605F1280207A863
:1020400009F0E9FF044600287FF47DAF082102AAC9
:1020500007A80AF014F8044600287FF474AF029B26
:1020600009216B8502AA07A80AF009F8044600288E
:102070007FF469AF029B0A21AB8505F1200207A816
:102080000AF015F8044600287FF45DAF3846FFF7E4
:1020900001FF85F83000C0B200EB800000F10B04B6
:1020A00007A80AF03BF884420ED2214605F1180237
:1020B00007A809F0FCFF044600287FF444AF95F818
:1020C000303033B900243EE700220023C5E906235F
:1020D000F5E76B6B002BF5D00F274FF0000895F854
:1020E0003030984504D3002EECD06FF006042AE778
:1020F0006A6B391F02EB081207A809F0C0FF4FEA0C
:102100000819044600287FF41EAF6A6BF91E4A4482
:10211000083207A809F07FFF044600287FF413AFB8
:1021200002AAB91E07A809F0AAFF044600287FF4F6
:102130000AAF6B6B029A4B445A81791E02AA07A818
:1021400009F09DFF044600287FF4FDAE6B6B029AF8
:102150004B449A816A6B39464A44043207A809F015
:102160008EFF0537044600287FF4EDAE08F1010824
:10217000B5E70124E7E600BFA410030014EB02005A
:10218000F3130300F11203001710030000232DE9DD
:10219000F04F16460B220D469946A1B002AFC7E993
:1021A0000F33BA62F860C7F843304A1E12F8013F95
:1021B0002C2B02D109F10109F8E7002BF6D14FF0E1
:1021C000FF32302409F1030886F8383086F83030C1
:1021D000B260F9684978994215D8414607F1340050
:1021E00009F071FE0446C0B10346AF4A0121AF4871
:1021F00009F0C9FF07F1340009F08FFE20467C3753
:10220000BD46BDE8F08F04FB03F0F16B01330144E0
:102210008A60F16B01448A82DBE7014607F13402F0
:10222000284609F02BFE044648B3C31D02D00346DE
:102230009F4ADBE7EA468AB002AA9E4BC2E907053D
:10224000C2E9053840F2024393849B4B42F8103FA9
:1022500000234FF432519548F9F716FF0123D54674
:102260007B61002107F1280307F13C0207F13400EC
:1022700009F031FF044620B10346904AB6E7786181
:10228000EFE78F4AB96A07F13C00FFF799FB386125
:1022900030B901218B4A854809F073FF0024A9E772
:1022A000012107F11C0207F1340009F0E8FE0446A1
:1022B00000289FD1FC69012C9CD0022C04D121461E
:1022C000814A7A4809F05DFF4FF0000A0125D046A7
:1022D000A9F10A037B607B68AB4203D9FB685B789A
:1022E00043450CD87B69002BD8D06FF00603012141
:1022F000764A6E4809F047FF6FF006047AE705F169
:102300000109494607F1200207F1340009F063FF93
:10231000044690B16D468AB002AA6D4BC2E90780AF
:10232000C2E90539052342F8103F00234FF421513B
:102330005E48F9F7A9FEAD465CE73B6AB3F1805F02
:1023400007DB0221634A594809F01DFF4FF0FF33B4
:102350003B623B6A07F12C023B650723A91C7B62A9
:1023600007F1340007F1240309F0B5FE044610B16B
:102370000346594A3AE77B6A07F11802603313446F
:1023800003F84C0C0A2107F14C0207F12F0009F069
:10239000FCFE044610B12346504A27E787F82F0079
:1023A0000A2107F1480207F12C0009F0EEFE04466D
:1023B0000028F0D107F12002E91C07F1340009F0F0
:1023C0000AFF044638B1012100904346444A374889
:1023D00007F0C8FA0EE73B6A07F12002291D07F152
:1023E00034007B6509F04BFE044610B103463D4ABC
:1023F000FCE63B6A07F16002691D07F13400A7F8AB
:102400005C3009F054FE044610B10346364AEDE64E
:1024100007F15802A91D07F1340009F030FE044607
:1024200010B10346314AE1E607F17002E91D07F1F8
:10243000340009F0F0FD044610B103462C4AD5E6FD
:1024400007F1720205F1080107F1340009F0E3FD1C
:10245000044610B10346274AC8E607F1740205F1A5
:10246000090107F1340009F0D6FD044610B1034616
:10247000214ABBE607F1680205F10A0107F13400C1
:1024800009F015FE044610B103461C4AAEE607F1FA
:102490001A0205F10B0107F1340009F0BCFD0446F6
:1024A00080B30346164AA1E62514030014EB02008C
:1024B000F31303005C14030005000001F112030094
:1024C0001710030099140300B814030070180300D8
:1024D000EF140300211503006415030084150300A5
:1024E0009D150300D3150300FD15030031160300ED
:1024F000531603007B1603009B160300BB16030054
:10250000E01603000C35294607F11A0207F13400E2
:10251000B7F91A9009F07FFD044610B10346514AFD
:1025200064E6B9F1000F00F08580B44607F1480E6B
:10253000BEE80F00ACE80F00BEE80F00ACE80F00EB
:102540009EE80F0097F81A908CE80F00B9F1000F81
:102550001DD0B9F10A0F15D90A240A230221424AD3
:10256000424809F010FE3B697B61102120460BF0C8
:10257000FBFD48B902213E4A3C4809F002FE08F141
:102580000108A8E64C46F0E7706386F830404FF04B
:102590000009BC60BB684B45F1D0726B691C02EB53
:1025A000091207F1340009F06AFD4FEA091B0446DD
:1025B00010B103462F4A19E6726BA91C5A4408321F
:1025C00007F1340009F027FD044610B103462A4AFA
:1025D0000CE607F12002E91C07F1340009F04FFD79
:1025E000044610B10346254A00E6736B3A6A5B4421
:1025F0005A81291D07F1200207F1340009F03FFD3F
:10260000044610B103461E4AF0E5736B3A6A5B4418
:102610009A81726B05355A442946043207F1340019
:1026200009F02DFD044610B10346164ADEE509F116
:102630000109AFE73023F46B07F1480C03FB0A44B0
:10264000BCE80F000FC4BCE80F000FC49CE80F00EB
:1026500084E80F0096F838300AF1010A013386F851
:1026600038308CE7031703002D17030014EB02002A
:1026700085170300B9170300DD17030007180300CF
:10268000291803004B1803007FB5002306460D46AA
:10269000CDE90233002947D0002845D0042102A803
:1026A00009F011FC044640B103460121204A2148AB
:1026B00009F069FD204604B070BD014602AA30460B
:1026C00009F0DCFB044630B103461B4A01211948DE
:1026D00009F059FD18E001210DF1060202A809F0E8
:1026E000B6FC044610B10346144AEFE7BDF80630C5
:1026F00002A82B7009F012FD022809D84FF0FF3212
:102700004FF0FF33C5E9022302A809F006FCD1E728
:10271000022105F1080202A809F0C9FC04460028BC
:10272000F2D00346064AD1E76FF01504C2E700BFB6
:10273000A410030014EB02009C180300CE18030041
:10274000F7180300F8B50E460446F0B1E9B10821C8
:102750000F4AFFF735F938B90E4801210E4A09F042
:1027600010FD6FF00400F8BD00250C4F0834214621
:1027700057F8040BF6F7B4FE08B93570F3E70135E6
:102780000A2DF4D16FF03C00EDE76FF01500EAE799
:102790002C19030014EB02003519030020F102008C
:1027A00070B5064C064EC5B2B44200D370BDD4E934
:1027B0000031284698470834F6E700BF241F03007D
:1027C000241F030010B515491548FEF7DFFD034629
:1027D00030B1144A0121BDE81040134807F0B8B8E1
:1027E000FEF708FE044610B1104A0346F2E7FEF772
:1027F000DFFE01210E4801F083FF2046FEF7E6FED2
:10280000034608B10B4AE5E701460B4801F078FFA3
:10281000034608B1094ADDE710BD00BFF419030003
:10282000FD190300061A030014EB0200271A030027
:10283000471A03005A1A03007B1A0300861A030082
:10284000034610B530B10A4A0121BDE810400948DD
:1028500007F07EB8084B1978084B1878FEF74AFF46
:10286000034608B1064AEFE7BDE81040FFF7AABFEC
:10287000A61A030014EB0200ADC70020AEC700206B
:10288000DB1A030010B50749074809F0CBFC0446E2
:1028900028B101210346054A054807F059F82046AA
:1028A00010BD00BF012B02004CD80020111B0300FB
:1028B00044EB02002DE9F041DFF8D4810D46D8F851
:1028C000704000AF072C00F008065BD0132C00F01E
:1028D000A080052C40F0B980D8F854806D496E482E
:1028E00009F09CFC18F4805F41D06C496A4809F0FB
:1028F00095FC172418F4006F04D06949664809F064
:102900008DFC182418F4007F0ED06649624809F047
:1029100085FC654B18F4004F9B6B04D00121634A82
:102920005D4807F015F8192418F4806F04D0604949
:10293000594809F073FC1A2418F4807F19D05D49B6
:10294000554809F06BFC1B24EB69002E40F09B807E
:10295000C3F3080222B96FEA53236FEA4323EB6102
:1029600029462046F9F75CFEBD46BDE8F0811624F5
:10297000C0E718F4005FE7D04F49474809F04EFC24
:102980001C24E1E7D8F85C4043484C4909F046FC78
:10299000600606D5D8F868300121494A3E4806F05D
:1029A000D7FFE10705D547493B4809F037FC262406
:1029B000CAE7A20705D54449374809F02FFC272468
:1029C000C2E7630705D54149334809F027FC2824AD
:1029D000BAE7200705D53E492F4809F01FFC2924F6
:1029E000B2E7E10605D53B492B4809F017FC2A243C
:1029F000AAE7A20605D53849274809F00FFC2B2481
:102A0000A2E723063DD53549234809F007FC2C24CD
:102A10009AE7D8F86C8032491F4809F0FFFB18F09C
:102A2000020F03D02F491C4809F0F8FB18F0010FE2
:102A300003D02D49184809F0F1FB18F0040F83D09A
:102A40002A49154809F0EAFB7EE7294A294BE8465E
:102A50008AB00F2CC8BF13466A462749103CC2E90A
:102A600005134FF400731384244BD46142F8103FD4
:102A700000234FF411510848F9F706FB0024C5461E
:102A800062E7252460E723F4FF7323F0010366E780
:102A90004CD800202401030044EB02003A0103005B
:102AA0009EFF02004B01030000ED00E06401030003
:102AB0007901030094010300FEFF02004B1B030099
:102AC000641B0300741B03008A1B0300A81B030084
:102AD000C31B0300E01B0300F51B03000F1C0300D6
:102AE000221C03003C1C03006C1C03009A1C030006
:102AF000C1010300AC010300A202030004000001B5
:102B000000B5104B89B05A6AD86C00929A6A20F0CE
:102B100005000192DA6A694602921A6B03925A6BB7
:102B200004929A6B0592DA6B06921A6C1B6D0792EF
:102B30009B0748BF40F00400FFF7BCFE09B05DF8FA
:102B400004FB00BF4CD800202DE9F0411F46164B76
:102B5000044693F800800D461646A2B0B8F1000F67
:102B600015D1684606F0BDFF3A4631462846289BF7
:102B7000A0470446684606F0B5FFB8F1000F02D042
:102B80000A4803F0E1FD204622B0BDE8F0814FF095
:102B9000FF324FF0FF33054803F05EFD0028E0D020
:102BA0006FF08304EFE700BF64E4002034C9002025
:102BB000002300B589B0CDE9063303AB04930423A9
:102BC00003900593A9B10B6806934B680793022302
:102BD000111E18BF01210848CDE9002140F2F5314E
:102BE00004AA00F02BF80028B8BF012009B05DF856
:102BF00004FB0123ECE700BF0501004070B5382657
:102C000094B006AB05460C463246002118460BF040
:102C1000EDFACDE90454CDE9020654B1012304AA2A
:102C2000009200210448019302AA00F007F814B0B2
:102C300070BD2046FBE700BF0001004010B4B1F5B5
:102C4000004F029C0ED2042B0CD8042C0AD824046A
:102C500044EA0364134644EA0102014610BC0348F7
:102C6000FFF772BF6FF0800010BC7047217C01003D
:102C700030B50468ACB1B4FA84F30122C3F11F0388
:102C8000DBB29A4024EA0202D0E8EF5FA54204D109
:102C9000C0E8EC2FBCF1000FF6D1EAD102480B706E
:102CA00030BD0248FCE700BF0000AD0B0200AD0BD9
:102CB00010B50368CB40DB0710D401238B400268BA
:102CC00043EA0201D0E8EF4F944204D1C0E8EC1F80
:102CD000BCF1000FF6D1F2D1014810BD0148FCE76C
:102CE0000000AD0B0400AD0B014BC3F804057047A9
:102CF00000700140F7B5044618B1012822D003B096
:102D0000F0BD0222264B0646C3F808230122DA60F2
:102D1000C3F80401D3F80431012342F21075204FA7
:102D20008DF80730D4B1012CE9D1D7F80C3403F475
:102D3000803386BB002BE2D0012009F0A0FA013DD0
:102D4000F3D1DCE70022164B0DF10706C3F80803A8
:102D50005860C3F80021D3F80031DDE7D7F8183404
:102D600003F480333EB9002BC9D0012009F087FA63
:102D7000013DF3D1C3E7D7F8182402F00302327003
:102D8000002BBCD09DF807000128B8D109F077FAD4
:102D9000013DC7D1B3E7D7F80C2402F00102EEE7FA
:102DA00000500040044B1A7922B9012218601A71B0
:102DB0000248704702487047C0D800200000AD0BA1
:102DC0000C00AD0B08B5074B1B6833B10520F9F7B4
:102DD000DDFF10B90520F9F7B7FF0122024BC3F858
:102DE000182508BDC0D800200050004010B510B113
:102DF000012848D010BD294BD3F81814D3F8182453
:102E0000C90324D502F00303022B05D0012B02D005
:102E10000020FFF76FFF0123204A0220C2F8183577
:102E200008224FF48273002103F1804303F5A0438D
:102E300019601C68012402F1804202F5A04214606E
:102E4000174A12681AB3154BC3F80403D2E7D3F834
:102E50001424D207DFD5D3F81C2402F00302013A70
:102E6000012AD5D80E4A12681AB10222C3F80423E7
:102E7000C0E7D3F80421002AFBD00022C3F80421C4
:102E8000D3F80431B6E700224FF48073CBE71A6819
:102E9000002AFCD019601B68ACE700BF005000405E
:102EA000C0D8002010B5164BD3F8002152B1002035
:102EB000C3F80001D3F800210122C3F80823114B05
:102EC0001B6898470E4BD3F8042182B10022C3F847
:102ED0000421D3F80421D3F81824D3F818240221AC
:102EE00002F00302012A03D1C3F818159A6010BD3D
:102EF000C3F80813034B0120BDE810401B681847B6
:102F000000500040C0D8002001460148FFF7B0BE85
:102F100044C60020036803F01F025B0902600248F8
:102F200018BF0020704700BF0025844070B43224D1
:102F30000279184B624352FA81F2083233F8124098
:102F4000E10524D5C4F3432124F4F85423F81240B6
:102F500064240026027904FB02340E3434F8025F44
:102F600015F4807F03D0C5F34325A9420FD0013665
:102F7000202EF3D164240025624302EBC1029D5050
:102F8000027904FB023070BC5830FFF791BE70BC70
:102F9000704700BF48C6002032235843034B50FA05
:102FA00081F1083133F81100400B704748C600200A
:102FB00032235843054B50FA81F1083133F81100A0
:102FC00080F00200C0F34000704700BF48C60020F8
:102FD00032235843044B50FA81F1083133F8110081
:102FE000C0F34010704700BF48C60020024611F0F1
:102FF000010004D003490B6A13600B6203B900207F
:10300000704700BF00258440F0B50546002001262A
:10301000044607468C420BD1114BD3F87C2132B1C8
:103020000022C3F87C21D3F87C3140F00040F0BD91
:10303000E3B29B0003F580729B0806FA03F31D427E
:103040000BD002F1804202F54432D2F800C0BCF14C
:10305000000F02D01760126818430134DAE700BF8E
:10306000001003402DE9F3470546544B296DD3F872
:103070000403C0B240F00040FFF7C6FF061E18DA96
:1030800000236846E96D00934FF00108FFF7AEFF9B
:1030900095F85C30DA0758D4296D4FF00040FFF7FF
:1030A000B3FF6846E96DFFF7A1FF0028F0D126F0D5
:1030B00000460124002E68D102B0BDE8F08794FAE2
:1030C000A4F4B4FA84F4E00804F1080335F813908A
:1030D00004F007021DF8003008FA02F223EA0203A6
:1030E0000DF8003001A80194FFF714FF019B4FEA8F
:1030F0009901803350F82370C9F3820A4B07D146F7
:10310000C7F3014725D552462846214609F01AF94A
:1031100001A80194FFF7FEFE019BFFB2803350F837
:103120002330C3F301439F4207D10021204609F019
:10313000FAF83946204609F0F6F801A80194FFF79D
:10314000E9FE019B08FA03F30362009C002CB6D150
:10315000A2E7022F0DD10321204609F0E4F80AF07E
:103160000503012BE9D14A462146284609F0EAF831
:10317000E3E70221204609F0D6F8BAF1030FF2D0B6
:10318000032FDAD1BAF1020FECE796FAA6F3B3FAFD
:1031900083F304FA03F29B0003F1804303F5443305
:1031A000D3F8101526EA0206D3F810252846C2F3F4
:1031B0000142C1F3042109F0C5F87BE70010034088
:1031C00032222DE9F3410379214F534353FA81F31E
:1031D000083337F813300546DB070C46CEB234D53A
:1031E00009F0CDF895F8048021464046FFF7F0FE3F
:1031F00060B121464046FFF7CFFE2A6800B202EBDD
:1032000080030022C3F81025C3F810252846214664
:10321000FFF78CFE32222B7901A802FB0366002304
:10322000083627F816300194FFF774FE019B00EB77
:103230008300D0F80022074B134043F00203C0F88C
:103240000032054802B0BDE8F0810448FAE700BF4B
:1032500048C60020F0F8FCFF0000AD0B0400AD0BE9
:103260002DE9F043D2F8009004460D46164685B08D
:10327000B9F1000F34D032220079DFF8D081424317
:1032800052FA81F2083238F81230CFB29B0703D5D8
:10329000FFF79EFE00283BD100230DF10F02CDE980
:1032A00000338DF80E308DF80F300DF10E014B46C6
:1032B000284608F0EFFF3221237901FB037308331E
:1032C00038F8132022F0020228F81320237901FB9A
:1032D0000377083738F8173043F0010328F8173020
:1032E0007368002B43D04FF0320C22791F780CFB0F
:1032F00002F2D3F804E052FA85F2544B083233F864
:103300001200E9B210F0020F04D0BEF1000F18D085
:103310004F482FE020F4604020F0200023F81200F6
:10332000BEF1000F0DD0032FF2D8726850682268EA
:1033300090F800E002EB8E02FFB9C2F81075C2F8F7
:1033400010754FF0320C22790CFB0212083233F860
:10335000120020F01C0023F8120022790CFB02114D
:10336000083133F8112042EA870223F81120B368AC
:1033700063BB384805B0BDE8F083D2F8108528F06B
:103380000308C2F81085226802EB8E00D0F81025E1
:1033900022F4473222F44072C0F810252A02D0F8F5
:1033A000108502F4F85242EA074242EA0802C0F8E5
:1033B000102522790CFB0212083233F8120040EA81
:1033C0004E3040F0200023F81200BAE72946D3E936
:1033D00000872046FFF7AAFDB8F1000FC9D064238B
:1033E00020791A4E4343F218F358984504D1536894
:1033F0009F4201D100210CE0642303FB00600DF12A
:103400000F015830FFF734FC124B9842B2D19DF8AF
:103410000F1064222379534303EBC10346F8038062
:1034200023795343322203EBC10333445F60237992
:10343000534353FA85F3083336F8132042EA412206
:1034400042F4807226F8132093E700BF48C600209C
:103450000400AD0B0000AD0B2DE9F04305460C4612
:103460001F4685B09AB306793046FFF7A1FD20B11B
:1034700021463046FFF7ACFD80BB32235E43DFF8C8
:10348000FC9056FA84F6083639F816305FFA84F85C
:1034900013F01C0F02D05378012B1FD001238DF89D
:1034A0000F3000232046CDE900230DF10F01931CBE
:1034B000013208F0EFFE32222B7902FB038808F17B
:1034C000080839F8183043F0030329F81830002FA2
:1034D00051D021462879FFF76BFD18B1284805B077
:1034E000BDE8F0833E782B68244903EB8603C3F8DC
:1034F0001005C3F8100532202B794FEA860C4343A0
:1035000053FA84F3083331F813E0E2B22EF4604E3C
:103510002EF0200E21F813E097F801E0BEF1000F25
:1035200029D02B68BF789C44DCF810354FEA0E4E4A
:1035300023F4981323F4F853CCF81035230203F442
:10354000F8530EF4403E3F05DCF8108543EA0E03C5
:1035500007F480173B4343EA0803CCF810352B7976
:1035600000FB0322083231F8123043EA463343F0BD
:10357000200321F812300348B1E700BF48C60020FD
:103580000400AD0B0000AD0B30B564250479044B8D
:1035900005FB0434A160017905FB0133DA6030BD1D
:1035A00048C6002038B505790C462846FFF710FDBF
:1035B00058B132235D43064B55FA84F4083433F88E
:1035C000143004485B0B137038BD0348FCE700BFA0
:1035D00048C600200000AD0B0400AD0B2DE9F04102
:1035E000064607796420184D00FB075898F860409C
:1035F00044BB40462146402210300AF0F7FD2146E8
:103600003068D8F850608E4212D10023C0F87C3167
:10361000D0F87C3140F30730F9F796FB642303FBC5
:1036200007550123094885F86030AB65BDE8F08196
:10363000CBB29B0003F580727C2B04BF845083586F
:103640000131E0E70248F1E748C600200000AD0B79
:103650000C00AD0B64210279044B01FB023393F89B
:103660006000003818BF0120704700BF48C6002026
:1036700064235422007913FB002302481844FFF707
:1036800017BB00BF48C6002064235422007913FBF7
:10369000002302481844FFF7EBBA00BF48C60020D9
:1036A00073B503680D46D3F8041306460029A4BF7A
:1036B0004FF00041C3F80413047929462046FFF770
:1036C00087FC00B329462046FFF772FCD8B1294693
:1036D0002046FFF761FC002501B23468890001F53E
:1036E0008073E550E35833680B44D3F8101541F06C
:1036F0000101C3F8101522B1012332688340C2F8DA
:10370000043302B070BD32235C43104B54FA85F48D
:10371000083433F81430C3F38203042B11D0052B83
:1037200011D001A80195FFF7F5FB019A0369D34079
:1037300003F00103991C284602B0BDE8704008F070
:10374000F2BD0321F7E70221F5E700BF48C60020DC
:103750000148FFF787BC00BFACC6002070B5084C1D
:103760000E462379154643B92A20F9F7EDFA0123CD
:10377000044823712660A56070BD0348FCE700BFC4
:10378000C8D800200000AD0B0C00AD0B002330B5F5
:103790000D4A50F8234003F5A2710133082B42F87B
:1037A0002140F6D10023084A00F11C0103F5B27450
:1037B00051F8045F0133082B42F82450F6D1036C12
:1037C000C2F8043330BD00BF00A0024038B5002469
:1037D000154D2A20C5F81045C5F81445C5F81845FB
:1037E000C5F81C45C5F82045C5F82445C5F8284549
:1037F000C5F82C45C5F89045C5F89445C5F89845D9
:10380000C5F89C45C5F8A045C5F8A445C5F8A84528
:10381000C5F8AC45F9F7A6FA4FF0FF33C5F8083301
:10382000024B1C7138BD00BF00A00240C8D8002068
:103830000123024A8340C2F80433704700A00240CB
:103840000123024A8340C2F80833704700A00240B7
:10385000F8B5012600270B4B0B4DD3F80C4304B9E8
:10386000F8BD94FAA4F0B0FA80F006FA00F324EA66
:103870000304064B82009F502B68002BEFD0A968F1
:103880009847ECE700A00240C8D8002000A1024001
:1038900010B4CC7B8A6803682CB9D1E90041C3F825
:1038A0000845C3F80C15C3F824252822037953438F
:1038B000054AD3582BB1006810BC40F30730F9F724
:1038C00043BA10BC704700BFD4D8002070B5817BCC
:1038D000E9B9046804F01F0364091AD140F20C65C9
:1038E000104A114E02EB8303D3F8001231402943F2
:1038F000C3F80012416801F01F0349090DD102EB22
:103900008303D3F8002232402A43C3F80022012067
:1039100070BD803351F82330FFDE803354F82330FC
:10392000FAE700BF00258440F0F8FCFF2DE9F041E4
:10393000074690F80480282000FB08F0144E0C463F
:10394000351895F82210F1B9A96032506B6085F8EE
:10395000251085F824106CB1A37B204685F827300C
:10396000FFF7B4FF88B1637B2146384685F82630DF
:10397000FFF78EFF282303FB08660123054886F81E
:103980002230BDE8F0810448FBE70448F9E700BFB6
:10399000D4D800200000AD0B0C00AD0B0400AD0B23
:1039A000062103680279C3F800152821034B01FBA7
:1039B0000233022283F82220704700BFD4D80020AF
:1039C000282102790B4B01FB023300219960026828
:1039D0000948C2F80803D2F8000220F4BC50C2F82B
:1039E0000002C2F80015012283F8241083F8222077
:1039F000704700BFD4D8002002029C012DE9F84F87
:103A000028239046002290F80490AE4D046803FBF2
:103A1000095383F823204B680E4633B1CB6803F07B
:103A20006043B3F1005F40F085813378023B012BA6
:103A300006D8336903F06043B3F1005F40F07A8148
:103A4000A14BC4F80833282303FB095393F824102F
:103A500001F0FF0239B19B68DFF870B2C4F804339B
:103A60005846BDE8F88F18F0140F0CBF0121002153
:103A700083F82410317809EB890783F820107178D6
:103A800005EBC70783F82110F168D96071681961E7
:103A900031695961B168C3F81C809961C8F300119C
:103AA00083F825107378C4F88835C4F86021D4F8F9
:103AB0006031C4F84821D4F84831C4F82421D4F83E
:103AC0002431C4F80421D4F8043118F0010318BFDC
:103AD0000123C4F8503518F0020318BF0123C4F8BD
:103AE00040353378032B00F2A480DFE803F07999A6
:103AF00062024FF48073C4F80032D7E90323C4F89C
:103B00004425C4F848350123A3604FF480112046B2
:103B100008F0A2FC0028F8D1D7E90523C4F8442511
:103B2000C4F8483528234FF4802203FB09539A60D8
:103B3000DFF89CB1282202FB09F218F0080AAB5802
:103B400005EB020013D13178032910D0012940F090
:103B500086802160002B6FD0282202FB09F2716859
:103B6000AA5821B9002A00F0BB80012262612822F4
:103B700002FB09F2A918AA58002A00F0B18018F037
:103B8000040F1CBF00228A6018F0400F06D12822C3
:103B900002FB0952916841F002019160282202FB68
:103BA0000952916841F4007191609268C4F804234D
:103BB00056E7D7E90323C4F84425C4F84835D7E9C4
:103BC0000523C4F83425C4F838354FF48453C4F8B9
:103BD0000032012323622823022203FB0953A6E7B4
:103BE00018F0200FD7E90323C4F8442514BF4FF47D
:103BF00080724FF40072C4F848354FF0280315BFA7
:103C0000C4F80022C4F800224FF48022022214BF1C
:103C100003FB095303FB09539A600123236287E7DF
:103C2000D7E90323C4F83425C4F838354FF480535A
:103C3000CDE7DFF8A0B07DE7026902B961612649EE
:103C4000DFF898A0204608F007FC012210F4007F5E
:103C500018BF626110EA0A0F1F49F3D07CE7012107
:103C6000A160002B7FF478AF006918B31B4B1AEAF0
:103C7000030F7FF471AF2046174908F0EDFB10F4F5
:103C8000007F8246F2D04FF08071204608F0E4FBBE
:103C9000D4F8001280B111F4007003D101228246E1
:103CA00022626261CB05E1D54FF48021204608F005
